:020000040800F2
:1000000000000220AD8F00081D8300082183000836
:1000100025830008298300082D83000800000000C4
:1000200000000000000000000000000081550108F1
:1000300031830008000000001156010875560108C0
:10004000FD8F0008FD8F0008FD8F0008DD8300088C
:10005000FD8F0008FD8F0008FD8F0008D183000888
:10006000FD8F0008AD160008FD8F0008FD8F000809
:10007000FD8F0008FD8F0008FD8F0008FD8F000830
:10008000FD8F0008FD8F0008FD8F0008FD8F000820
:10009000FD8F0008FD8F0008FD8F0008ED8300082C
:1000A000FD8F0008FD8F0008FD8F0008FD8F000800
:1000B00035830008FD8F0008FD8F0008FD8F0008C4
:1000C000FD8F0008FD8F0008FD8F000841830008A8
:1000D000FD8F00084D830008FD8F0008598300083C
:1000E000FD8F0008FD8F0008FD8F0008FD8F0008C0
:1000F000FD8F0008FD8F0008FD8F0008FD8F0008B0
:10010000FD8F000871830008FD8F0008FD8F000837
:100110007D830008FD8F000895830008FD8F00088F
:10012000FD8F0008FD8F0008FD8F0008A1830008E7
:10013000FD8F0008AD830008FD8F0008FD8F0008CB
:10014000FD8F0008FD8F0008FD8F0008B9830008AF
:10015000FD8F0008C5830008FD8F0008FD8F000893
:10016000FD8F0008FD8F0008FD8F0008FD8F00083F
:10017000FD8F0008FD8F0008FD8F000800000000C3
:08018000FD8F0008FD8F00084F
:1001900010B5054C237833B9044B13B10448AFF3C1
:1001A00000800123237010BD6006002000000000C5
:1001B000F034020808B5034B1BB103490348AFF301
:1001C000008008BD0000000064060020F034020832
:1001D00010F8012B11F8013B012A28BF9A42F7D0F1
:1001E000D01A7047034613F8012B002AFBD1181AC6
:1001F000013870470000000000000000000000000F
:1002000001F0FF01102A2BDB10F0070F08D010F8C7
:10021000013B013A8B422DD010F0070F42B3F6D1CB
:10022000F0B441EA012141EA014122F007047FF0E4
:1002300000070023F0E80256083C85EA010586EA3B
:10024000010685FA47F5A3FA87F586FA47F6A5FA77
:1002500087F68EB9EED1F0BC01F0FF0102F0070283
:1002600032B110F8013B013A83EA010313B1F8D12E
:100270000020704701387047002D06BF354603380F
:10028000073815F0010F07D1013015F4807F02BF48
:10029000013015F4C03F0130F0BC0138704700BF99
:1002A00081F0004102E000BF83F0004330B54FEA27
:1002B00041044FEA430594EA050F08BF90EA020F94
:1002C0001FBF54EA000C55EA020C7FEA645C7FEA27
:1002D000655C00F0E2804FEA5454D4EB5555B8BF4A
:1002E0006D420CDD2C4480EA020281EA030382EABB
:1002F000000083EA010180EA020281EA0303362D4D
:1003000088BF30BD11F0004F4FEA01314FF4801C1F
:100310004CEA113102D0404261EB410113F0004F31
:100320004FEA03334CEA133302D0524263EB4303E8
:1003300094EA050F00F0A780A4F10104D5F1200E86
:100340000DDB02FA0EFC22FA05F2801841F10001E1
:1003500003FA0EF2801843FA05F359410EE0A5F1B5
:1003600020050EF1200E012A03FA0EFC28BF4CF0E6
:10037000020C43FA05F3C01851EBE37101F000459C
:1003800007D54FF0000EDCF1000C7EEB00006EEBA9
:100390000101B1F5801F1BD3B1F5001F0CD3490833
:1003A0005FEA30004FEA3C0C04F101044FEA44528A
:1003B00012F5800F80F09A80BCF1004F08BF5FEA11
:1003C000500C50F1000041EB045141EA050130BDF1
:1003D0005FEA4C0C404141EB0101013C28BFB1F503
:1003E000801FE9D291F0000F04BF01460020B1FA4E
:1003F00081F308BF2033A3F10B03B3F120020CDA21
:100400000C3208DD02F1140CC2F10C0201FA0CF0FE
:1004100021FA02F10CE002F11402D8BFC2F1200C63
:1004200001FA02F120FA0CFCDCBF41EA0C01904019
:10043000E41AA2BF01EB0451294330BD6FEA040462
:100440001F3C1CDA0C340EDC04F11404C4F120024D
:1004500020FA04F001FA02F340EA030021FA04F35F
:1004600045EA030130BDC4F10C04C4F1200220FAB6
:1004700002F001FA04F340EA0300294630BD21FAF4
:1004800004F0294630BD94F0000F83F4801306BFBA
:1004900081F480110134013D4EE77FEA645C18BFAE
:1004A0007FEA655C29D094EA050F08BF90EA020F45
:1004B00005D054EA000C04BF1946104630BD91EA3D
:1004C000030F1EBF0021002030BD5FEA545C05D140
:1004D0004000494128BF41F0004130BD14F580047F
:1004E0003CBF01F5801130BD01F0004545F0FE41F3
:1004F00041F470014FF0000030BD7FEA645C1ABF28
:10050000194610467FEA655C1CBF0B46024650EA5E
:10051000013406BF52EA033591EA030F41F400218A
:1005200030BD00BF90F0000F04BF0021704730B510
:100530004FF4806404F132044FF000054FF00001E5
:1005400050E700BF90F0000F04BF0021704730B5A6
:100550004FF4806404F1320410F0004548BF40427B
:100560004FF000013EE700BF42004FEAE2014FEAD0
:1005700031014FEA02701FBF12F07F4393F07F4FAB
:1005800081F06051704732F07F4208BF704793F0AE
:100590007F4F04BF41F40021704730B54FF46074C1
:1005A00001F0004521F000411CE700BF50EA0102C4
:1005B00008BF704730B54FF000050AE050EA01026D
:1005C00008BF704730B511F0004502D5404261EBDD
:1005D00041014FF4806404F132045FEA915C3FF41E
:1005E000D8AE4FF003025FEADC0C18BF03325FEABB
:1005F000DC0C18BF033202EBDC02C2F1200300FA6C
:1006000003FC20FA02F001FA03FE40EA0E0021FA90
:1006100002F11444BDE600BF70B54FF0FF0C4CF47E
:10062000E06C1CEA11541DBF1CEA135594EA0C0F30
:1006300095EA0C0F00F0DEF82C4481EA030621EA6B
:100640004C5123EA4C5350EA013518BF52EA0335A6
:1006500041F4801143F4801338D0A0FB02CE4FF058
:100660000005E1FB02E506F00042E0FB03E54FF088
:100670000006E1FB03569CF0000F18BF4EF0010E80
:10068000A4F1FF04B6F5007F64F5407404D25FEA7C
:100690004E0E6D4146EB060642EAC62141EA55512F
:1006A0004FEAC52040EA5E504FEACE2EB4F1FD0C71
:1006B00088BFBCF5E06F1ED8BEF1004F08BF5FEAEF
:1006C000500E50F1000041EB045170BD06F00046A1
:1006D00046EA010140EA020081EA0301B4EB5C044E
:1006E000C2BFD4EB0C0541EA045170BD41F4801146
:1006F0004FF0000E013C00F3AB8014F1360FDEBF6B
:10070000002001F0004170BDC4F10004203C35DA46
:100710000C341BDC04F11404C4F1200500FA05F3C9
:1007200020FA04F001FA05F240EA020001F000426A
:1007300021F0004110EBD37021FA04F642EB0601E0
:100740005EEA430E08BF20EAD37070BDC4F10C040A
:10075000C4F1200500FA04F320FA05F001FA04F2CE
:1007600040EA020001F0004110EBD37041F10001BA
:100770005EEA430E08BF20EAD37070BDC4F12005C5
:1007800000FA05F24EEA020E20FA04F301FA05F22D
:1007900043EA020321FA04F001F0004121FA04F2D5
:1007A00020EA020000EBD3705EEA430E08BF20EAA5
:1007B000D37070BD94F0000F0FD101F000464000DF
:1007C00041EB010111F4801F08BF013CF7D041EA61
:1007D000060195F0000F18BF704703F00046520065
:1007E00043EB030313F4801F08BF013DF7D043EA36
:1007F0000603704794EA0C0F0CEA135518BF95EAEC
:100800000C0F0CD050EA410618BF52EA4306D1D172
:1008100081EA030101F000414FF0000070BD50EA91
:10082000410606BF1046194652EA430619D094EA1B
:100830000C0F02D150EA013613D195EA0C0F05D105
:1008400052EA03361CBF104619460AD181EA030159
:1008500001F0004141F0FE4141F470014FF0000011
:1008600070BD41F0FE4141F4780170BD70B54FF0AC
:10087000FF0C4CF4E06C1CEA11541DBF1CEA13552C
:1008800094EA0C0F95EA0C0F00F0A7F8A4EB05040E
:1008900081EA030E52EA03354FEA013100F0888005
:1008A0004FEA03334FF0805545EA131343EA1263CE
:1008B0004FEA022245EA111545EA10654FEA002683
:1008C0000EF000419D4208BF964244F1FD0404F53C
:1008D000407402D25B084FEA3202B61A65EB030598
:1008E0005B084FEA32024FF480104FF4002CB6EB55
:1008F000020E75EB030E22BFB61A754640EA0C00D5
:100900005B084FEA3202B6EB020E75EB030E22BF14
:10091000B61A754640EA5C005B084FEA3202B6EB55
:10092000020E75EB030E22BFB61A754640EA9C0014
:100930005B084FEA3202B6EB020E75EB030E22BFE4
:10094000B61A754640EADC0055EA060E18D04FEAA2
:10095000051545EA16754FEA06164FEAC30343EA42
:1009600052734FEAC2025FEA1C1CC0D111F4801F0F
:100970000BD141EA00014FF000004FF0004CB6E708
:1009800011F4801F04BF01430020B4F1FD0C88BFA7
:10099000BCF5E06F3FF6AFAEB5EB030C04BFB6EBB2
:1009A000020C5FEA500C50F1000041EB045170BDA5
:1009B0000EF0004E4EEA113114EB5C04C2BFD4EBD2
:1009C0000C0541EA045170BD41F480114FF0000E56
:1009D000013C90E645EA060E8DE60CEA135594EAD2
:1009E0000C0F08BF95EA0C0F3FF43BAF94EA0C0FD5
:1009F0000AD150EA01347FF434AF95EA0C0F7FF44A
:100A000025AF104619462CE795EA0C0F06D152EA9D
:100A100003353FF4FDAE1046194622E750EA410681
:100A200018BF52EA43067FF4C5AE50EA41047FF492
:100A30000DAF52EA43057FF4EBAE12E74FF0FF3CF7
:100A400006E000BF4FF0010C02E000BF4FF0010CC8
:100A50004DF804CD4FEA410C7FEA6C5C4FEA430C41
:100A600018BF7FEA6C5C1BD001B050EA410C0CBF90
:100A700052EA430C91EA030F02BF90EA020F0020F2
:100A8000704710F1000F91EA030F58BF994208BF59
:100A900090422CBFD8176FEAE37040F00100704716
:100AA0004FEA410C7FEA6C5C02D150EA013C07D16D
:100AB0004FEA430C7FEA6C5CD6D152EA033CD3D0B8
:100AC0005DF8040B704700BF8446104662468C46B2
:100AD0001946634600E000BF01B5FFF7B7FF0028E5
:100AE00048BF10F1000F01BD4DF808EDFFF7F4FF0E
:100AF0000CBF012000205DF808FB00BF4DF808ED99
:100B0000FFF7EAFF34BF012000205DF808FB00BFBB
:100B10004DF808EDFFF7E0FF94BF012000205DF8DD
:100B200008FB00BF4DF808EDFFF7CEFF94BF012092
:100B300000205DF808FB00BF4DF808EDFFF7C4FF8B
:100B400034BF012000205DF808FB00BF4A0011D22D
:100B500012F5001211D20DD56FF47873B3EB625217
:100B60000ED44FEAC12343F0004343EA505323FA23
:100B700002F070474FF00000704750EA013002D198
:100B80004FF0FF3070474FF0000070474FEA4102CE
:100B9000B2F1E04324BFB3F5001CDCF1FE5C0DD9DB
:100BA00001F0004C4FEAC0024CEA5070B2F1004F25
:100BB00040EB830008BF20F00100704711F0804F28
:100BC00021D113F13872BCBF01F00040704741F4ED
:100BD00080114FEA5252C2F11802C2F1200C10FAF1
:100BE0000CF320FA02F018BF40F001004FEAC123D5
:100BF0004FEAD32303FA0CFC40EA0C0023FA02F379
:100C00004FEA4303CCE77FEA625307D150EA01334E
:100C10001EBF4FF0FE4040F44000704701F000401E
:100C200040F0FE4040F40000704700BF80F00040FC
:100C300002E000BF81F0004142001FBF5FEA4103B4
:100C400092EA030F7FEA226C7FEA236C6AD04FEAB4
:100C50001262D2EB1363C1BFD218414048404140F9
:100C6000B8BF5B42192B88BF704710F0004F40F4AB
:100C7000000020F07F4018BF404211F0004F41F4C7
:100C8000000121F07F4118BF494292EA030F3FD093
:100C9000A2F1010241FA03FC10EB0C00C3F12003A6
:100CA00001FA03F100F0004302D5494260EB400035
:100CB000B0F5000F13D3B0F1807F06D340084FEAA0
:100CC000310102F10102FE2A51D2B1F1004F40EB95
:100CD000C25008BF20F0010040EA030070474900FD
:100CE00040EB0000013A28BFB0F5000FEDD2B0FA9A
:100CF00080FCACF1080CB2EB0C0200FA0CF0AABFBD
:100D000000EBC25052421843BCBFD040184370475A
:100D100092F0000F81F4000106BF80F40000013260
:100D2000013BB5E74FEA41037FEA226C18BF7FEA37
:100D3000236C21D092EA030F04D092F0000F08BF79
:100D40000846704790EA010F1CBF0020704712F060
:100D50007F4F04D1400028BF40F00040704712F19F
:100D600000723CBF00F50000704700F0004343F004
:100D7000FE4040F4000070477FEA226216BF08463A
:100D80007FEA23630146420206BF5FEA412390EAFD
:100D9000010F40F4800070474FF0000304E000BFF3
:100DA00010F0004348BF40425FEA000C08BF7047A4
:100DB00043F0964301464FF000001CE050EA010268
:100DC00008BF70474FF000030AE000BF50EA01027D
:100DD00008BF704711F0004302D5404261EB41016A
:100DE0005FEA010C02BF84460146002043F0B6438F
:100DF00008BFA3F18053A3F50003BCFA8CF2083AB4
:100E0000A3EBC25310DB01FA02FC634400FA02FCBC
:100E1000C2F12002BCF1004F20FA02F243EB0200C3
:100E200008BF20F00100704702F1200201FA02FC25
:100E3000C2F1200250EA4C0021FA02F243EB020018
:100E400008BF20EADC70704753B94AB9002908BFCF
:100E500000281CBF4FF0FF314FF0FF3000F0BEB94B
:100E6000ADF1080C6DE904CE00F03CF8DDF804E0CB
:100E7000DDE9022304B0704738B5002200230446A0
:100E80000D46FFF73BFE28B920462946BDE838400D
:100E900000F00AB8204605F1004100F005F8404294
:100EA00061EB410138BD00BFD0B50C4B00220646B6
:100EB0000F46FFF7B1FBFFF749FE0446FFF732FB91
:100EC000074B0022FFF7A8FB02460B463046394687
:100ED000FFF7EAF9FFF73AFE2146D0BD0000F03DEA
:100EE0000000F0412DE9F047089D8E4604468846F3
:100EF000002B4AD18A42174662D9B2FA82F64EB125
:100F0000C6F1200301FA06F820FA03F3B74043EADA
:100F10000808B4404FEA174E1FFA87FCB8FBFEF1F1
:100F2000230C0EFB118843EA084301FB0CF29A42A2
:100F300009D9FB1801F1FF3080F0EA809A4240F2B3
:100F4000E78002393B449A1AA3B2B2FBFEF00EFBD3
:100F5000102243EA024300FB0CFC9C4509D9FB1814
:100F600000F1FF3280F0D6809C4540F2D3803B44B4
:100F7000023840EA0140A3EB0C0300211DB1F3400D
:100F80000022C5E90032BDE8F0878B4205D90DB1DA
:100F9000C5E9000100210846F5E7B3FA83F100290D
:100FA00046D1734502D3824200F20581841A6EEB6A
:100FB000030201209046002DE5D0C5E90048E2E794
:100FC000002A00F09080B2FA82F6002E40F0A48051
:100FD0008A1A030C4FEA174E80B2BCB20121B2FB51
:100FE000FEFC0EFB1C2243EA024304FB0CF29A4275
:100FF00007D9FB180CF1FF3802D29A4200F2E080C8
:10100000C4469B1AB3FBFEF20EFB123340EA0343C5
:1010100002FB04F49C4207D9FB1802F1FF3002D214
:101020009C4200F2CA8002461B1B42EA0C40A5E724
:10103000C1F120068B4022FA06F71F430EFA01F495
:1010400020FA06F32EFA06FE4FEA1749234300FA68
:1010500001F81FFA87FCBEFBF9F01C0C09FB10EE2F
:1010600044EA0E4400FB0CFEA64502FA01F209D93F
:101070003C1900F1FF3A80F09C80A64540F299802F
:1010800002383C44A4EB0E041FFA83FEB4FBF9F3D0
:1010900009FB13444EEA044403FB0CFCA44508D9A5
:1010A0003C1903F1FF3E80F08280A4457FD9023BCA
:1010B0003C4443EA0040A4EB0C04A0FB02EC644572
:1010C0007346E14662D35FD05DB1B8EB030264EBD7
:1010D000090404FA06F622FA01F31E43CC40C5E9DE
:1010E000006400214FE7B1FBF2FC010C41EA0E4124
:1010F00080B240EA01423B4638463C46B846BE46CE
:101100002026B1FBF7F1A2EB080241EA0C4166E7A9
:10111000014618E710462CE7C6F120022EFA02F32A
:10112000B740B14020FA02F24FEA174E0A43B3FB30
:10113000FEF8BCB20EFB1833110C41EA034108FB68
:1011400004F9B04089454FEA104380B23ED979187E
:1011500008F1FF3C01D289451FD8A1EB0901B1FB81
:10116000FEF909FB04F80EFB191192B242EA0142A2
:10117000424529D2BA1809F1FF31C4D24245C2D240
:10118000A9F102013A44BEE7F0459DD2BEEB02034D
:101190006CEB070C0138E14696E7A7EB09094944D7
:1011A000A8F1020CB1FBFEF909FB04F8DBE773467A
:1011B0007FE7504666E70846FDE63B44023A33E7E0
:1011C000ACF1020C3B441CE749469CE7A1EB09014A
:1011D000C446B1FBFEF909FB04F8C4E7704700BF41
:1011E000044B026800211970D36843F02003D360D8
:1011F000704700BF8806002038B50B4C23784FF4A9
:101200001652054643F00103426023700DF02EF89C
:101210002A68D36843F08003D3602378DB07FCD4CB
:101220002078C0F3400038BD8806002010B4084C78
:101230000068237843F001032370064CC3682160E3
:10124000054943F080030A705DF8044BC3607047A2
:1012500088060020840600208206002030B554074E
:101260004FEAD20319D001334FF0FF0E01EB030C0C
:10127000013B13F0FF030CF801ECF7D1084C0068B8
:101280002378084D43F001032370C368064C29609E
:1012900043F080032270C36030BD002BE4D1EDE742
:1012A000880600208406002082060020E9B100B5EF
:1012B0008646084400211EF801CB08228CEA01036F
:1012C00043F3000323F0730383EA5101531E13F029
:1012D000FF02C9B24FEA5C0CF0D17045EBD1007847
:1012E000401A18BF01205DF804FB0078401A18BFAF
:1012F0000120704738B503681968DC688906024622
:1013000001D5A5062FD41968D8680C062AD5010680
:1013100028D55268B2F5165F49D04548027832B9EF
:10132000444C454924680A70444924780C70444967
:101330000978914245D0414C2178013211F00105E4
:1013400018BFFF25D2B25D604908530721700270B3
:1013500008D1394A3749137809680133DBB2137071
:10136000CB5C237038BD44685968B4F5165FC9B2C8
:1013700048D0344C344D20782B784008FF2908BFE2
:1013800040F0800020702E485A1C0078D2B2904263
:101390002A7002F007011BD00029E3D12B4B25490D
:1013A0001A78086824788454511C197038BDF022CA
:1013B0005A60DA681E49002022F080020870DA6064
:1013C00038BDDA68002122F080020170DA6038BD91
:1013D00002332278DBB239B103F00701013352083E
:1013E000DBB20029F8D12270184812490378096845
:1013F000CA5417490B78002262F300032A70027066
:101400000B7038BD124CB1F1F003217818BF0123E5
:1014100063F341014FF4E133217043600CF026FF88
:1014200023780949002262F300030A70237038BD53
:101430007E060020840600207D0600207C06002019
:101440008206002080060020810600207F06002002
:10145000880600200000000000B51F481F499FEDCE
:101460001A7B4FF4803285B00023C0E900120122BC
:10147000CDE90033CDE9023380ED0A7B836003615F
:10148000037680F82030C360C26180F8303042615A
:1014900007F090FE68B99FED0E7B00230E48029383
:1014A00069468DED007B08F011F828B905B05DF8AC
:1014B00004FB06F0D5F9EEE706F0D2F905B05DF8C9
:1014C00004FB00BFAFF300800100000F000000002C
:1014D0000A000000010000009006002000200140EA
:1014E00000B5194A016889B000239142CDE9023361
:1014F000CDE90433069302D009B05DF804FB02F590
:101500008C320093506C40F480705064506C00F446
:101510008070009000980193136B0C4843F0040313
:101520001363136B9FED067B03F00403019302A981
:101530008DED027B019B09F045F909B05DF804FBD4
:1015400001000000030000000020014000080240EC
:10155000064A08B5536943F008030920536108F0AF
:10156000DDF8BDE80840092008F0A6B8003C0140BD
:10157000092008F0AFB800BF10B4144B1B689A687C
:101580009207FCD50022DA609A68D407FCD5D968A6
:101590009A689007FCD50022DA609A68D207FCD5D9
:1015A000D8689A689407FCD50022DA609A68D20756
:1015B000FCD5DC6802020B0403F47F0392B2E0B2B4
:1015C000134318435DF8044B704700BFC8F7002071
:1015D00010B51D4C23787BB11C4BD3ED007AF4EE93
:1015E000C07AF1EE10FA08D9194BD3ED007AF4EE77
:1015F000C07AF1EE10FA13DA10BD164B012293E80F
:10160000030005F037FB144A0121042004F022FFF7
:10161000114A0121082004F01DFF0023237010BD92
:101620000C4B012293E8030005F024FB0A4A012138
:10163000042004F00FFF084A0021082004F00AFFEC
:101640000023237010BD00BF15BB00200000002048
:10165000F4BA00203C68020824F60020114A124B1C
:1016600010681B684FEA404CDA050CF0007C8102E0
:1016700002F0807242EA0C0201F08061114382059F
:1016800002F000620A43C1064FEA03704FEA834347
:1016900003F0005300F0404018BF42F0805218435E
:1016A0001043704728F6002024F600202DE9F0436F
:1016B0002DED028B954A964B964D974C4FF4007149
:1016C00083B0C2F880115A69110744BF08225A61D9
:1016D000FFF752FF296803464FF40050236004F0DF
:1016E000B3FE002840F0B28023688C4C8C4E1A0266
:1016F000D4E9002148BF43F07F43D21841EBE371A6
:10170000C4E90021874A3368126801339342336089
:10171000C0F08B80844F3B6801333B60834B1B7868
:10172000002B40F0AC80824B1B78002B40F0C28035
:1017300029684FF4005004F087FE002840F0AB8089
:101740007C4BDFF8309293ED008A7B4BD4E90001AB
:10175000D3ED008AFFF73AFB784B07EE900A93ED42
:10176000007A77EEC77A0022F5EEC07AF1EE10FA31
:10177000A8BF87EE880A4FF000034FF00008C4E9C5
:101780000023C6F80080B8BF87EEA80A89ED000ADA
:10179000FFF71EFF6A4B0120196804F055FE04464E
:1017A000002862D0674C684EFFF758FF236896F810
:1017B00000E0DFF8C4C1D9ED007A64493F684FF416
:1017C000B469DA0009FB0E229CF800E067F3170009
:1017D000013302EB0109C9ED017A23608850BEF1A3
:1017E000000F1ED05A4A126897421AD38CF8008014
:1017F00000F01CF9574B584A18683378013303F04E
:101800001F03337001A923681360C4F8008012F02D
:101810006DFC29684FF4805004F016FE002869D052
:1018200023684E4A12689A4250D9019B4BB14FF03F
:10183000E0234FF08052C3F8042DBFF34F8FBFF366
:101840006F8F03B0BDEC028BBDE8F08329684FF4C5
:10185000805004F0F9FD00287FF446AF404B02466B
:1018600093E8030005F006FA3EE700F0DFF83D4A92
:10187000137803F0FF01002B37D01470D5E7384BF5
:10188000002293E8030005F0F5F9294B1B78002BA3
:101890003FF44EAF0EE029684FF4805004F0D4FDC1
:1018A00000287FF44DAF2E4B012293E8030005F092
:1018B000E1F945E7092007F00DFF29684FF40050D2
:1018C00004F0C2FD00283FF43BAFE4E73278224841
:1018D00020490360531C03F01F03002208682260A4
:1018E00001A9337012F002FC9FE71F4B1A7832B146
:1018F00019709AE71D4B186813F000F990E71C4B1C
:1019000001A9186812F0F2FB8FE700BF00E100E0C8
:10191000003C014020F6002008BB002000BB002056
:1019200018BB0020040000201CBB002017BB0020B7
:1019300016BB0020ECBA0020E8BA0020F0BA002064
:1019400024F60020E0BA0020E4BA0020D8060020E7
:1019500010BB002014F60020DCBA0020D8BA00200A
:101960004C68020861BB002060BB002000F600202C
:1019700010F60020F8BA00200CBB0020174B10B561
:1019800093E80300012205F075F9154B154C93E817
:101990000300002205F06EF9134B002293E80300C8
:1019A00005F068F9114B012293E8030005F062F994
:1019B0000F4B002293E8030005F05CF994E8030064
:1019C000002205F057F90A2007F0E2FB94E8030033
:1019D0000122BDE8104005F04DB900BFA035020856
:1019E00098350208A83502089035020888350208A3
:1019F000B035020808B50A4BDA6822F00202DA6054
:101A00009A6842F002029A605A6942F00202072084
:101A10005A6107F083FEBDE80840072007F04CBE7E
:101A2000003C0140072007F055BE00BF08B5FFF796
:101A30009FFDFFF7F7FF08480CF008F9074B00225D
:101A400093E8030005F016F9BDE80840044A0021B8
:101A5000012004F0FFBC00BFB8F800204C68020869
:101A600024F600200000000038B5634C4FF480706D
:101A7000216804F0E9FC00285CD121684FF4005093
:101A800004F0E2FC0346002854D15C4A216813703C
:101A90004FF4805004F0D8FC0128594D06D0296835
:101AA000012004F0D1FCB0FA80F04009554B2968C0
:101AB0001870042004F0C8FC00287BD0524B002290
:101AC0001A7021684FF4805004F0BEFC01284DD1FB
:101AD0004E4B9FED4F6AD3ED006A9FED4E7A4E4B11
:101AE000C6EE267A67EE877AFCEEE77AC3ED007AD7
:101AF00004F0A6FA494B186004F030F94849494807
:101B0000494A00230B70494903600B609FED387B05
:101B100047494FF480500B60216882ED007B04F050
:101B200093FC012821682DD04FF4805004F08CFCE8
:101B300058B138BD21684FF4805004F085FCA0F105
:101B40000103B3FA83F35B099FE72168802004F067
:101B50007BFC002848D121684FF4807004F074FCAD
:101B6000002836D1BDE83840FFF7F2BC21684FF4B9
:101B7000805004F069FC0028BAD12E4A264B126826
:101B80001A60B5E7802004F05FFCF8B91F4B93EDB5
:101B9000000A04F067FA2168202004F055FC0128AF
:101BA000C7D12968202004F04FFC0128C1D1224B65
:101BB000187038BD21684FF4007004F045FC00280F
:101BC0003FF47CAF104B01221A707AE7FFF712FF47
:101BD000E1E71A4B002293E8030005F04BF8B3EE5F
:101BE000040A04F03FFABDE7FFF704FFB3E700BFC4
:101BF000000000000000000020F6002017BB0020BD
:101C000024F6002016BB002015BB002040BD00209C
:101C10000050C3476666663F04000020D8BA002023
:101C2000E4BA0020E0BA002000BB002018BB00206E
:101C30001CBB002048BD002014BB00204C680208DB
:101C400070B59A4C237882B000224F2B019211D0AC
:101C5000974D0120296804F0F7FB00286FD1237805
:101C60004F2B31D023783F2B7AD0012004F0C6FAD5
:101C700002B070BD6378462BEAD1A378462BE7D13A
:101C8000E678002EE4D1FFF773FCFFF7CBFE89481E
:101C9000874D894C0BF0DAFF884B324693E80300FE
:101CA00004F0E8FF01202A46314604F0D3FB216806
:101CB0004FF4805004F0C8FB01286CD08049814863
:101CC00004F08EFA02B070BD63784E2BCAD17E4B01
:101CD0001B78002BC6D12968012004F0B5FB002831
:101CE00040F09280774E744C33782168042B00F0DA
:101CF000B280012B216800F08B8021684FF4805066
:101D000004F0A2FB012800F08E8001210846684AF9
:101D100004F0A0FB6D496B480123052204F0BEF9D5
:101D200021684FF4805004F08FFB10B9684B0322F8
:101D30001A70642007F02CFAFFF796FE98E75E4EC3
:101D40001020316804F080FB002888D031684FF4FF
:101D5000805004F079FB012881D104F067FA87E70D
:101D60006378002B81D12968012004F06DFB58B9FC
:101D70002968012004F068FB002865D055495148C6
:101D800004F02EFA02B070BD534A524B92E80300A1
:101D900018601971F2E72168202004F055FB012832
:101DA0008CD12968202004F04FFB012886D14B4BB1
:101DB0001A78012A82D14A4A1E701368494C83F06E
:101DC0000103136004F030F8474B48491A6809686A
:101DD000474B1268474811F05DF8207000285BD12E
:101DE000444811F09BF92070002840F0BD80414824
:101DF00011F010FA01462070002840F0BE802C4AF5
:101E0000102004F027FB59E70B2004F0F7F92FE727
:101E10004FF4805004F018FB00287FF46EAF1A20B6
:101E200004F0ECF924E72168202004F00DFB0128E0
:101E300006467FF46AAF2968202004F005FBA8B9A4
:101E4000102004F0DBF913E72B4A224B92E8030041
:101E50001860998092E74FF4805004F0F5FA08B1C9
:101E6000337846E7072004F0C9F901E723481D4D00
:101E7000202103F0FBFF21491E480A2210F02CFD0F
:101E8000287000283ED01E4A3146022004F0E2FAB3
:101E90000C2004F0B3F9EBE6194A0121042004F008
:101EA000D9FA0E2004F0AAF9E2E600BF5CF50020A2
:101EB00024F60020B8F8002020F600204C68020824
:101EC000BC350208DEE100205EF500201C68020837
:101ED000DDE1002020BB0020CC35020814BB00202F
:101EE0006CBD002070DD002058BD00205CBD0020CE
:101EF00054BD002074DD0020D43502081CBC002035
:101F000028F6002003F0E6FF2048FEF76BF91F4992
:101F1000024601AB1E4810F0BDFF28700028BBD15F
:101F20001B4811F0FBF804462870E8B93146194AFD
:101F3000102004F08FFA184B184A19491C60194BED
:101F400014600C6030463146124A1C6004F082FA7C
:101F5000154916483346052204F0A0F8642007F01E
:101F600017F9FFF781FD83E6114A0121082004F0EB
:101F700071FA0F2004F042F97AE60D4A012110208F
:101F800004F068FA0D2004F039F971E670BD002004
:101F900074DD002024F6002064BD00206CBD00200C
:101FA00060BD002068BD00201C680208DEE1002042
:101FB00028F6002070B5174C0120216804F044FA7F
:101FC00028B1154D1020296804F03EFA70B9216837
:101FD000012004F039FA28B10F4B1020196804F0E1
:101FE00033FA70B1BDE87040FFF73EBD29684FF489
:101FF000805004F029FA0128E9D1BDE8704004F0CE
:1020000015B9064A0346BDE87040106819461A46DD
:1020100011F0F4BE24F6002020F6002010F6002077
:1020200038B523481DF0B7FC224B0446196801203F
:1020300004F00AFA20BB621E41F287339A421AD892
:102040001D4B1C4A1C600121084604F003FA1B4981
:102050001B4B096801224FF480501A7004F0F4F908
:1020600000B3184B022264201A7007F091F8BDE803
:102070003840FFF7F9BCBDE83840012004F0BEB895
:102080000E4D1020296804F0DFF90028D3D029680C
:102090004FF4805004F0D8F90128CCD1BDE8384085
:1020A00004F0C4B8084B186812F0CCFFD9E700BFA1
:1020B0005CF5002024F6002010BB002020F6002054
:1020C0000CBB0020DDE1002000F6002030B5544CB0
:1020D0008BB02168012004F0B7F9002834D1514BAE
:1020E0001A783F2A1BD01A784E2A40D02168012046
:1020F00004F0AAF9044600286AD109AA08ABCDE980
:1021000000324949474807AB06AA1EF047FC43B2D4
:10211000042B63D0012004F071F80BB030BD5A7865
:10212000002AE0D1414A4249D47890785378127815
:10213000CDE900043F481EF00FFC3E493E480BB07D
:10214000BDE8304004F04CB83C4D1020296804F044
:102150007BF90028C3D029684FF4805004F074F94B
:102160000128BCD10BB0BDE8304004F05FB85B780B
:10217000452BBBD1324B1A78572AB7D15B78002B4D
:10218000B4D1304B1A783F2AC4D15B78002BC1D12F
:1021900005AB4FF47A710422CDE90121009330227E
:1021A0000123A021284809F0E1F89DF816209DF8A8
:1021B00017401F499DF815301E48CDE900249DF8B1
:1021C00014201EF0C9FB1B491B4804F009F8A4E7C2
:1021D00003200BB0BDE8304004F010B8DDE9060183
:1021E000089A60F3070461F30F24099862F3174417
:1021F0004FF47A7105AACDE9002360F31F640291C0
:1022000001233022A0211048059409F013F8322050
:1022100006F0BEFF0D49084803F0E2FF7DE700BF6E
:1022200024F600205CF50020F035020854FA002066
:10223000DC35020820BB0020DEE1002020F6002073
:102240005EF500203CF50020A0F50020BC3502081A
:1022500030B5544C8BB02168012004F0F5F800280B
:1022600034D1514B1A783F2A1BD01A784E2A40D0CD
:102270002168012004F0E8F8044600286AD109AA80
:1022800008ABCDE900324949474807AB06AA1EF022
:1022900085FB43B2042B63D0012003F0AFFF0BB0EA
:1022A00030BD5A78002AE0D1414A4249D47890782A
:1022B00053781278CDE900043F481EF04DFB3E49AB
:1022C0003E480BB0BDE8304003F08ABF3C4D1020C3
:1022D000296804F0B9F80028C3D029684FF4805069
:1022E00004F0B2F80128BCD10BB0BDE8304003F0D7
:1022F0009DBF5B78452BBBD1324B1A78572AB7D19B
:102300005B78002BB4D1304B1A783F2AC4D15B786C
:10231000002BC1D105AB4FF47A710422CDE9012124
:10232000009334220123A021284809F01FF89DF8CA
:1023300016209DF817401F499DF815301E48CDE91D
:1023400000249DF814201EF007FB1B491B4803F0D6
:1023500047FFA4E703200BB0BDE8304003F04EBFB9
:10236000DDE90601089A60F3070461F30F24099878
:1023700062F317444FF47A7105AACDE9002360F3A4
:102380001F64029101233422A0211048059408F013
:1023900051FF322006F0FCFE0D49084803F020FFF3
:1023A0007DE700BF24F600205CF50020F035020830
:1023B00050FA0020DC35020820BB0020DEE10020BE
:1023C00020F600205EF500203CF50020A0F500205E
:1023D000BC35020830B5544C8BB02168012004F0A4
:1023E00033F8002834D1514B1A783F2A1BD01A7881
:1023F0004E2A40D02168012004F026F80446002827
:102400006AD109AA08ABCDE900324949474807AB70
:1024100006AA1EF0C3FA43B2042B63D0012003F0D6
:10242000EDFE0BB030BD5A78002AE0D1414A424956
:10243000D478907853781278CDE900043F481EF0A4
:102440008BFA3E493E480BB0BDE8304003F0C8BEB1
:102450003C4D1020296803F0F7FF0028C3D02968FD
:102460004FF4805003F0F0FF0128BCD10BB0BDE861
:10247000304003F0DBBE5B78452BBBD1324B1A7882
:10248000572AB7D15B78002BB4D1304B1A783F2A4A
:10249000C4D15B78002BC1D105AB4FF47A71042213
:1024A000CDE90121009338220123A021284808F01A
:1024B0005DFF9DF816209DF817401F499DF81530C7
:1024C0001E48CDE900249DF814201EF045FA1B4952
:1024D0001B4803F085FEA4E703200BB0BDE83040A5
:1024E00003F08CBEDDE90601089A60F3070461F38E
:1024F0000F24099862F317444FF47A7105AACDE9C5
:10250000002360F31F64029101233822A0211048A8
:10251000059408F08FFE322006F03AFE0D49084877
:1025200003F05EFE7DE700BF24F600205CF500208E
:10253000F03502084CFA0020DC35020820BB0020F0
:10254000DEE1002020F600205EF500203CF50020B2
:10255000A0F50020BC35020830B5644C8DB0216870
:10256000012003F071FF002833D1614B1A783F2A14
:1025700016D01A784E2A3FD02168012003F064FF5C
:10258000054600286FD121684FF4007003F05CFF0E
:1025900000286ED117200DB0BDE8304003F02EBEEC
:1025A0005A78002AE5D1534A534950791379D4789F
:1025B000CDE90230907853781278CDE900044F4885
:1025C0001EF0CAF94D494E480DB0BDE8304003F049
:1025D00007BE4C4D1020296803F036FF0028C4D0F8
:1025E00029684FF4805003F02FFF0128BDD10DB0B2
:1025F000BDE8304003F01ABE5B78452BBCD1424B9E
:102600001A78572AB8D15B78002BB5D13F4B1A788E
:102610003F2A3FD15B78002B3CD104AB4FF47A7159
:102620000622CDE90121009340220123A021384850
:1026300008F09CFE9DF815209DF814309DF813407D
:102640002D492E48CDE902329DF812209DF8113017
:10265000CDE900249DF810201EF07EF92749284876
:1026600003F0BEFD19E003200DB0BDE8304003F0DB
:10267000C5BD0BA80AA909AA08ABCDE90210CDE98E
:10268000003224491A4807AB06AA1EF087F940B267
:10269000062804D0012003F0B1FD0DB030BDDDE906
:1026A0000612089B61F3070562F30F25099A0A9940
:1026B0008DF8141063F317454FF47A7404ABCDE929
:1026C0000030029462F31F650B9C114804950123AE
:1026D0004022A0218DF8154008F0ACFD322006F014
:1026E00057FD0D49064803F07BFDD6E724F6002090
:1026F0005CF50020C8FA00200036020820BB00204C
:10270000DEE1002020F600205EF500203CF50020F0
:10271000A0F5002020360208BC35020830B5334C45
:1027200087B0002321680593012003F08DFE002867
:102730003DD12F4D2B783F2B2AD02168012003F06B
:1027400083FE002849D12B782A4AD35C5B073FD50A
:1027500027481DF020F94FF6FE73421E9A4205905D
:1027600040D8254C05AB4FF47A710422CDE9012104
:10277000009360220123A0212060204808F05AFD28
:10278000322006F005FD1E491E4803F029FD0CE02D
:102790006B78002BD1D1184B1B491A681B481EF0CF
:1027A000DBF81A49174803F01BFD07B030BD184D80
:1027B0001020296803F048FE0028BAD029684FF499
:1027C000805003F041FE0128B3D103F02FFDECE768
:1027D000012003F013FD07B030BD032003F00EFD10
:1027E00007B030BD022003F009FDDEE724F600202B
:1027F0005CF50020A970020874030020A0F50020F9
:10280000BC350208DEE100205039020820BB002060
:1028100020F600202DE9F043674C85B021680120A7
:1028200003F012FE00283FD1644D2B783F2B10D0CF
:1028300063496248FDF7CCFC0446002842D02B785F
:10284000432B00F08180012005B0BDE8F04303F088
:10285000D5BC6B78002BEBD121684FF4007003F0EE
:10286000F3FD38B921684FF4805003F0EDFD0028E6
:1028700000F09180534C544B0C2293ED000A402100
:102880000023204603F0DCF92046FDF7ABFC4F4B5C
:102890000219198821529B784D489370214605B042
:1028A000BDE8F04303F09CBC4A4B4FF480501968DC
:1028B00003F0CAFD012869D0062005B0BDE8F04349
:1028C00003F09CBC434E444D444FD6F80080D7F8EB
:1028D0000090012301462B703246414B3B604FF480
:1028E000805003F0B7FD324621464FF4006003F0FC
:1028F000B1FD32462146802003F0ACFD3246214630
:102900004FF4807003F0A6FDFFF7AEF82B78002B94
:10291000FCD1344B9FED347AD3ED007AC7F80090A8
:10292000F4EEC77AF1EE10FAC6F8008006DB9FEDF0
:102930002F7AF4EEC77AF1EE10FA2ED9182005B0EE
:10294000BDE8F04303F05ABC6B784C2B7FF47BAFAF
:10295000274B1A78522A7FF476AF5B78002B7FF4EE
:1029600072AF1948009004234FF47A720024CDE925
:10297000013204601F4801232822A02108F05AFCDC
:10298000322006F005FC1C49114888E705B0BDE877
:10299000F04303F04BBC172056E70B4C0094042384
:1029A0004FF47A72CDE901321248C4ED007A012366
:1029B0002822A021E2E700BF24F600205CF50020D9
:1029C0003836020820BB00206CBB002068370208A4
:1029D000DEE1002020F6002061BB002048BD002081
:1029E000A0860100F8BA00200050C3C70050C347BA
:1029F0005EF50020A0F50020BC350208D0B5734874
:102A0000734C84B01CF0C4FF2168012057EC106B9C
:102A100003F01AFD68B16F4B4FF48050196803F052
:102A200013FD012822D0062004B0BDE8D04003F0F9
:102A3000E5BB21684FF4007003F006FD002842D08A
:102A4000654C2378432B47D030463946FEF79EF835
:102A50002378502B07EE900A64D023784E2B0AD0AF
:102A6000012004B0BDE8D04003F0C8BB04B0BDE80D
:102A7000D04003F0DBBB6378452BF1D1574B1A787C
:102A8000472AEDD15B78002BEAD1504B1A783F2AC8
:102A900000F09580B7EE007AF4EEC77AF1EE10FA06
:102AA000DEDB9FED4F7AF4EEC77AF1EE10FAD7D85D
:102AB00004234FF47A724B4C4B480094CDE9013219
:102AC0000123502254E021684FF4805003F0BCFCF5
:102AD0000028B5D11720A7E763784C2BB4D1A37891
:102AE000522BB1D1E378002BAED1404B3D4C00933B
:102AF0004FF07E524FF47A770426CDE90167A0218A
:102B00001A60226001234A22374808F093FB3220E2
:102B100006F03EFBCDE901673348009401235022C3
:102B2000A02128E063784F2B97D12C4B1A78532A99
:102B300093D15B78002B90D1244B1A783F2A26D072
:102B4000B7EE007AF4EEC77AF1EE10FA88DB9FED6B
:102B5000247AF4EEC77AF1EE10FA81D804234FF408
:102B60007A72224C20480094CDE9013201234A2296
:102B7000A021C4ED007A08F05DFB322006F008FBCE
:102B80001B491C4804B0BDE8D04003F029BB5B786A
:102B9000002BD5D1154A184C92ED000A40210A228B
:102BA000204603F04DF82046FDF71CFB134B02199D
:102BB00019889B7821520F4893702146E2E75B7891
:102BC000002B7FF467AF074AE5E700BF3CF5002024
:102BD00024F6002020F600205CF500205EF50020A1
:102BE0000050C34764BB0020A0F5002068BB002054
:102BF000BC350208DEE1002020BB00206837020857
:102C00002DE9F04F2DED028B87B08148814C05A94D
:102C10001DF006FD2168012057EC106B03F014FC39
:102C200078B17D4C4FF48050216803F00DFC0128F1
:102C300025D0032003F0E2FA07B0BDEC028BBDE81B
:102C4000F08F21684FF4007003F0FEFB08B3059B82
:102C50006F4A93420BD01B784BB9704C2378502BA2
:102C600022D023784E2B02D16378452B4ED0012001
:102C700003F0C4FA07B0BDEC028BBDE8F08F22462A
:102C80000021102003F0E6FB07B0BDEC028BBDE88D
:102C9000F08F21684FF4805003F0D6FB0028D6D186
:102CA000172003F0ABFAC7E763784F2BD9D125463D
:102CB00015F8023F532BD4D1A04618F8033F002B40
:102CC000CFD130463946FDF761FFDFED557A08EE8A
:102CD000100AB4EEE78AF1EE10FA06DBDFED517A66
:102CE000B4EEE78AF1EE10FA1AD9022003F086FA60
:102CF0000027494EDFF85091BA46C9F80070C6F86F
:102D000000A007B0BDEC028BBDE8F08F464D2B78DC
:102D1000472BACD1A84618F8013F002BA7D1D0E72C
:102D20003D4EDFF828B1DFF82091D6F800A0D9F8A1
:102D3000007001238BF8003032463C4BC9F800305C
:102D400000214FF4805003F085FB324600214FF400
:102D5000006003F07FFB32460021802003F07AFB05
:102D6000324600214FF4807003F074FBFEF77CFEC6
:102D70009BF80030002BFBD12378502B06D0237812
:102D80004E2B29D0012003F039FAB6E763784F2B98
:102D9000F5D12B78532BF2D198F80030002BEED1DF
:102DA000234B244A009392ED007A2348C7EE087A19
:102DB0004FF47A714A22C3ED007A0423CDE9013140
:102DC0000123A02108F036FA322006F0E1F91B4970
:102DD0001B4803F005FA90E76378452BD2D12B7896
:102DE000472BCFD198F80030002BCBD1154B114A8F
:102DF000009392ED007A1048C7EE087A4FF47A7289
:102E0000C3ED007A0423CDE9013201235022D8E733
:102E10003CF5002024F6002020F600205CF5002080
:102E2000000096C4000096445EF50020A0860100D4
:102E300068BB0020F8BA0020A0F50020BC350208CD
:102E4000DEE1002064BB002048BD002060BB002004
:102E5000174B10B51968012003F0F6FAB0B9154BFD
:102E60001A783F2A04D0BDE81040012003F0C6B90B
:102E70005B78002BF7D11049104A11481DF06CFD0A
:102E8000BDE810400E490F4803F0AAB90E4C1020BF
:102E9000216803F0D9FA0028E1D021684FF480506E
:102EA00003F0D2FA0128DAD1BDE8104003F0BEB930
:102EB00024F600205CF500204C3602084436020857
:102EC00020BB0020DEE1002020F600202DE9F04F9D
:102ED000DFF8749185B0D9F80010012003F0B4FA3E
:102EE000002872D1534B1A783F2A05D0012005B033
:102EF000BDE8F04F03F082B95D78002DF6D1DFF820
:102F00004C81D8F80030002B52D0DFF844B14A4C45
:102F1000DFF840A12E460DE0D9F800104FF4007004
:102F200003F092FA98B906EB8603354658F8233039
:102F3000002B3DD005EB850308EB830301361A7A9D
:102F4000022A4FEA8507F6B253D0042AE4D03D4462
:102F500008EB850758F82530FA68009240215A4658
:102F600020461DF0C3FCD9F800104FF4007003F0A8
:102F70006BFA012848D02046FDF734F95146C0F1DC
:102F80003F0220461DF0BCFD2046FDF72BF92B4FDC
:102F9000054601232A462146384603F07FF80028DB
:102FA000F7D106EB8603354658F82330002BC1D104
:102FB000224C322006F0ECF82149204603F010F9AB
:102FC0000023237005B0BDE8F08F1E4C102021684F
:102FD00003F03AFA002885D021684FF4805003F0BE
:102FE00033FA01287FF47EAF05B0BDE8F04F03F05F
:102FF0001DB9D9F8001003934FF4007003F024FAC0
:10300000039B58B11A7AA0E72046FDF7EBF839691F
:10301000C0F13F0220461DF073FDACE7D9F8001067
:1030200003934FF4805003F00FFA039B0028E9D17B
:1030300079E700BF5CF5002020BB0020DEE1002026
:10304000BC35020820F6002024F60020580000209D
:10305000603602086837020838B56D4D01202968CE
:1030600003F0F2F9002833D16A4C23783F2B19D0B2
:103070002968012003F0E8F9002840F087802378D0
:10308000492B37D023784F2B00F08D802378532B9A
:1030900050D023784F2B00F09E80BDE838400120AF
:1030A00003F0ACB86378002BE2D15B4C8020216840
:1030B00003F0CAF9002857D0584A594B10681279C2
:1030C00018601A71BDE838405549564803F088B871
:1030D000514C1020216803F0B7F90028C4D02168B2
:1030E0004FF4805003F0B0F90128BDD1BDE838405D
:1030F00003F09CB863784E2BC4D14B4B1D78002D48
:10310000C0D1454A8020012103F0A4F9424A4FF47E
:103110008070294603F09EF93F4A4FF4005029463B
:1031200003F098F903F0A0F9BDE838403F493D4865
:1031300003F056B86378592BABD13B4B1A78542A1D
:10314000A7D15D78002DA4D1334A29464FF4807071
:1031500003F080F9304A8020294603F07BF92E4A9B
:1031600001214FF40050DBE721684FF4807003F039
:103170006BF980B12E4A2A4B1068928818609A80A9
:10318000BDE838402649274803F02AB8BDE8384052
:10319000062003F033B821684FF4005003F054F9CF
:1031A000B8B1244AE7E76378552B7FF46FAF1E4B25
:1031B0001A78542A7FF46AAF5D78002D7FF466AFE9
:1031C000154A4FF48070012103F044F9124A80201F
:1031D0009FE7194ACFE76378462B7FF45EAF124B27
:1031E0001A78462A7FF459AF5C78002C7FF455AFEB
:1031F000094A21464FF4807003F02CF9064A8020DA
:10320000214603F027F9044A4FF40050214687E78E
:1032100024F600205CF5002020F600206C36020821
:1032200020BB0020DEE100205EF50020BC35020856
:10323000743602087C360208D435020838B53E4C94
:103240000120216803F000F930B13C4D10202968BD
:1032500003F0FAF800284AD121684FF4007003F017
:10326000F3F870B1364B1A784F2A16D01A784F2AD5
:103270004FD01A783F2A24D0BDE83840012002F010
:10328000BDBF21684FF4805003F0DEF80028E9D17B
:10329000BDE83840172002F0B1BF5A784E2AE5D178
:1032A0009A78002AE2D1254A01214FF4006003F008
:1032B000D1F803F0D9F8BDE838402249224802F09D
:1032C0008FBF5B78002BD7D11C4C4FF40060216876
:1032D00003F0BAF8B0B921684FF4006003F0B4F815
:1032E00018B3BDE838401949174802F079BF29687A
:1032F0004FF4805003F0A8F80128ADD1BDE8384064
:1033000002F094BF124A114B1068127918601A71BA
:10331000E7E75A78462AACD10E4A11784629A8D157
:1033200051780029A5D1054ABFE70B4A074B106821
:10333000928818609A80D4E724F6002020F60020B6
:103340005CF50020BC350208DEE1002020BB002037
:10335000CC3502085EF50020D435020810B53D4B8F
:103360008CB01968012003F06FF800285ED13A4B49
:103370001A783F2A3CD005AB0024009337493648E1
:10338000059404AB03AACDE903441DF007FB40B24A
:10339000032828D1039B04993148172B94BFDCB232
:1033A0000394059B8DF818403B2986BF00210491AA
:1033B000C9B23B2B88BF00234FF0000298BFDBB29D
:1033C0008DF8191006A9CDE9092288BF05938DF85B
:1033D0001A308DF81B2009F04FFB2249224802F0D9
:1033E000FFFE0CB010BD012002F008FF0CB010BDB4
:1033F0005C78002CBFD1224606A9194809F03EFA94
:10340000224605A9164809F075FA9DF81A409DF85C
:1034100019309DF818201549009415481DF09CFAA4
:103420001349114802F0DCFE0CB010BD114C102005
:10343000216803F009F8002899D021684FF48050E2
:1034400003F002F8012892D10CB0BDE8104002F060
:10345000EDBE00BF24F600205CF50020F435020824
:1034600048F60020BC350208DEE100209036020854
:1034700020BB002020F6002010B53A4B86B019681A
:10348000012002F0E1FF002858D1374B1A783F2A7B
:103490003CD005AB0024009334493348059404AB79
:1034A00003AACDE903441DF079FA40B2032828D1DC
:1034B00003980499059B1F2886BF01200390C0B282
:1034C0000C2986BF01210491C9B2632B8CBF002354
:1034D000DBB24FF000028DF80A008DF809104FF0B2
:1034E000010402A9224888BF05938DF80B308DF89E
:1034F000084009F03FFB1F491F4802F071FE06B06B
:1035000010BD012002F07AFE06B010BD5A78002AE4
:10351000BFD102A9164809F0EDF99DF80B409DF8BE
:1035200009309DF80A201549009415481DF014FA39
:103530001349114802F054FE06B010BD114C102082
:10354000216802F081FF00289FD021684FF480504D
:1035500002F07AFF012898D106B0BDE8104002F0D1
:1035600065BE00BF24F600205CF50020B8360208D6
:1035700048F60020BC350208DEE10020A43602082F
:1035800020BB002020F6002038B53C4C01202168EB
:1035900002F05AFF002847D1394B1A783F2A24D02D
:1035A0002168012002F050FF002838D1344B1A78EE
:1035B0004F2A07D01A784F2A47D0BDE8384001205B
:1035C00002F01CBE5A784E2AF4D19A78002AF1D122
:1035D0002C4A0121202002F03DFF02F045FFBDE80A
:1035E00038402949294802F0FBBD5B78002BD7D130
:1035F000244D2020296802F027FF002831D0244ADA
:10360000244B1068127918601A7122491F4802F081
:10361000E7FD2168012002F017FF0028C6D0BDE8B1
:103620003840032002F0EABD164D1020296802F050
:103630000BFF0028B0D029684FF4805002F004FF3F
:103640000128A9D102F0F2FDAAE75B78462BB4D19C
:10365000114B1A78462AB0D159780029ADD1094AC0
:10366000B8E72968202002F0EFFE0028CDD10B4AF0
:10367000084B1068928818609A80C6E724F60020EC
:103680005CF5002020F60020BC350208DEE10020B9
:10369000CC35020820BB00205EF50020D43502089E
:1036A0003E4B10B51968012002F0CEFE30BB3C4BFA
:1036B0001A784F2A0AD01A784F2A31D01A783F2A1E
:1036C00044D0BDE81040012002F098BD5A784E2A3F
:1036D000F1D19A78002AEED13249334801230522EC
:1036E00002F0DCFC322005F053FD304A01211020AD
:1036F00002F0B0FEBDE8104002F0B6BE2B4C102028
:10370000216802F0A1FE0028D1D021684FF480503A
:1037100002F09AFE0128CAD1BDE8104002F086BD31
:103720005A78462ACAD1224A11784629C6D15178F8
:103730000029C3D110201D4A02F08CFE02F094FE35
:10374000BDE810401B49184802F04ABD5B78002BC9
:10375000B7D1164C1020216802F076FE50B92168CE
:10376000102002F071FE88B1BDE8104012490E48E9
:1037700002F036BD114A104B1068127918601A71A8
:10378000BDE810400C49084802F02ABD0C4A0A4B1B
:103790001068928818609A80E6E700BF24F600203F
:1037A0005CF5002024680208DEE1002020F60020FD
:1037B0005EF50020BC35020820BB0020CC35020895
:1037C000D435020870B5694D0120296802F03CFE2D
:1037D000002840F09C80664B1A783F2A04D0BDE850
:1037E0007040012002F00ABD5B78002BF7D12968F8
:1037F000012002F029FE0446003C29684FF0020037
:1038000018BF012402F020FE08B144F00204296828
:10381000042002F019FE08B144F0040429680820CD
:1038200002F012FE08B144F008042968102002F0EA
:103830000BFE08B144F010042968202002F004FEB9
:1038400008B144F020044B4E4FF40060316802F0A0
:10385000FBFD08B144F4804429684FF4007002F085
:10386000F3FD08B144F4004431684FF4805002F095
:10387000EBFD08B144F480343168022002F0E4FD2D
:1038800008B144F400343168042002F0DDFD08B1D1
:1038900044F4802429684FF4007002F0D5FD00281C
:1038A00049D13168102002F0CFFD08B144F48014F2
:1038B0003168202002F0C8FD08B144F400143168DA
:1038C0004FF4007002F0C0FD08B144F48004316888
:1038D000802002F0B9FD002840D044F40004316893
:1038E000802002F0B1FD78B329684FF4006002F047
:1038F000ABFD08B144F000741F49204822461DF07A
:103900002BF8BDE870401D491D4802F069BC194CF8
:103910001020216802F098FD00283FF45CAF216878
:103920004FF4805002F090FD01287FF454AFBDE8C1
:10393000704002F07BBC3168082002F085FD002851
:10394000AFD044F40024ACE731684FF4807002F04B
:103950007BFD0028C8D044F08074C5E731684FF47F
:10396000807002F071FD0028B7D1B8E724F600207E
:103970005CF5002020F60020C836020820BB00209D
:10398000DEE1002038B51D4C0120216802F05CFD0D
:1039900028B11B4D1020296802F056FD10BB21688C
:1039A0004FF4007002F050FDB8B1164B1A783F2A60
:1039B00004D0BDE83840012002F020BC5B78002B29
:1039C000F7D10F4B10491A6810481CF0C5FFBDE82D
:1039D00038400E490E4802F003BCBDE838401720BD
:1039E00002F00CBC29684FF4805002F02DFD012834
:1039F000D5D1BDE8384002F019BC00BF24F6002044
:103A000020F600205CF50020C836020820BB00200C
:103A1000DEE1002038B5284C0120216802F014FDB9
:103A200000BB264D2B783F2B0DD02168012002F0E2
:103A30000BFD00283AD12B78432B25D0BDE8384028
:103A4000012002F0DBBB6B78002BEED11C4B1D4933
:103A50001A681D481CF080FFBDE838401A491B4811
:103A600002F0BEBB1A4D1020296802F0EDFC0028C0
:103A7000D7D029684FF4805002F0E6FC0128D0D15D
:103A8000BDE8384002F0D2BB6B784C2BD6D1114B3D
:103A90001A78522AD2D15B78002BCFD1084A0E492E
:103AA00013600A48BDE8384002F09ABBBDE83840D0
:103AB000062002F0A3BB00BF24F600205CF5002026
:103AC00028F60020C836020820BB0020DEE10020D6
:103AD00020F600205EF50020BC35020870B53F4C92
:103AE0000120216802F0B0FC60BB3D4D3D492846F5
:103AF000FCF76EFBD0B13C492846FCF769FB002877
:103B000044D03A492846FCF763FB064600284CD0CF
:103B10002B783F2B23D0192002F070FBBDE87040BA
:103B20002E4A00214FF4007002F094BC224601217D
:103B30004FF4007002F08EFCBDE870402C492D4817
:103B400002F04EBB2C4C4FF48050216802F07CFCFC
:103B5000012820D0BDE87040062002F04FBB6B78F2
:103B6000002BD8D121684FF4007002F06DFC28B30F
:103B7000224A234B1068186021491E4802F030FB8E
:103B8000BDE870401A491B4802F02ABB22460121B9
:103B90004FF48050CEE72168102002F055FC002839
:103BA000D8D0BDE8704002F041BB014622464FF438
:103BB000007002F04FFC22463146E9E721684FF4DD
:103BC000805002F041FC20B10E4A0D4B1068186085
:103BD000D2E70D4A0A4B10681860CDE724F60020A2
:103BE0005CF500200CBC0020FCBB0020D436020891
:103BF000BC350208DEE1002020F60020DC36020899
:103C000020BB0020E0360208E436020870B5884C7C
:103C100086B0002321680120CDE9043302F014FCB2
:103C2000002871D1834B1A78552A4BD01A78532A21
:103C30007CD081497F48FCF7CBFA00283DD17F4BEF
:103C40004FF48070196802F0FFFB002840F0D2802A
:103C50007B4B1A783F2A00F0D58001232168002B86
:103C600000F0AA804FF4007002F0EEFB002800F094
:103C7000BD802168012002F0E7FB0446002840F0E7
:103C8000BD8070496E4805AB04AA1CF087FE02286F
:103C900013D1DDE904136C4A6C485370C3F3042359
:103CA00043EA41136A49137001220A6023462246FF
:103CB0002146006810F0A2F802E0012002F09EFA0E
:103CC00006B070BD5A78492AB0D19A78442AADD14D
:103CD000DA78002AAAD15A4B1A783F2AEDD15B78BC
:103CE000002BEAD15B4B5C4AD3E90001D2E90032F8
:103CF000CDE9001059495A481CF02EFE5849594840
:103D000002F06EFA06B070BD574D1020296802F01F
:103D10009BFB002886D029684FF4805002F094FB6A
:103D200001287FF47FAF02F081FAC9E75B784E2B60
:103D30007FF47FAF4D4B1B78002B7FF47AAF404B65
:103D40001A783F2A40D021684FF4007002F07CFBC3
:103D500000284BD02168012002F076FB00284DD1CD
:103D60003748FCF73FFA1428A7D8414C34491025AE
:103D7000421C4FF47A7620461CF0DDFF00940123AC
:103D80002022A221CDE901563A4807F053FA2C44EB
:103D9000322005F0FDF901233022A221CDE90156A0
:103DA0000094344807F046FA322005F0F1F9324920
:103DB0002C4802F015FA83E7012002F045FB30B3EE
:103DC000062002F01BFA7BE75B78002BBBD1284969
:103DD00023481CF0CDFE294A2149148892780346D5
:103DE00020481C809A7002F0FBF969E7172002F066
:103DF00005FA65E7082002F001FA61E7032002F006
:103E0000FDF95DE75B78002B3FF428AF25E70E4B0B
:103E10001B491A785878130203F4F85303435209E4
:103E20000F481CF099FD0E490E4802F0D9F947E7FA
:103E300024F600205CF500204C3B020828F6002008
:103E40003CF5002018370208C8BB002004F600200B
:103E500084BB0020CCBB0020D4BB0020EC36020881
:103E600020BB0020DEE1002020F600205EF50020CF
:103E7000DCBB0020A0F50020BC3502086837020832
:103E80000C37020870B5914D88B02968012002F006
:103E9000DBFA00284DD18E4C8E492046FCF798F96C
:103EA000B8B98D4C23783F2B34D16378002B31D1B6
:103EB0008A498B481CF05CFE8A4A894914889278AA
:103EC000034689481C809A7008B0BDE8704002F033
:103ED00087B986492046FCF77BF900283CD17E4B08
:103EE0001A783F2A40F08B805B78002B40F0878067
:103EF0007F4A8049D2E90040D2E90232CDE900048C
:103F000077481CF029FD7649774808B0BDE8704035
:103F100002F066B97048FCF765F90F2803D82378DA
:103F2000002B40F0AD800A2008B0BDE8704002F0E0
:103F300065B9714C1020216802F086FA0028AAD0D9
:103F400021684FF4805002F07FFA0128A3D108B015
:103F5000BDE8704002F06AB92378532B55D0674909
:103F60005B48FCF735F9002849D15B4B1A783F2AAA
:103F700000F0A28029684FF4007002F065FA002872
:103F800000F0938007AB002400935D4952480794EA
:103F900006AB05AACDE905441CF000FD40B203289C
:103FA00040F09080059A069B079C56494C481F2A72
:103FB00084BF012205920C2B84BF01230693632C3E
:103FC00088BF0024009488BF07941CF0C5FC4E4BAA
:103FD000434918461CF0A7FE4FF47A71034610229D
:103FE000CDE901210093A22148480123802207F056
:103FF00021F947493C4802F0F3F808B070BD0120B0
:1040000008B0BDE8704002F0F9B863784E2BA6D135
:10401000A378002BA3D1304B1A783F2A47D02968C8
:104020004FF4007002F010FA00283ED02A48FCF746
:10403000D9F81428E3D8374C2749421C10252046CC
:104040004FF47A761CF077FE01234022A2210094DF
:10405000CDE901562D4807F0EDF82C44322005F04B
:1040600097F8A22101235022CDE901562748009458
:1040700007F0E0F8322005F08BF825491A4823E7CD
:10408000164B1549421C18461CF055FE10220346DB
:104090004FF47A71CDE901210093A2211B4801233D
:1040A00007F0C8F81A4910480EE717203CE75B787C
:1040B000002BB4D11749FCE65B78002B7FF45AAF94
:1040C0001149F6E6012002F099F896E724F600205F
:1040D0005CF50020203702083CF5002088BB00205A
:1040E00020BB002068370208DEE1002028370208E4
:1040F00098BB00203037020820F60020483702081D
:10410000B83602085037020870BB0020A0F5002026
:10411000BC350208A8BB002030B5484C85B02168EA
:10412000012002F091F930B1454D1020296802F0CC
:104130008BF9002851D121684FF4007002F084F906
:1041400048B3404D2B783F2B0DD03F493D48FCF7FD
:104150003FF830B32B78432B4BD0012005B0BDE89E
:10416000304002F04BB86B78002BEED121688020F4
:1041700002F06AF9002854D0344A354B106891880F
:104180009279186099809A713149324805B0BDE83A
:10419000304002F025B8172005B0BDE8304002F0ED
:1041A0002DB82D4A2D4B92E803004FF47A7483E822
:1041B000030008222A480294CDE90032A2210123FB
:1041C000702207F037F8322004F0E2FF2549214839
:1041D00005B0BDE8304002F003B829684FF48050C4
:1041E00002F032F90128A6D105B0BDE8304002F056
:1041F0001DB86B784C2BB0D11B4B1A78522AACD11E
:1042000058780028A9D1154C009408234FF47A72ED
:10421000CDE90132A221C4E9000001231048702237
:10422000CFE72168802002F00FF90028ACD10F4BB6
:10423000074A03CB10605160A6E700BF24F60020B8
:1042400020F600205CF5002074370208643702086D
:1042500020BB0020DEE10020D4BB0020CCBB00202E
:10426000A0F50020BC3502085EF500206C3702087E
:1042700070B5524E524C316882B0012002F0E4F821
:1042800030B12168102002F0DFF8002840F0828071
:1042900021684FF4805002F0D7F8002874D0494DBF
:1042A0002B783F2B31D02A78474B995C490765D54D
:1042B00069785B5C5B0761D5302A0CBF0021012166
:1042C0003F4A042002F0C6F86B783D4A302B0CBF01
:1042D00000210121022002F0BDF831684FF4007086
:1042E00002F0B2F840B1AB78354A302B0CBF002158
:1042F0000121082002F0AEF83449354801F070FF82
:1043000002B0BDE8704002F0AFB86B78002BCAD1A4
:104310002168042002F098F821680546022002F086
:1043200093F82A4603462B492B481CF015FB3168AD
:104330004FF4007002F088F80246002837D0216858
:10434000082002F081F86C460246244920461CF001
:1043500003FB214620481CF0C4FB214B1E481B6870
:10436000ADF800301A0C21468DF802201CF0B9FB84
:104370001949174801F034FF02B070BD012002B0A6
:10438000BDE8704001F03ABF052002B0BDE87040C2
:1043900001F034BF21684FF4805002F055F8012835
:1043A0007FF476AF02B0BDE8704001F03FBF6C46CD
:1043B0000C4920461CF0D0FACBE700BF24F60020C1
:1043C00020F600205CF50020A9700208BC35020828
:1043D000DEE100207C37020820BB00208437020881
:1043E000683702088837020838B52F4D0120296840
:1043F00002F02AF808BB2D4C2D492046FBF7E8FEB9
:1044000068B32378452B0DD029684FF4007002F073
:104410001BF810B12378412B3AD0BDE83840012079
:1044200001F0ECBE6378582BEED1A378542BEBD17E
:10443000E378002BE8D11F4B12E01F4C10202168BD
:1044400002F002F80028D6D021684FF4805001F025
:10445000FBFF0128CFD1BDE8384001F0E7BE174B84
:10446000174C93ED000A012203234021204601F05E
:10447000E7FB2046FBF7B6FE124B021919882152C2
:104480009B78937021461048BDE8384001F0A8BEE3
:104490006378442BC1D10D4B1A78432ABDD15B7888
:1044A000002BBAD10A4BDBE724F600205CF5002094
:1044B0008C3702080800002020F600200C000020A5
:1044C00020BB002068370208DEE100205EF50020F6
:1044D0001000002038B53B4C0120216801F0B4FFEA
:1044E000002830D1384D2B783F2B13D02168012084
:1044F00001F0AAFF002860D134493348FBF768FE79
:10450000002832D02B784F2B3DD0BDE83840012019
:1045100001F074BE6B78002BE8D12D4C4FF4805025
:10452000216801F091FF002839D02A4A2A4B1068EF
:1045300091889279186099809A71BDE8384026492F
:10454000264801F04DBE224D1020296801F07CFF65
:104550000028C7D029684FF4805001F075FF01286A
:10456000C0D1BDE8384001F061BE194A01214FF4C5
:10457000805001F06FFF01F077FFBDE83840184927
:10458000164801F02DBE6B78532BBED1154B1A780F
:10459000432ABAD159780029B7D10D4AE7E72168F3
:1045A0004FF4805001F050FF0028C6D10E4A0A4B4C
:1045B0001068928818609A80BFE7BDE838400320F1
:1045C00001F01CBE24F600205CF50020AC37020888
:1045D00020F600209C37020820BB0020DEE10020EE
:1045E000BC3502085EF50020A437020810B51B4C4C
:1045F0000120216801F028FF216820B1012001F08D
:1046000023FFA0B910BD4FF4007001F01DFF20B9C9
:10461000BDE81040172001F0F1BD02F04DF801F0A7
:104620003DFFBDE810400E490E4801F0D9BD0E4CCB
:104630004FF48050216801F007FF012804D0BDE845
:104640001040062001F0DABD2168102001F0FCFEC8
:104650000028F4D0BDE8104001F0E8BD24F60020A9
:10466000BC350208DEE1002020F60020194B10B511
:104670001968012001F0E8FEA8B917491748FBF7AF
:10468000A7FD58B91649174801F0AAFD4FF47A70F2
:1046900004F07EFDBDE8104005F02EB8BDE81040E6
:1046A000012001F0ABBD104C4FF48050216801F0A7
:1046B000CBFE012804D0BDE81040062001F09EBDCD
:1046C0002168102001F0C0FE0028F4D0BDE81040A1
:1046D00001F0ACBD24F60020743702085CF5002020
:1046E000BC350208DEE1002020F6002070B5364D12
:1046F000364C84B028461BF04EF92168064601204E
:1047000001F0A2FE216828B1012001F09DFE30BB1E
:1047100004B070BD4FF4007001F096FE002832D056
:104720002B783F2B35D0012329480278002B34D039
:104730001AB301234FF47A72CDE901320090FF22BF
:10474000A0210670234806F075FD322004F020FDFC
:104750002149224804B0BDE8704001F041BD204C21
:104760004FF48050216801F06FFE012820D0062010
:1047700004B0BDE8704001F041BD012004B0BDE8C7
:10478000704001F03BBD172004B0BDE8704001F05F
:1047900035BD6B78002BC7D0C5E7124912481CF015
:1047A000DBF811490D4804B0BDE8704001F018BDB8
:1047B0002168102001F048FE0028D8D004B0BDE8E0
:1047C000704001F033BD00BF5CF5002024F60020EE
:1047D00080BB0020A0F50020BC350208DEE10020EF
:1047E00020F600207439020820BB00202DE9F0419A
:1047F000B14C82B0002321680193012001F024FE16
:1048000000287BD1AD4D2B783F2B73D0012321683D
:104810008BB9202001F018FE002800F08280A84B00
:10482000A84A03CB10605160A649A74801F0D8FC04
:1048300002B0BDE8F081012001F006FE002840F042
:104840008A80A2499D48FBF7C3FC002800F08980BC
:104850009F499A48FBF7BCFC0646002870D02B788D
:10486000522B00F0AA802B784C2B00F00D812B7876
:10487000522B00F0538197499048FBF7A9FC002880
:1048800000F0EE8094498D48FBF7A2FC002840F030
:104890005D8192499248934F01220EF01DF83870C5
:1048A000002840F07081904DDFF83482864E01ABD5
:1048B0004FF48072294640460EF0BAF93870019ADA
:1048C00001232946304601F0E9FB0446052010F09B
:1048D00023FB002CF3D1019BB3F5807FE7D07A4C0A
:1048E0007F480EF097FC8149204601F079FC0023B7
:1048F00023709DE76B78002B89D087E77C4D4FF4C0
:104900008050296801F0A0FD01287FF47BAF296861
:10491000102001F099FD00283FF474AF01F086FCEF
:1049200086E72168202001F08FFD00287FF47CAF0E
:10493000704B644A03CB1B8810605160138173E78E
:104940002168202001F080FD0128044674D01C203D
:1049500001F054FC6CE7062001F050FC02B0BDE809
:10496000F0812168202001F06FFD044608BB624BF6
:10497000024693E8030002F07DF9C82004F008FC29
:1049800003F0E8FA5D495E4801220DF04BFF554BFC
:104990001870002846D0012108465A4A01F05AFDF5
:1049A000454A2020214601F055FD122001F026FC49
:1049B0003EE71B2001F022FC3AE76B78532B7FF493
:1049C00052AF514B1A78542A7FF44DAF5C78002CCB
:1049D0007FF449AF2146384A474D202001F03AFD87
:1049E0002246464920460DF01DFF484808F02EFAA1
:1049F000464803F075FB464B95E8030001221C7006
:104A000002F038F9C82004F0C3FB95E80300224601
:104A100002F030F9C82004F0BBFB34492A4801F009
:104A2000DFFB05E7244A0121202001F013FD2F4977
:104A3000254801F0D5FBFBE63049324630460DF003
:104A4000F1FE284B01461870002800F083802046B4
:104A50002C4A214601F0FEFC132001F0CFFBE7E6D3
:104A60001F4C1E49012220460DF036FF1D4B1870C9
:104A700000287FD12046E4680EF0CCFB2549114880
:104A800022461BF069FFCFE66B78532B7FF4EFAE25
:104A90001D4B1B78002B7FF4EAAE1F4801F08EFC03
:104AA000104B187000284CD0112001F0A7FB1A4BB6
:104AB00000221A70BCE600BF24F600205CF500203E
:104AC000B837020820BB0020DEE10020CC37020806
:104AD000D4370208E8370208F03702083CF5002016
:104AE00074DD002070DD00203CBC0020BC350208D5
:104AF00020F60020C0370208446802087036020819
:104B0000A4DF002028F600205EF5002040F70020FA
:104B1000D4460120503902083CBD00206B784D2B53
:104B20007FF4A9AE1C4B1B78002B7FF4A4AE1B486E
:104B30000EF0A2FC1A4B1870B8B1142001F05EFB05
:104B400076E61849184801F04BFBB0E7012001F068
:104B500055FB6DE6154B164A1970202001F07AFCC2
:104B60001049114801F03CFB62E60E490E4801F085
:104B700037FB5DE60F4A0121022001F06BFC152096
:104B800001F03CFB54E60B4A0121022001F062FCDB
:104B9000162001F033FBA2E65EF500203CF5002074
:104BA00070DD0020BC350208DEE10020D446012083
:104BB00024F6002028F6002030B53B4C85B0216853
:104BC000012001F041FC002852D1384D2B783F2BB9
:104BD0003BD02168012001F037FC00285BD12B7805
:104BE000334AD35C5B072AD530481AF0D4FE314BE8
:104BF000A0F10A029A4254D803F1CC532E4A2F490D
:104C000003F5252303F2627302FB0033B1EB730F4C
:104C100015D92B4C0094A2FB002004234FF47A7288
:104C2000C008CDE90132A02101231C2220602548C3
:104C300006F000FB322004F0ABFA234912E0012019
:104C400005B0BDE8304001F0D9BA6B78002BC0D177
:104C50001B4B1E491A681E4802EB820252001BF0D1
:104C60007BFE1B491B4805B0BDE8304001F0B8BAD7
:104C7000194D1020296801F0E7FB0028A5D029680C
:104C80004FF4805001F0E0FB01289ED105B0BDE853
:104C9000304001F0CBBA032005B0BDE8304001F050
:104CA000ADBA0220CCE700BF24F600205CF500205E
:104CB000A970020836420F00CDCCCCCC9999991935
:104CC00048BD0020A0F50020BC350208503902087C
:104CD00020BB0020DEE1002020F6002000000000C4
:104CE000F0B52DED028B5048504C85B01AF050FEB7
:104CF0002168012057EC106B01F0A6FB002848D179
:104D0000494B1A783F2A26D02168012001F09CFBEC
:104D1000002867D139463046FBF738FF08EE100A05
:104D2000FBF722FC3EA3D3E9002306460F46FBF720
:104D3000F9FEF2EE047AB4EEE78A00283ED0F1EEF6
:104D400010FA57D946DC012005B0BDEC028BBDE856
:104D5000F04001F053BA5B78002BD5D1344C354A82
:104D6000402192ED000A2046012200F069FF204612
:104D7000FBF738FA304B0219198821529B782F48DB
:104D80009370214605B0BDEC028BBDE8F04001F008
:104D900027BA2B4D1020296801F056FB0028AFD010
:104DA00029684FF4805001F04FFB0128A8D105B0CD
:104DB000BDEC028BBDE8F04001F038BAF1EE10FA1C
:104DC00008DC17A3D3E9002330463946FBF796FEEB
:104DD0000028B8D0022005B0BDEC028BBDE8F04041
:104DE00001F00CBA032005B0BDEC028BBDE8F04029
:104DF00001F004BA0F4C009404234FF47A72CDE909
:104E00000132A021012308220E4884ED008A06F019
:104E100011FA322004F0BCF90B490848B2E700BF90
:104E20009A9999999999B93F5CF5002024F6002048
:104E300020BB002040BD002068370208DEE10020D2
:104E400020F60020A0F50020BC35020870B5AD4C5E
:104E500084B02168012001F0F7FA002840F09F801B
:104E6000A94D2B783F2B00F08180A849A648FBF77D
:104E7000AFF9002840D1A64D2B783F2B00F0C18020
:104E80002168012001F0E0FA002840F09D802B7895
:104E9000A04AD25C510702D42D2B40F0A0809C4840
:104EA0001AF076FD51EC100BFBF770FE9FED9A7A2D
:104EB00007EE900AF4EEC77AF1EE10FA00F1918055
:104EC0009FED967AF4EEC77AF1EE10FA00F389803E
:104ED00004234FF47A72924C92480094CDE9013247
:104EE00001230C22A021C4ED007A06F0A3F93220A0
:104EF00004F04EF98C494CE08C498348FBF768F983
:104F0000002840F09780824D2B783F2B62D021689B
:104F1000012001F099FA002856D12B787D4AD25C05
:104F2000520701D42D2B5AD179481AF031FD51EC9A
:104F3000100BFBF72BFE9FED787A07EE900AF4EE4C
:104F4000C77AF1EE10FA4CD49FED747AF4EEC77A7A
:104F5000F1EE10FA45DC04234FF47A72744C714878
:104F60000094CDE9013201231022BBE76B78002BBE
:104F70007FF47BAF6F4C4FF40070216801F064FA4E
:104F8000002830D06C4A6D4B1068127918601A7185
:104F90006A496B4804B0BDE8704001F021B9654D25
:104FA0001020296801F050FA00283FF459AF296811
:104FB0004FF4805001F048FA01287FF451AF04B05B
:104FC000BDE8704001F032B9032004B0BDE8704084
:104FD00001F014B96B78002B99D1554A16E00120E5
:104FE000F3E70220F1E721684FF4007001F02CFA9A
:104FF0000028CDD1534A514B1068928818609A808E
:10500000C6E76B78002B7FF43BAF454A4B4C92EDE3
:10501000000A40210622204600F012FE2046FBF73F
:10502000E1F8494B021919889B7821524448937042
:105030002146AFE72168012001F006FA0028C3D11C
:105040002B784F2B24D02B784F2B3CD02B78432B15
:10505000C5D16B784C2BC2D13C4B1A78522ABED1A9
:105060005D78002DBBD13A4B2A4693E8030001F04E
:1050700001FE04202946234A01F0ECF921680420AE
:1050800001F0E2F9002830D0324B00221A7031E7EB
:105090006B784E2BD7D12D4B1E78002ED3D12C4BB5
:1050A000324693E8030001F0E5FD3146154A04203D
:1050B00001F0D0F91F4A01214FF4007001F0CAF944
:1050C00001F0D2F916E76B78462BBFD11F4B1A7847
:1050D000462ABBD159780029B8D1164A4FF400703E
:1050E00001F0B8F901F0C0F904E7124B4FF4007079
:1050F000196801F0A9F90028C6D0164B01221A70D0
:10510000F8E600BF24F600205CF50020F83702081E
:105110003CF50020A9700208000096C400009644E7
:10512000F4BA0020A0F50020BC35020800380208BF
:105130000000002020F60020CC35020820BB002013
:10514000DEE10020D4350208683702085EF5002051
:105150003C68020815BB002070B53448344C84B05C
:105160001AF019FC21680546012001F06DF90028AC
:105170003DD12E4B1A783F2A29D02168012001F019
:1051800063F900284CD16B1E632B43D8012D294CA9
:10519000274A256014BF014629464FF4806001F07C
:1051A00059F94FF47A720423CDE90132A021012389
:1051B00046220094204806F03DF8322003F0E8FF34
:1051C0001E491F4804B0BDE8704001F009B85B7883
:1051D000002BD2D1174B1B491A681B481BF0BCFB94
:1051E0001949174804B0BDE8704000F0F9BF174EE8
:1051F0001020316801F028F90028BAD031684FF446
:10520000805001F021F90128B3D104B0BDE870400D
:1052100001F00CB8022004B0BDE8704000F0EEBF11
:10522000032004B0BDE8704000F0E8BF5CF500204A
:1052300024F6002044BD0020A0F50020BC35020863
:10524000DEE100205039020820BB002020F60020BB
:1052500080B54FF4FA600FF05FFE544B93E8030003
:1052600001F01CFD002847D1514904465148FAF786
:10527000AFFF514A002800F093802146802001F0C2
:10528000E9F84E4A01214FF4003001F0E3F84C4AAE
:1052900001214FF4805001F0DDF8494A002110202F
:1052A00001F0D8F8464A0021202001F0D3F8444A02
:1052B0000021802001F0CEF8414A00214FF4807097
:1052C00001F0C8F83E4A00214FF4007001F0C2F826
:1052D0003C483D4B384A4FF07E54012104604FF466
:1052E0008060196001F0B6F8384A394B118892781D
:1052F00019809A70FCF7A4FC2F4DDFF8DC80354E46
:105300002E4FDFF8ACA0DFF8AC9014E00021402075
:1053100001F0A0F8294A01214FF4807001F09AF8B9
:1053200039682A4669B30121022001F093F84FF44D
:10533000FA700FF0F1FD2968012001F085F80446AC
:1053400080B9D8F800306BB10822514648461BF0AE
:1053500096FB2A46C8B90121802001F07BF8002382
:10536000C8F8003096E8030001F098FC2A460028AF
:10537000CCD10121402001F06DF839682A4600297E
:10538000D1D1022001F066F8D1E72146802001F05A
:1053900061F80A4A01214FF4003001F05BF8DEE7C2
:1053A0000121802001F056F871E700BF346802083F
:1053B000CCBB0020D4BB002024F6002028F600201F
:1053C00020F6002040BD002044BD0020C435020866
:1053D0005CF500202C68020834F600200000000074
:1053E0002DE9F0472DED028B8CB0002207A93E4835
:1053F000DFF80C81DFF80CA13C4C9FED3D8ADFED1E
:105400003D8A394D07F03AFA3748002201A907F0E2
:1054100071FA33A7D7E900674FF00009204603F07F
:1054200075FF4FF0FF31204603F0F4FF204604F0F3
:1054300049F807EE900AF8EE677A17EE900AFBF744
:1054400093F832463B46FBF7E7F800222A4BFAF77F
:105450002BFFFBF79BFB03464FF47A70C8F8003034
:105460000FF05AFD002202A9284607F007FA002291
:1054700001A9284607F03EFA9DF81CC09DF80830A7
:105480009DF81DE01D4AA3EB0C039DF809C0C3EB7A
:105490000313ACEB0E0C0CEB830300214FF4006004
:1054A000CAF80030B9F1000F01D11E2BB6DDD8EDDE
:1054B000007AF4EEC87AF1EE10FA04D4F4EEE87A49
:1054C000F1EE10FA04DD00F0C5FF4FF00109A5E789
:1054D0000A4A01214FF4006000F0BCFFF5E700BF6D
:1054E00008AC1C5A643BAF3F48F6002090060020F1
:1054F00000005C42000082420000494024F6002087
:105500001000002050BD00200B4C08B52068002181
:105510000EF0FCFE4FF0E0264FF080554FF0FF31CB
:1055200020680EF0F3FE00F0A1FEC6F8045DBFF3A4
:105530004F8FBFF36F8FF1E71CF6002080B5144D3D
:10554000144F2868144C154E84B000210EF0DEFE76
:1055500028684FF0FF310EF0D9FE97ED000A0023C6
:1055600007221021684600F06BFB6846FAF73AFE06
:1055700003460DEB000EB4F800C0A2782DF803C06E
:10558000694630468EF8022000F02AFEE0E700BFB0
:1055900010F60020F8BA002068370208DEE100208B
:1055A0002DE9F04FB04EB148B14DB24CDFF8108349
:1055B000DFF810A3DFF810B3A3B0402220211BF0C6
:1055C00088FA306800210EF0A1FE4FF0FF313068FC
:1055D0000EF09CFE216895F800904FF4805000F08A
:1055E00033FF216890BB102000F02EFF0028ECD084
:1055F000A14BDAF800201878A04F09F1FF390328F1
:105600004FF4B46309F01F0903FB098108BF9A48EE
:105610004FF001034FEAC20218BF58463B6000F04A
:105620003DFD974B18700028CFD0924A00211020E2
:1056300000F010FF934A01214FF4803000F00AFF80
:105640008D4A00238BF800301370BEE74FF4805072
:1056500000F0FAFE0128B8D12B78013B4FF4B46971
:1056600003F01F0309FB038393ED010A07220023C4
:10567000202109A800F0E4FA09AB00932B788249B5
:10568000013B03F01F0309FB03F311A858F80320A3
:10569000130E22F07F421BF05FF92168042000F016
:1056A000D3FE0128814600F0B2802168022000F07C
:1056B000CBFE0128814600F09580744B4FF40070BA
:1056C000196800F0C1FE002870D111A8FAF78AFD10
:1056D0006F4911AB8146034411A80A8820F80920BC
:1056E0008A789A70216809F1020310201F4600F0A1
:1056F000ABFE002841D12168202000F0A5FE002843
:105700003FF463AF11A942F2200307F0030221F82E
:105710000930C2F10402554911A81BF0F1F911A892
:10572000FAF760FD5B4B821E814611A840F60D2101
:105730001B688152584A1068002B7DD0012B00F065
:105740008A80B0F57C6F7FF640AF524A83F0010348
:105750001360514A00231360504A194610681A46D4
:105760000EF04CFB4FF0E0234FF08052C3F8042DB5
:10577000BFF34F8FBFF36F8F27E701233A4611A97D
:10578000584600F08BFC3E4B18700028B3D0394AC5
:105790000021102000F05EFE3A4A01214FF48030D3
:1057A00000F058FE00238BF80030A4E721680820A1
:1057B00000F04AFE0128814687D111A8FAF712FDB0
:1057C000374B93ED000A374B11A91B880B524A4601
:1057D00005A80023102100F033FA05A911A81BF039
:1057E00080F972E711A8FAF7FDFC2F4B93ED000A40
:1057F0002C4B11A91B880B524A4605A800231021E7
:1058000000F01EFA05A911A81BF06BF955E711A8C5
:10581000FAF7E8FC254B93ED000A224B11A91B88EF
:105820000B524A4605A80023102100F009FA05A9E9
:1058300011A81BF056F938E703931D4B4A4618444C
:1058400011A91BF078FA1B4B186848441860124BDA
:105850001860039B75E70393174B4A46184411A938
:105860001BF069FA154BEFE714F600201400002036
:10587000E4BA002020F60020DDE100204CBD00202D
:10588000DCE1002028F600200838020824F6002079
:10589000683702086CBD002068BD00200CF60020AF
:1058A0001000002014380208080000200C0000201E
:1058B00070CD002064BD002070BD002060BD0020C0
:1058C000D8060020DCBA0020DEE100202DE9804867
:1058D000DFF8F880374FD8F80000374CDFF8F09049
:1058E000364EDFF8F0B0364DDFF8ECA083B0002183
:1058F0000EF00CFD16E052460021202000F0AAFD1B
:10590000304A0121042000F0A5FD28460DF082FC5C
:10591000307078BB2C4A0021102000F09BFD2368DA
:1059200000221A604FF0FF31D8F800000EF0EEFCB4
:1059300000F07AFA2368D9F800101A6828463B4626
:105940000DF0A8FA014630700028D4D123683A68D7
:105950001868904214D05246202000F07BFD194A6E
:105960000121202000F076FD28460DF053FC307018
:105970000028CFD0134A0121102000F06BFDC9E7A9
:10598000DBF80020092A03D80132CBF80020C7E752
:105990002846CBF8001001910DF0C0FB0199307042
:1059A0000028BCD05246202000F054FD054A0121B9
:1059B0000820A8E754BD002058BD002070DD00205D
:1059C00074DD002028F6002024F600200CF60020CC
:1059D0005CBD0020E0E1002020F6002010B582B080
:1059E00000240F4B0194196B41F4800119631B6B68
:1059F00003F480032246062101933B20019B03F020
:105A00001FFE3B2003F058FE22460621452003F0EE
:105A100017FE452002B0BDE8104003F04DBE00BFA8
:105A2000003802400F4A104BD2F8FC1021F0807170
:105A3000C2F8FC10D2F8FC1041F08071C2F8FC10E2
:105A40001A6822F001021A601A68002042F001026E
:105A50001A60586000BF00BF00BF5868B0FA80F0FD
:105A60004009704700ED00E0001000E030B5002470
:105A700083B001250AF042F819F07CFCCDE900540E
:105A800023463B493B484FF480720EF085FFCDE939
:105A900000542346384939484FF480720EF07CFF99
:105AA0000223CDE900343649364823464FF40072CC
:105AB0000EF072FF344B35493548CDE900534FF4B1
:105AC000C07223460EF068FFCDE9005423463149E9
:105AD00031484FF420720EF05FFF0323CDE900340C
:105AE000042523462D492E484FF4A0620EF054FFA2
:105AF000CDE9005423462B492B484FF4A0620EF009
:105B00004BFFCDE9005423460625284928484FF489
:105B100000720EF041FF2346CDE900542549264886
:105B20004FF4F0620EF038FF0723CDE9003423492B
:105B3000234823464FF400620EF02EFF0823CDE9E0
:105B400000342049204823464FF400620EF024FF21
:105B5000CDE900541D491E4823464FF400720EF053
:105B60001BFF204603B0BDE830400EF045BF00BF2C
:105B7000183802083173000820380208E153000881
:105B8000303802085152000800F600204038020860
:105B9000097A00084C380208DD6E00085438020803
:105BA0000955000860380208CD5800086C38020812
:105BB0003D5500087C380208A15500088C380208C1
:105BC000318B000898380208C5840008A438020800
:105BD0008D890008704700BF014B586A704700BFAD
:105BE000000C0040704700BF704700BFFEE700BFD9
:105BF000FEE700BF044B10B40360044C0C6080232C
:105C00005DF8044B13607047E4E30020E4E10020FA
:105C100010B5094C0FCC88B00DF1040CACE80F00A6
:105C200094E807008CE80700002101A80DF06AFD48
:105C3000024B186008B010BD083502088CE4002043
:105C4000072AB5EEC00AF0B5174628BF0727F1EEC0
:105C500010FA4CBFF1EE407AF0EE407ABDEEE77AF2
:105C60008BB0F8EEC76A064677EEE67A0D461C461C
:105C7000002A6BD04FF0000C01220CF1010C5FFAEE
:105C80008CFE02EB820277454FEA4202F5D806EE1F
:105C9000902AF8EE666A67EEA67AF6EE006A77EE6C
:105CA000A67AFCEEE77A17EE903A934205D317EE08
:105CB000103A013307EE103A0023B5EEC00AF1EEB8
:105CC00010FA009702AF4CBF224A234A01932021C9
:105CD00017EE103A38461AF009FE84422CD9012DED
:105CE0009DF8083024D9721E1444A919241A0239C7
:105CF0004FF0200C01E08A4204D0104602F801CF98
:105D0000A242F8D1C6F102020244B11803B3501CFA
:105D100085421DD9013A324402E0A94207D2084621
:105D200002F8013F17F8013F411C002BF5D1064452
:105D3000002333700BB0F0BD013D2A463946304692
:105D40001AF003FF002373550BB0F0BD0122A4E746
:105D50000E46EDE7C0380208CC380208274B284A27
:105D60001B68D2ED007A1B05F8EE677A21D525492C
:105D7000254A264B92ED006AD3ED006A91ED007A38
:105D80002349244B244AB8EE477A27EE866A67EE09
:105D9000A66A26EE076A66EE876A91ED007AC3ED81
:105DA000006A27EE877A1D4B82ED006A83ED007A48
:105DB00070471B4B1B78ABB1124B1549D3ED006AF2
:105DC00091ED007A134B144AF8EE666A27EE877A53
:105DD00066EEA76AC3ED006A104BC2ED006A83ED60
:105DE000007A70470B4B0C4AC3ED007A9FED0D7A99
:105DF0000A4BC2ED007A83ED007A704720F600204E
:105E00000400002044BD002068BB002064BB0020CB
:105E10006CBB0020E8BA0020ECBA0020F0BA0020E9
:105E200060BB002000000000094B1B6833B9094922
:105E3000094B0A480A4A08601A607047012B00D0D3
:105E400070470449044B0748074A08601A607047C6
:105E50006CBD00205CBD002058BD002070BD00203E
:105E600060BD002070CD002064BD002070B5154ECF
:105E70008EB00D46044609A90022304606F0FEFC0D
:105E800008A90022304606F035FD0F4A9DF826107D
:105E900006929DF825200D4BCDE904219DF8241094
:105EA0009DF82220CDE902219DF821109DF82320A4
:105EB0002046CDE90021064A29461AF017FD0EB00A
:105EC00070BD00BF48F60020F838020888BB0020EB
:105ED000D83802082DE9F041474E484C484F494D0B
:105EE00082B031460022204606F0C8FC2046464CCF
:105EF0003946002206F0FEFC4FF00008434A4449B0
:105F000085F8008020461AF027FD214628461AF021
:105F1000E8FDBB7800937B78FA783E4920461AF07A
:105F20001BFD214628461AF0DCFDB37800937378F8
:105F30003278394920461AF00FFD2846FAF752F90F
:105F4000214628441AF014FE3449024608681060BD
:105F5000334890ED000A8888897990804346917192
:105F6000204601224FF48051FFF76AFE2046FAF7DF
:105F700039F92C4A03461E191068E0509388B38003
:105F8000214628461AF0ADFD274B28491A682046BD
:105F90001AF0E2FC214628461AF0A3FD244B2549BD
:105FA0001A682046C2F38003C2F340021AF0D4FC00
:105FB000214628461AF095FD1F4B186820609B88E3
:105FC000A3802846FAF70EF9214628441AF0D0FD9E
:105FD000421B02F003021949C2F1080228461AF0D6
:105FE0008FFD2846FAF7FEF8023840F60D232B52B3
:105FF00002B0BDE8F08100BF6CF6002048F600203A
:1060000068F6002070BD002070CD002088BB002005
:10601000FC38020808390208203902083839020819
:1060200040BD00204039020844BD00204839020824
:1060300020F60020583902086839020814000020B0
:10604000074B4FF4FA601B68B0FBF3F0B42804D898
:10605000B3F5FA6F88BF01207047B420704700BFC6
:10606000040000209FED0B7AC7EE007A10B50A4CB1
:10607000236800225A622046FCEEE77A17EE903A37
:10608000013BE36007F0B8FF2046BDE8104007F091
:10609000A3BD00BFA037A04CB8F800202DE9F04305
:1060A000464F1D463B6883B004461646002B69D018
:1060B000DFF82481C8F8001021780139032921D89C
:1060C000DFE801F058361302D8F800103C48B2B2AD
:1060D00008F004F905B925703B68002B59D0C0B20F
:1060E00000233B6003B0BDE8F083364BD8F80020B6
:1060F0001868009200231A46694601960DF07EFE4C
:1061000001284CD105B925703B68002B38D1D8F84F
:1061100000302D492D4833445A1AB2F5606F88BFBC
:106120000B4602600020C8F8003003B0BDE8F083E1
:10613000DFF8A890D8F8002000920023D9F80000DA
:1061400001961A4669460DF059FE0128DAD06420FE
:1061500003F01EF8D9F8000000210DF04BFD1C4B98
:1061600093F82D305A0722D505B925703B6813BB2B
:106170000120B7E7D8F80000B1B219F017FAA9E783
:106180000020ADE7DFF85080D8F800001AF0D3FD0A
:1061900092E70028BBD0C0B203B0BDE8F083642012
:1061A00002F0F6FF0A4B93F82D305B07DCD4094B65
:1061B00001221A60D8E7012092E700BF4CBD002001
:1061C00060F90020FCF50020DCE4002090E40020D1
:1061D00064FA002098E400205400002008F6002013
:1061E00070B5054608460C46F9F7FCFF2146024605
:1061F00000232846BDE87040FFF750BF10B5084C9B
:106200000849024620461AF0A7FB2046F9F7EAFFA4
:1062100021460246BDE8104003480023FFF73EBF79
:1062200020BB002070390208DEE100200B480C4939
:10623000036810B50B4C23F01003036004222046C2
:106240001AF08AFB2046F9F7CDFF21460246BDE849
:10625000104005480023FFF721BF00BF20F60020B3
:106260007039020820BB0020DEE10020F0B583B0C9
:10627000414D424B424A4349434800951AF08EFB38
:1062800002283DD0032828D001280BD13F4A40499D
:106290003B481AF083FB3F493F4A002301280B701B
:1062A00013703FD03D4B1B68DB0705D53C4C226883
:1062B00041F21003934357D03A493B4800221AF069
:1062C0004BFB3948F9F78EFF374902463748002320
:1062D00003B0BDE8F040FFF7E1BE2C4A2C49284846
:1062E0001AF05CFB2B4A2A49044624481AF056FB54
:1062F0000128294A2E49284631D01AF04FFBD1E710
:10630000224A23491E481AF049FB224A20490446E2
:106310001A481AF043FB204B002201281A70C1D101
:10632000012CBFD1234F39680029BBD0174E3D4601
:10633000002404E055F8141F01340029B2D030467F
:10634000F9F746FF0028F5D104EB840407EB840736
:10635000194A7B68136003B0BDE8F04018471AF093
:106360001DFB01289ED1DBE722F010030D490E48EA
:1063700023600422A3E700BFDCF40020FCF400202B
:106380001CF500207C3902089CE400207CF50020EC
:10639000903902085CF500203CF5002024F600202E
:1063A00020F600207039020820BB0020DEE100202A
:1063B0008839020858000020F4F50020F0B5A5B097
:1063C000014601A80CF05AFF002832D11B4F1C4D8A
:1063D0001C4E0EA901A80CF0F9FF044618BB9DF84D
:1063E0004E4004B32E2CF4D09DF84030DB06F0D4A0
:1063F0000DF14E02394628461AF0AEFA2846F9F752
:10640000F1FE0123024629463046FFF747FE0028E9
:10641000F4D1142002F0BCFE0EA901A80CF0D6FFA6
:1064200004460028DBD001A80CF0A2FF204625B0CE
:10643000F0BD0446204625B0F0BD00BF5836020826
:1064400020BB0020DEE10020014214BF012000201B
:10645000704700BF136819B923EA00001060704745
:1064600018431060704700BF00B585B0094B00931A
:106470004FF47A710422CDE9012101230022A021E9
:10648000054804F0D7FE322005B05DF804EB02F0B9
:106490007FBE00BF20F60020A0F500202DE9F041CE
:1064A0006F4C704B84B04FF47A7504260093CDE99D
:1064B000016501230022A021204604F057FF6A4A0B
:1064C0000092CDE9016501230822A021204604F0B5
:1064D0004DFF664A0092CDE9016501231022A021FB
:1064E000204604F043FF624A0092CDE90165012392
:1064F0000C22A021204604F039FF5E4A0092CDE92B
:10650000016501231C22A021204604F02FFF5A4AD6
:106510000092CDE9016501232822A021204604F044
:1065200025FF564A0092CDE9016501234622A021AC
:10653000204604F01BFF524A0092CDE90165012379
:106540004A22A021204604F011FF4E4A0092CDE9D4
:10655000016501235022A021204604F007FF4A4A8A
:106560000092CDE9016501236022A021204604F0BC
:10657000FDFE1027454B00933A46CDE901750123F6
:10658000A221204604F0F2FE4FF02008404B009379
:106590004246CDE901850123A221204604F0E6FE12
:1065A0003C4B009308230193029501237022A22102
:1065B000204604F0DBFE384B0093CDE90185012332
:1065C0004022A221204604F0D1FE344B0093CDE9B5
:1065D000017501238022A221204604F0C7FE304B22
:1065E0000093CDE9017501238022B021204604F0FB
:1065F000BDFE2C4A0092CDE9016501233022A02185
:10660000204604F0B3FE284A0092CDE9016501233B
:106610003422A021204604F0A9FE244A0092CDE9AC
:10662000016501233822A021204604F09FFE204B63
:1066300000930622CDE9012501234022A021204616
:1066400004F094FE01231B4A0092CDE90135FF229C
:10665000A021204604F08AFE04B0BDE8F08100BF0E
:10666000A0F5002020F6002040BD00200000002002
:10667000F4BA002048BD00206CBB002044BD0020BF
:1066800068BB002064BB00207403002088BB00208E
:10669000DCBB0020CCBB0020A8BB002070BB0020CE
:1066A00098BB002054FA002050FA00204CFA002039
:1066B000C8FA002080BB00202DE9F043AF4BB04C5E
:1066C000DFF82C8385B04FF47A7504270022CDE9DA
:1066D00001750093A0211A602046012304F0AAFD51
:1066E000322002F055FDA74BA74A0093CDE9017572
:1066F000A0211A6020460123082204F09BFD3220CD
:1067000002F046FDA14BA24A0093CDE90175A021FC
:106710001A6020460123102204F08CFD322002F082
:1067200037FD9C4B9C4A0093CDE90175A0211A606E
:10673000204601230C2204F07DFD322002F028FDCA
:10674000964B00936422CDE90175A0211A60204682
:1067500001231C2204F06EFD322002F019FD904B43
:1067600000930022CDE90175A0211A602046012383
:10677000282204F05FFD322002F00AFD894B0093CD
:106780000126CDE9017546221E60A0213346204630
:1067900004F050FD322002F0FBFC834B0093CDE966
:1067A00001754A22C3F80080A0213346204604F038
:1067B00041FD322002F0ECFC7C4BCDE9017550220A
:1067C000C3F80080A02100932046334604F032FD38
:1067D000322002F0DDFC764B764A0093CDE901755C
:1067E000A0211A6020463346302204F023FD3220D7
:1067F00002F0CEFC704B00936FF07F42CDE9017543
:10680000A0211A6020463346342204F013FD3220C2
:1068100002F0BEFC694B6A4A0093CDE90175A021E4
:106820001A6020463346382204F004FD322002F07C
:10683000AFFC644B029506220192634A00931A60F2
:1068400040F205529A80A02133464022204604F0AF
:10685000F1FC322002F09CFC5C4B019742F2127278
:1068600002950093A0211A6020463346602204F06E
:10687000E1FC322002F08CFC554A564B106891889E
:10688000927902954FF010080093534F1860CDF89D
:106890000480204699809A71A2213346424604F032
:1068A000C9FC322002F074FC0FCFDFF848C1CDF8EC
:1068B00000C04FF020090295CDF80490CCF80C30C0
:1068C0003B78CCF80000CCF80410CCF808208CF809
:1068D00010304A463346A221204604F0ABFC322059
:1068E00002F056FC3D4A3E4B106812790295009327
:1068F00018601A710823019370223346A2212046A2
:10690000384F04F097FC322002F042FC0FCFDFF842
:10691000E8C0CDF800C0CDE90195CCF80C303B883B
:10692000ACF81030BB78CCF80000CCF80410CCF8F0
:1069300008208CF8123040223346A221204604F071
:1069400079FC322002F024FC274A029503CA274D25
:10695000CDF80480009569601188298191782860BC
:10696000A972334680222046A22104F063FC322023
:1069700005B0BDE8F04302F00BBC00BF20F60020DC
:10698000A0F5002040BD00200000204100000020B4
:1069900000009644F4BA0020000096C448BD0020D0
:1069A0006CBB002044BD002068BB002064BB0020FD
:1069B00054FA0020C0A8000A50FA00204CFA002027
:1069C000C0A80001C8FA002000125E017403002074
:1069D0009439020888BB00209C390208B0390208AB
:1069E000CCBB0020B8390208CC39020870BB0020AB
:1069F00000401C46DCBB0020A8BB00200A4A0B4B11
:106A000003CA70B40A4D0B4C2860696003CB0A4E70
:106A10001B882381336812782A722060616043F4F6
:106A20000063336070BC7047D8390208E43902084B
:106A30000CBC0020FCBB002020F600202DE9F04F0C
:106A400000248FB0CDE90844CDE90A44764B009488
:106A50000C941A6BDFF8DC81744EDFF8DCA1744F04
:106A6000DFF8D8B1DFF8D89142F010021A631A6B40
:106A700002F010020092009A01941A6B42F0040294
:106A80001A631A6B02F004020192019A02941A6BC3
:106A900042F020021A631A6B02F020020292029A5C
:106AA00003941A6B42F080021A631A6B02F08002A0
:106AB0000392039A04941A6B42F001021A631A6B50
:106AC00002F001020492049A05941A6B42F0020249
:106AD0001A631A6B02F002020592059A06941A6B69
:106AE00042F040021A631A6B02F040020692069AC4
:106AF00007941A6B42F008021A631B6B03F0080339
:106B00000793404601227C21079B04F037F8224678
:106B10003046402104F032F850460122102104F0A2
:106B20002DF822463846012104F028F8224658461E
:106B3000112104F023F8224640464FF2807104F000
:106B40001DF8224648464CF2B30104F017F801251F
:106B50004FF2FC7308A94046CDE90835CDE90A4457
:106B600003F030FE30464023022608A90893CDE901
:106B700009540B9603F026FE082208A950464FF44C
:106B80000413CDE908230A9403F01CFE1023504699
:106B900008A90893CDE909540B9603F013FE08A940
:106BA0003846CDE90855CDE90A4603F00BFE02222E
:106BB00008A938464FF44413CDE908230A9603F098
:106BC00001FE5846112308A90893CDE909560B96F2
:106BD00003F0F8FD404608A940F603020023CDE982
:106BE00008230A9403F0EEFD4FF40042384608A94A
:106BF0000023CDE908230A9403F0E4FD4CF2B3032B
:106C000008A948460893CDE909540B9403F0DAFD2E
:106C10000822002308A94846CDE908230A9403F076
:106C2000D1FD0FB0BDE8F08F0038024000140240E3
:106C30000004024000100240000002400018024020
:106C4000000C0240022800D0704708B5074B4FF4F3
:106C500080501968FFF7F8FB012803D0044B00228D
:106C60001A6008BDBDE80840FAF772BC20F60020A3
:106C70001CBB002082B002AB03E90300BDF8041086
:106C800002B003F07BBF00BF82B002AB03E9030098
:106C9000BDF8041002B003F075BF00BF82B002ABB4
:106CA00003E90300BDF8041002B003F061BF00BFA8
:106CB00010B50C480C4A0D4C0023C0E900424FF4BB
:106CC00080418022C0E90233C0E90413C0E90633E1
:106CD000026204F0E7F900B910BDBDE8104000F011
:106CE000BFBD00BFA0F50020801A06000054004080
:106CF00030B5174B026889B000249A42CDE90244AE
:106D0000CDE90444069401D009B030BD114D009482
:106D10002B6B114843F002032B632B6B03F0020330
:106D200000934FF4C0721223CDE9022302A9042379
:106D30000693009A03F046FD01942B6C43F4001374
:106D40002B642B6C03F400130193019B09B030BD3D
:106D500000540040003802400004024038B5134C93
:106D6000134D2368134823F44013236000220121AC
:106D700003F004FF01222021284603F0FFFE012238
:106D80008021284603F0FAFE00228021284603F0E5
:106D9000F5FE06484FF4806103F0EAFE236843F4F1
:106DA000801323600028DCD138BD00BF00100240F2
:106DB000000C02400014024070B51D4C002220213E
:106DC00006461C4803F0DAFE656805F071FC1A4BB4
:106DD000A3FB0032920C63685B1B9342FBD3154DFF
:106DE00080210122284603F0C9FE144A4FF0F063C7
:106DF00093613309DB019361B3039BB2C6F3810650
:106E00000F4AAA611E43AE61646805F051FC0A4B4B
:106E10000749A3FB0032920C4B681B1B9342FBD328
:106E2000BDE8704003480022802103F0A7BE00BFE8
:106E3000001000E0000C024083DE1B430010024003
:106E4000000003C010B50446FFF788FF0448002285
:106E5000012103F093FE2046BDE81040FFF7ACBFD0
:106E60000014024010B501EB810100EBC10000F0FD
:106E70007F04FFF773FF05480022012103F07EFE27
:106E800044F08000BDE81040FFF796BF00140240B8
:106E900010B50446FFF762FF01220448114603F0D3
:106EA0006DFE2046BDE81040FFF786BF001402408B
:106EB00070B504787CB1084E0546FFF74FFF0122FC
:106EC0001146304603F05AFE2046FFF775FF15F8CD
:106ED000014F002CF1D170BD001402402DE9804813
:106EE00091B0B94BB948BA4EDFF818A3DFF8188350
:106EF000DFF818B3B74F002502951A6B42F008026D
:106F00001A631A6B02F008020292029A03951A6B36
:106F100042F010021A631A6B02F010020392039AF5
:106F200004951A6B42F020021A631B6B03F02003D6
:106F30000493A0220123CDE90A230AA90022049B7D
:106F400000230124CDE90C2303F03CFCA2480A9461
:106F50000AA903F037FC4FF4F063A0480A930AA98A
:106F600003F030FC4CF2030398480A930AA903F09B
:106F700029FC214698482A4603F000FE2A46202193
:106F8000924803F0FBFD322002F002F93820FFF7AF
:106F900013FF204602F0FCF83820FFF70DFF2046D3
:106FA00002F0F6F80C20FFF707FF032002F0F0F8DC
:106FB0002046FFF701FF032002F0EAF80620FFF762
:106FC000FBFE032002F0E4F82046FFF73BFF8020A1
:106FD000FFF738FF8020FFF735FF8148FFF768FF94
:106FE000A820FFF72FFF7F48FFF762FF4FF4FA60FA
:106FF00002F0CEF82046FFF725FF8020FFF722FFA2
:107000008020FFF71FFF7848734CFFF751FFA8203F
:10701000FFF718FF7549764A0AA819F09DFC0AA8DF
:10702000FFF746FF4FF4FA6002F0B2F831684FF410
:107030008050FFF709FA002840F08E809AE803009C
:107040000A908DF82C100AAB3A46112105A819F0C8
:107050004DFCFFF783FE00220121204603F08EFD48
:107060008020FFF7A9FE9DF814507DB10DF11409A1
:10707000FFF774FE01221146204603F07FFD2846EB
:10708000FFF79AFE19F8015F002DF1D1594B5A4ACA
:10709000112105A819F02AFCFFF760FE002201214A
:1070A000204603F06BFD8620FFF786FE9DF8145006
:1070B0007DB10DF11409FFF751FE01221146204662
:1070C00003F05CFD2846FFF777FE19F8015F002DFD
:1070D000F1D1D8F800100120FFF7B6F905460028D5
:1070E00041D031684FF48050FFF7AEF98146002857
:1070F00040F09080DFF818C1BCE80F0005AD0FC567
:10710000DCF800302B70FFF729FE4A4601212046AB
:1071100003F034FDA820FFF74FFE9DF814507DB119
:107120000DF11409FFF71AFE01221146204603F063
:1071300025FD2846FFF740FE19F8015F002DF1D12B
:107140004FF47A700DF0E8FE31684FF48050FFF78D
:107150007BF900283FF472AF284B93E803000A90B4
:107160008DF82C106FE7DBF800202549130E0193F2
:10717000C2F30743009305A8C2F30723D2B219F064
:10718000EBFBFFF7EBFD2A460121204603F0F6FC5E
:10719000A820FFF711FE9DF81450002DD0D00DF15E
:1071A0001409FFF7DBFD01221146204603F0E6FC3F
:1071B0002846FFF701FE19F8015F002DF1D14FF4C9
:1071C0007A700DF0A9FEBFE700380240000C0240C3
:1071D00020F60020483A0208001402400010024045
:1071E000F0390208043A0208183A02082C3A020858
:1071F0004436020888BB0020543A0208403A02088C
:10720000643A0208383A020824F6002060FA0020A6
:10721000803A02081A4B112193ED000A07220D2330
:1072200005A8FEF70DFD05A8F8F7DCFF154A034693
:10723000106805AAD050FFF791FD002201212046D9
:1072400003F09CFCA820FFF7B7FD9DF81450002D1B
:107250003FF476AF0DF11409FFF780FD01221146CE
:10726000204603F08BFC2846FFF7A6FD19F8015FC6
:10727000002DF1D14FF47A700DF04EFE64E700BF9F
:10728000F8BA0020603A020810B588B0224B234CAF
:10729000002201921A6B42F008021A631B6B03F082
:1072A0000803019308220123CDE9022302A9002249
:1072B00020460023CDE90423019B03F083FA102329
:1072C00002A92046029303F07DFA202302A920465A
:1072D000029303F077FA402302A92046029303F0B9
:1072E00071FA0F4B012293E80300FFF7C3FC0D4B2B
:1072F000012293E80300FFF7BDFC0B4B012293E84A
:107300000300FFF7B7FC094B012293E80300FFF7E6
:10731000B1FC08B010BD00BF0038024000100240B0
:10732000746802086C680208646802085C680208F5
:107330002DE9F047DFF86891554FD9F800203B78E8
:10734000544EDFF86081544C544DDFF85CA1002AA4
:107350005BD0FF2B14BFD6E90001D8E90001002261
:10736000FFF788FC21684020FFF76EF802460028EE
:107370005BD195E80300FFF77DFC64200DF0CCFDA8
:10738000D9F800203B78002A6CD0FF2B14BFD6E937
:107390000001D8E900010122FFF76CFC21684020C0
:1073A000FFF752F8002857D021688020FFF74CF8EB
:1073B00000284BD095E803000122FFF75BFC216811
:1073C0000120FFF741F802469AE80300002A5BD04B
:1073D0000122FFF74FFC21681020FFF735F83B78BA
:1073E0000246002847D0FF2B14BFD8E90001D6E998
:1073F00000010122FFF73EFC4FF448700DF08CFDB8
:10740000D9F800203B78002AA3D1FF2B14BFD6E97E
:107410000001D8E900010122FFF72CFC216840207F
:10742000FFF712F802460028A3D021688020FFF75A
:107430000BF828B921684020FFF706F800289CD0F7
:1074400095E803000122FFF715FC96E7216840202C
:10745000FEF7FAFF0028B2D095E803000022FFF7FC
:1074600009FCACE7FF2B14BFD6E90001D8E9000105
:10747000FFF700FC92E7FF2B14BFD8E90001D6E923
:107480000001FFF7F7FBB7E7FFF7F4FBA3E700BF47
:1074900080BB00206C68020824F600207468020893
:1074A00028F60020646802085C68020830B50023F2
:1074B00095B0CDE90B33CDE90333CDE9053323494D
:1074C00001930D930793086C214A40F080500864A3
:1074D000096C01F08051019101990293136843F402
:1074E00080431360136803F48043029302244FF433
:1074F000800305204FF480310822CDE90E434FF47C
:10750000A873CDE90801CDE91023029801210222D8
:10751000072308A8CDE912230A9104F015FE08B14B
:1075200072B6FEE70F220346CDE903244FF4A055BF
:107530004FF4805203A80521CDE90535079205F0E7
:1075400019F808B172B6FEE715B030BD0038024038
:107550000070004080B501F0EFFDFFF7A7FFFFF7D7
:107560006DFAFEF73BFA08F045F9FFF78DFEFEF7DE
:1075700059FAFFF79DFBFEF791FFFFF73FFAFAF785
:10758000FDF901F0BFFB8548854C864D864E874F3F
:10759000DFF83882DFF83892F9F722FE01F07AFB43
:1075A0008348F9F71DFE01F091FB824982480122D0
:1075B00006F0B0FE00F052FC00F0BAFDF9F74CFF07
:1075C00001F0D4F801F098F8002204217B4803F080
:1075D000D5FA022001F0DCFD78480122042103F0F5
:1075E000CDFA00220321092002F02AF8032200210B
:1075F00001200CF099FB03220346002101202360A7
:107600000CF092FB03220021286001200CF08CFB7F
:1076100003223060002101200CF086FB0322386039
:10762000002101200CF080FB0322C8F8000000219B
:1076300001200CF079FB0322C9F800000021012091
:107640000CF072FB23685E4C2060002B5ED02A6831
:10765000002A52D03268002A6AD03A68002A70D0D4
:10766000D8F80020002A5AD0D9F80020002A7AD071
:1076700000286FD0184600231A4619460CF0BEFBAE
:1076800000231A46194628680CF0B8FB00231A4656
:10769000194630680CF0B2FB00231A4619463868C8
:1076A0000CF0ACFB00231A461946D8F800000CF089
:1076B000A5FB00231A461946D9F800000CF09EFBE2
:1076C00000231A46194620680CF098FB0022082176
:1076D00007200CF029FB3B4B186000284CD00022FF
:1076E000082107200CF020FB374A106000284CD0FE
:1076F000FEF78EFA0BF0F0FFFEE74FF0300383F356
:107700001188BFF36F8FBFF34F8FFEE74FF0300349
:1077100083F31188BFF36F8FBFF34F8FFEE74FF0F6
:10772000300383F31188BFF36F8FBFF34F8FFEE7F2
:107730004FF0300383F31188BFF36F8FBFF34F8F88
:10774000FEE74FF0300383F31188BFF36F8FBFF371
:107750004F8FFEE74FF0300383F31188BFF36F8F35
:10776000BFF34F8FFEE74FF0300383F31188BFF371
:107770006F8FBFF34F8FFEE74FF0300383F3118815
:10778000BFF36F8FBFF34F8FFEE74FF0300383F3EC
:107790001188BFF36F8FBFF34F8FFEE718F90020FA
:1077A0001CF6002018F6002014F600200CF600202D
:1077B000A8F90020F8F9002060F90020001002402C
:1077C000F8F5002008F60020FCF5002010F6002057
:1077D00004F6002038B50368B3F1804F03D01C4A8B
:1077E000934216D038BD1B4D044629684FF4805093
:1077F000FEF72AFE012829684FF480700DD0FEF7AD
:1078000023FEF8B9144A236800211160104A9342FC
:10781000E8D1BDE8384001F0A9BCFEF715FE48B13B
:107820000E4B012293E80300FFF724FAF9F790FECC
:107830002368D4E729684FF40050FEF705FE0028BE
:10784000EED1F3E7054B93E80300FFF71DFAD9E704
:107850000010004020F600201CBB00204C680208ED
:1078600072B6FEE730B583B0BE2308220DF10701E2
:1078700005468DF80730F9F7D9FC0A4C2378DA076A
:10788000FCD4094948222846F9F7E8FC2378DB07AD
:10789000FCD409210448F9F709FDB0FA80F0400949
:1078A00003B030BD880600203CF6002070B582B0E1
:1078B0000646002308460D468DF80730F9F79CFC74
:1078C000B0B1BEB1552308220DF1070128468DF84D
:1078D0000730F9F7ABFC0F4C2378D907FCD44022D2
:1078E00031462846F9F7A2FC2378DA07FCD40120B8
:1078F00002B070BDCC2308220DF1070128468DF897
:107900000730F9F793FC034C2378DB07FCD4012004
:10791000EEE700BF8806002010B50C46FFF7C6FF53
:1079200000B910BD2046BDE81040FFF79BBF00BF67
:1079300030B589B00C46FFF7B9FF08B909B030BDC2
:10794000482308220DF1070120468DF80730F9F78A
:107950006DFC154A1378DB07FCD401234FF48072C9
:107960000024002502A91148CDE90223CDE90445F0
:1079700002F028FF01224FF480710C4803F0FEF85A
:1079800032200DF0C9FA4FF480721223CDE90223A0
:107990000648072302A9CDE90445069302F012FF29
:1079A000012009B030BD00BF88060020000C024055
:1079B00030B583B00D46FFF779FF08B903B030BD8D
:1079C0004E2308220DF1070128468DF80730F9F7FC
:1079D0002DFC0A4C2378DA07FCD4094A094912889D
:1079E0000A807F23284618228B70F9F71FFC237822
:1079F000DB07FCD4012003B030BD00BF88060020A7
:107A0000C8BB002038F600202DE9F04F754B764EAC
:107A1000DFF81092DFF810B2DFF81082734F2DED0F
:107A2000028B0FCB8DB003AC002584E80F008DF8DE
:107A30000A506F4C6F4D9FED708A07E08BED008A06
:107A4000D8F8000041F288310CF060FC29684FF44E
:107A50008050FEF7F9FC30B129680420FEF7F4FCF1
:107A6000002840F0B78031680120FEF7EDFC00BB34
:107A70003846F9F7C1FB002800F0A280D9F80030A1
:107A8000002B00F0D5804FF0000A39465046C9F867
:107A900000A0FFF78DFF002800F08E805046394689
:107AA000FFF746FF002800F0878054495448FEF74E
:107AB00097FB29684FF48050FEF7C6FC28B931685F
:107AC0000120FEF7C1FC0028BAD14E48F9F794FB1B
:107AD0000028B3D000234B488DF80B30F9F78CFB0E
:107AE00000285DD0CC2347488DF80B3008220DF1DB
:107AF0000B01F9F79BFB2378D907C3F3000AFAD4EB
:107B00004048FFF7AFFE00284AD03F4B3D488DF874
:107B10000BA093F804A0F9F76FFB002840D0CC230A
:107B200038488DF80B3008220DF10B01F9F77EFB78
:107B30002378DA07FCD4442332488DF80A3008222F
:107B40000DF10A01F9F772FB237813F00103FBD161
:107B500001222E48019307A9CDE90933CDE9072277
:107B600002F030FE01221146284803F007F84FF4D6
:107B70007A700DF0D1F90122019B0792122223485D
:107B8000089207A90822CDE909330B9202F01AFEE8
:107B9000019B1C491846FFF7BFFE002840F0EB8010
:107BA0001B4A13680133092B13603FF647AF194B8B
:107BB0001B68CBF8003043E70920FEF71FFB78E78E
:107BC000154B164A18605860154B83ED008A012347
:107BD00013606EE731680120FEF736FC00283FF4A1
:107BE00042AF45E72435020824F6002018F90020AA
:107BF0008806002020F60020003C1CC6BC35020888
:107C0000DEE10020A8F900203CF600200000024040
:107C10002CF6002064030020D4BB002034F60020A2
:107C20000C00002084BB00200800002004F6002087
:107C3000332308220DF10A0138468DF80A30F9F78E
:107C4000F5FA237813F00103FBD1764A76491360E5
:107C500038464022F9F702FB94F800A01AF0010A16
:107C6000FAD171480721F9F721FB002879D16D4A33
:107C70008DF80B00012338461360F9F7BDFA002890
:107C800060D0CC2308220DF10B0138468DF80B3063
:107C9000F9F7CCFA2378DA07C3F3000AFAD43846A6
:107CA000FFF7E0FD00284DD0604B8DF80BA0384663
:107CB00093F804A0F9F7A0FA002843D0CC230822B7
:107CC0000DF10B0138468DF80B30F9F7AFFA237838
:107CD000DB07FCD4442308220DF10A0138468DF855
:107CE0000A30F9F7A3FA237813F00103FBD101223C
:107CF000CDE909334E48019307A94FF48073CDE9CC
:107D0000073202F05FFD01224FF48071484802F013
:107D100035FF4FF47A700DF0FFF84FF4807307933E
:107D20001222019B4248089207A90722CDE9093394
:107D30000B9202F047FD019B3E491846FFF7ECFD10
:107D4000002844D13C4A13680133092B13600ED834
:107D50003A4B3B4A1B681360344B3A4A5B881380AA
:107D6000A7E6314BC3F800A0C3F804A0A1E6344B4A
:107D700083ED008AF0E73448F9F73EFA0CAACAF31B
:107D8000411302EB830353F8240C284B1B88184043
:107D9000F8F7D8FB2D4B0022F8F73EFCF8F7F6FE7B
:107DA0009FED2B7ACBF8000007EE900AF4EEC77A2D
:107DB000F1EE10FA03DD274B1B68CBF80030254AA3
:107DC000DBF800301360244A0023136038E61948BA
:107DD000F9F712FA0CAACAF3411302EB830353F822
:107DE000240C124B1B881840F8F7ACFB0022174BF1
:107DF000F8F712FCF8F7CAFE9FED157A104A07EE65
:107E0000900AF4EEC77AF1EE10FA106002DD0B4B27
:107E10001B6813600A4B094A1B681360064A00235B
:107E2000136099E734F60020D4BB00203CF6002014
:107E3000000C024018F9002030F6002068030020F2
:107E40000C000020C8BB0020A8F900200000B03FB3
:107E50000000A042640300202CF6002000B5284852
:107E6000284987B07F2200238260FF22CDE90133B9
:107E7000CDE90333C0E90013C0E90323C0E90533AA
:107E80000593009304F0AEFD68BB1D48012104F08A
:107E90005FFF43F2F223984202D107B05DF804FB82
:107EA00000221748ADF8042001A9CDE904228DF87D
:107EB000062004F0E1FDC8B9134B114800930022DD
:107EC000694604F057FEB8B900220D48114604F087
:107ED000C7FE70B90A4843F2F222012104F032FFD2
:107EE00007B05DF804FBFFF7BBFCCEE7FFF7B8FC7B
:107EF000E2E7FFF7B5FCEDE7FFF7B2FCE4E700BF10
:107F000048F60020002800400202181A00B50F4A67
:107F1000016885B000239142CDE9013302D005B05C
:107F20005DF804FB02224FF48073684600920393CD
:107F300004F006FC30B9064B0122C3F83C2E05B014
:107F40005DF804FBFFF78CFCF5E700BF002800405C
:107F500000004742054B064800220121C3E9000208
:107F6000C3E90222C3E904229961704740F7002067
:107F7000002C01402DE9F041524B02688AB00024E8
:107F80009A42CDE90444CDE90644089402D00AB0EF
:107F9000BDE8F08103F5863301945A6C42F4006227
:107FA0005A645A6C02F400620192019A02941A6BAC
:107FB00042F004021A631A6B02F004020292029A5F
:107FC00003941A6B42F008021A631B6B03F0080358
:107FD0004FF4F852039303270C26022304A9054605
:107FE0003948CDE90423CDE90776039B4FF0040817
:107FF00002F0E8FB02233548089604A9344ECDE987
:108000000483CDE9064702F0DDFB4FF480534FF4C3
:1080100080614FF48040C6E904132023C6E90603BB
:108020004FF400024FF44033C6E90A723362294A22
:10803000C6F824804FF40013336330464FF00063DA
:10804000C6E90244C6E9002301F076FBA0BB224C3E
:10805000224B23604FF000614023C4E9011300224A
:108060004FF48063C4E903234FF480514FF48043FD
:10807000C4E9051320224FF44033C4E90723042147
:108080000323C4E909134FF400024FF400132E64D4
:108090002046C4E90B23B56301F04EFB78B90022FA
:1080A0000521EC633120A56301F0CAFA312001F00B
:1080B00003FB0AB0BDE8F081FFF7D2FBC7E7FFF78B
:1080C000CFFBECE7002C014000080240000C02400E
:1080D000E0F600205864024080F60020A0640240D0
:1080E0000F4B02689A4200D070470E4A536C10B58D
:1080F00023F40063044653640B484FF4F85102F034
:108100007DFC0421094802F079FC206C01F0A8FBF9
:10811000E06B01F0A5FBBDE81040312001F0DABAB8
:10812000002C01400038024000080240000C0240D0
:1081300010B51149114C4FF482720023C4E90012AA
:1081400001204FF40072C4E904300821A2612046E6
:108150000A22C4E90233C4E90713C4E90933E2621D
:1081600005F026FC28B92268136843F04003136029
:1081700010BDFFF775FBF6E700300140C8F700209F
:1081800030B5294B02688BB000249A42CDE90444F3
:10819000CDE90644089401D00BB030BD03F584331B
:1081A00001945A6C214842F480525A645A6C02F489
:1081B00080520192019A02941A6B42F001021A63F2
:1081C0001A6B02F001020292029A03941A6B42F0B7
:1081D00002021A631B6B03F0020303936022022363
:1081E000CDE904230525022204A90323CDE90623B2
:1081F0000895039B02F0E6FA20220223CDE904232E
:1082000004A9032300220A480895CDE9062302F0B9
:10821000D9FA22462946232001F012FA232001F040
:108220004BFA0BB030BD00BF0030014000000240EF
:108230000004024082B00E4B00220092596C41F4BF
:1082400080415964586C00F480400090009801927D
:10825000186C40F0805018641B6C03F0805301933D
:10826000019B0F216FF0010002B001F0E9B900BFDE
:108270000038024070B588B0234B002202921A6C7D
:1082800042F010021A641B6C03F0100302930546BF
:1082900001A903A8029B04F031FA069BD3B904F0AC
:1082A0000DFA0346194A1A4C1A49A2FB03239B0CE8
:1082B000013B0022C4E90013204640F2E73322616B
:1082C000A260A261E36005F097FE064630B1304639
:1082D00008B070BD04F0F2F94300E3E7204605F072
:1082E0007BFC06460028F2D1362001F0E5F90F2D7F
:1082F00001D90126EBE732462946362001F0A0F9E4
:10830000054B1D60E3E700BF0038024083DE1B43DE
:1083100020F80020001000407C030020FEE700BF92
:10832000FEE700BFFEE700BFFEE700BFFEE700BFBD
:10833000704700BF014805F053BD00BFB8F80020EA
:10834000014805F099BB00BFC8F70020014806F0BE
:1083500079B800BF60F9002010B5044C2046F8F74A
:10836000C9FF2046BDE8104006F06CB818F900209F
:10837000014805F0F3B900BF40F7002010B5044CE8
:108380002046F8F7B7FF2046BDE8104006F05AB87F
:10839000A8F90020014805F023BD00BF20F8002007
:1083A000014801F033BB00BFE0F60020014802F0B5
:1083B0009DB800BF28FB0020014803F0ABB900BF07
:1083C000ACD00120014801F021BB00BF80F60020A5
:1083D000014B988802F0E0BB54680208014804F0A1
:1083E00097BC00BF48F60020704700BF704700BF31
:1083F00001207047024B16221A604FF0FF30704781
:10840000CCD60120014B16221A60FEE7CCD6012003
:1084100070B5161E07DD0C468D19AFF3008004F809
:10842000010BA542F9D1304670BD00BF70B5161ED4
:1084300007DD0C468D1914F8010BAFF30080A5423F
:10844000F9D1304670BD00BF4FF0FF30704700BF1C
:108450004FF400534B600020704700BF012070476D
:10846000002070470D490E4A0B6810B40D4C121BCA
:1084700083B11844904204D808605DF8044B184654
:108480007047094B5DF8044B0C221A604FF0FF3324
:1084900018467047054B0B60EBE700BF68F80020FB
:1084A0000000022000040000CCD60120E0D601200C
:1084B000034AD2F8883043F47003C2F8883070471A
:1084C00000ED00E02DE9F04F9BB00023DFF818929B
:1084D0007D4FDFF818B2DFF81882DFF818A2059395
:1084E0001D461E460022114610200DF0BDFB04461D
:1084F0000028F7D042F2117200210DF035FC40B98E
:10850000FF2120460DF08CFC05A920460DF0ACFCA7
:1085100018B120460DF008FCE4E7039020460DF06A
:108520001FFE20460DF000FC059C684B6268186831
:10853000518B039B41F040015183654904324FF058
:108540000A0C0A60C4F81CC01A4619460BF056FC07
:10855000059806A90DF0F2FC002832D00A30C0F2CE
:1085600097805C4B1A68002A40F08D805A4B19683E
:10857000002940F09B801F2409E0DDE908120598DE
:1085800000960DF0DFFD00286CD1013C08D0D8F832
:1085900000000A2208A90BF0FFFD01280346ECD0D9
:1085A00001200CF0B9FCD3E70598009601230422C2
:1085B00051460DF0C7FD002506980FF0BFF80028C2
:1085C00059DB06980DF1120207A90FF085F899F80A
:1085D000004014F0FD04E7D1BDF81210022389F821
:1085E000003019B9E8E70134A142E5D9079B1B5DCA
:1085F00005F168020DEB0200FA5C02F00302022AA8
:1086000004BF203BDBB20D2B05F1010500F8403C17
:1086100014D03F2DE7D95146059800960123042236
:108620000DF090FDDBF800100120FDF70DFF98B96B
:1086300089F80060BDF812100025D4E70AA900F8F7
:10864000406C264818F06FFB2549002308681A463D
:1086500019460BF0D3FBEDE7224A00211020FDF76D
:10866000F9FEE5E71F4A00211020FDF7F3FE012087
:108670000CF052FC6CE706980EF0BEFF154B1A6822
:10868000002A3FF473AF0123134A1360114B1E609D
:10869000DBF800100120FDF7D7FE48B905980DF072
:1086A0005FFD05980DF040FB05961BE71346EBE7D1
:1086B0000C4B4FF480501968FDF7C6FE0028EDD131
:1086C000F9F7B4F9EAE700BFA9700208F8F500204D
:1086D0007003002098E4002094E400209CE4002033
:1086E0001CF6002020F60020DEE1002024F6002009
:1086F00008F60020903D020800B51A484FF080426D
:1087000087B00260184A0023CDE90233CDE9043373
:10871000CDE90033C0E90133C0E90323836105F0EB
:108720006BFC98B94FF480530E48029302A905F0F0
:10873000A5FA98B9102200230A486946CDE900231A
:1087400005F088FC28B907B05DF804FBFFF788F84E
:10875000E8E7FFF785F807B05DF804FBFFF780F85E
:10876000E8E700BFB8F800207F2C800000B51A4869
:108770001A4A87B002605322002342604FF0FF3252
:10878000CDE90233CDE90433CDE90033C0E902324B
:108790000361836105F030FC98B94FF480530E48B3
:1087A000029302A905F06AFA98B9002200230A4848
:1087B0006946CDE9002305F04DFC28B907B05DF806
:1087C00004FBFFF74DF8E8E7FFF74AF807B05DF85C
:1087D00004FBFFF745F8E8E770F80020000C0040C4
:1087E00000B50368B3F1804F83B014D0154A9342AB
:1087F00002D003B05DF804FB134B002201921A6C07
:1088000042F008021A641B6C03F008030193019BF9
:1088100003B05DF804FB03F50E3300220092196CDF
:1088200041F0010119641B6C03F001030093032163
:108830001C20009B00F004FF1C2003B05DF804EB3B
:1088400000F03ABF000C00400038024010B5464C22
:10885000034607CC454C18609A606278DA73A278B8
:10886000434859601A74E27821785A7422799973CE
:108870009A744049027864791A754FF0310C827805
:10888000A3F80CC0DC7490F801C0C4789A754878DD
:108890000A7883F815C0DC751A768A785876C87815
:1088A000D8763548354C9A76354A0078217883F861
:1088B0002B00107892F801C01977302183F82D1021
:1088C00083F82E1083F82F1000F00F00D17894F861
:1088D00001E083F81DE000EB0C1092F804C083F86F
:1088E000300001F00F01907901EB0C1183F8311089
:1088F00092F807C0117A527A00F00F0000EB0C10CA
:1089000001F00F0194F802C083F8320001EB02116C
:10891000E0781C4A1C4C83F833105C62002141F261
:1089200027141C62D87783F81EC03320198583F87A
:108930002A105178147883F82C0083F83510907839
:10894000D17883F8344083F836001479507983F86D
:1089500037109179D27983F8384083F8390083F859
:108960003A1083F83B2010BD983D0208C8FA002059
:1089700054FA002050FA002080BB00204CFA00205E
:10898000A8BB002088BB0020B16B00B52DE9F04FDB
:108990005B4F5C4C8BB00022114620200DF064F937
:1089A00038600028F7D047F2FF7221460DF0DCF95D
:1089B0000028F0D1544D554EDFF86C81DFF86C91F2
:1089C0000AE049462046F7F703FC40B328680EF05A
:1089D00013FE30680EF010FE294638680DF0AEFA2E
:1089E0000EF0FEFD3C2130600EF018FE05A9824617
:1089F0000DF1120228680EF06FFE059C41462046DC
:108A0000F7F7E6FB0028DCD15046FFF71FFF404A8E
:108A10003168386847F2FF730DF0EEFAD6E73D494A
:108A2000062204F10C0018F02AF80028ECD1D4F842
:108A30001200D4F81610D4F81A20E48B0DF11A03A2
:108A4000009306AB07C34FF0040B1C804FF47A74FD
:108A500001233022A021CDE901B42F4802F0EAFB26
:108A6000322000F095FB0DF11E033422A021CDE948
:108A700001B400932848012302F0DCFB322000F00F
:108A800087FB0DF122033822A021CDE901B4009328
:108A90002148012302F0CEFB322000F079FB1F4B6E
:108AA00001201968FDF7D0FC83460028ACD10121D4
:108AB000FEF7D8F91A48FEF7FBF901215846FEF7F0
:108AC000D1F91848FEF7F4F94FF4967000F060FB06
:108AD0002E20FEF7DDF94FF4967000F059FB2E20A2
:108AE000FEF7D6F94FF4967000F052FB2E20FEF7F9
:108AF000CFF9204600F04CFB00F0FEFD84E700BFFC
:108B000008F90020606E020804F9002000F9002036
:108B10005C6E0208C8FA0020A0F5002024F60020B0
:108B2000C83D0208D83D0208A83D0208B83D020829
:108B30002DE9F04F4B4D4C4EDFF848B1DFF848A11E
:108B4000DFF84881DFF8489185B0002211462020E7
:108B50000DF08AF828600EF043FD2A6830609AB163
:108B6000D8B11046494642F211720DF0FDF8C0B17D
:108B700030680EF041FDD8F8000000210BF03AF803
:108B800028680DF0D1F8E0E718B10EF035FD2A683D
:108B90001AB964200CF0C0F9D7E710460DF0C4F8FC
:108BA000F7E7324BC82118680BF0B0FB0128DFD182
:108BB000BBF80020DAF8001028680DF003F92C4B00
:108BC0002C491B68032207460A70F3B901932A4B0C
:108BD0001B68002B44D11F24D8F800000A2202A9E8
:108BE0000BF0DAFA012809D1BDF80C20029930689F
:108BF0000EF044FD08B35FBB013CEDD101200CF049
:108C00008BF91B4B1B68002BE1D001231A4A136020
:108C1000174B00221A60194B01201968FDF714FC4C
:108C20000028A5D0164B4FF480501968FDF70CFCB6
:108C300000289DD1F8F7FAFE9AE7BBF80030DAF881
:108C40000020316828680DF0D7F90746002FD3D0EF
:108C50000B4A00211020FDF7FDFBF8F7E7FECDE7FA
:108C6000019BD3E710F900200CF90020F8F5002053
:108C700098E40020DDE1002094E4002024F60020A8
:108C800020F600207403002070030020FCF5002073
:108C9000606E020810B50B480B4C00234FF4E13115
:108CA0000C22C0E90041C0E90233C0E90432C0E946
:108CB000063305F0DBFA00B910BDBDE81040FEF741
:108CC000CFBD00BFA8F90020004C004010B50B48F4
:108CD0000B4C00234FF4E1310C22C0E90041C0E904
:108CE0000233C0E90432C0E9063305F08DFA00B959
:108CF00010BDBDE81040FEF7B3BD00BF60F9002015
:108D00000010014010B50B480B4C00234FF4E1312B
:108D10000C22C0E90041C0E90233C0E90432C0E9D5
:108D2000063305F0A3FA00B910BDBDE81040FEF708
:108D300097BD00BF18F90020004800400000000067
:108D400030B50368564A8FB000249342CDE90844F9
:108D5000CDE90A440C9407D0524A93422DD0524A8E
:108D6000934269D00FB030BD504B01941A6C5048FB
:108D700042F400221A641A6C02F400220192019A51
:108D800002941A6B42F001021A631B6B9FED407B49
:108D900003F00103029308A908238DED087B0C93CF
:108DA000029A01F00FFD22460621342000F048FC13
:108DB000342000F081FC0FB030BD3C4B03945A6C62
:108DC0003B4842F010025A645A6C02F010020392BF
:108DD000039A04941A6B42F001021A631A6B02F0B0
:108DE00001020492049A05941A6B42F002021A637B
:108DF0001B6B03F0020305934FF48062072508A95B
:108E00000223CDE908230C95059B01F0DBFC02232E
:108E1000402208A927480C95CDE90823CDE90A444A
:108E200001F0D0FC22460521252000F009FC252078
:108E300000F042FC0FB030BD1C4B06941A6C1E486B
:108E400042F480221A641A6C02F480220692069A76
:108E500007941A6B42F008021A631B6B9FED0E7B9E
:108E600003F00803079308A907238DED087B0C93F3
:108E7000079A01F0A7FC22460621272000F0E0FB1C
:108E8000272000F019FC0FB030BD00BFAFF3008009
:108E900001000000120000000001000012000000AC
:108EA000004C0040001001400048004000380240E3
:108EB0000000024000040240000C024070B52D4B3F
:108EC00002689A4282B03DD02B4C237813F0FB0FFE
:108ED0000FD02A4B2A492B48002405221C6005F09C
:108EE000FDF929492748012202B0BDE8704005F08C
:108EF00011BA254B254A1B78204DD25C02F00302A3
:108F0000022A08BF203B4FF0040108BFDBB22A68E9
:108F100021701F490D2B8B541AD001323F2A01DCDE
:108F20002A60DEE716491748002605222E6005F064
:108F3000D5F9184B01201968FDF786FAA0B900236E
:108F40002370CEE714491548012205F0E3F9BBE789
:108F5000002313488B542B6017F0E5FE114B01A939
:108F600018680BF0C3F8BCE70F4A31461020FDF734
:108F700071FAE4E700480040DEE10020F4F9002047
:108F80009468020860F90020F8F90020A97002082E
:108F9000FCF9002024F60020F0F9002018F9002048
:108FA0009CE400201CF6002020F60020DFF834D0DE
:108FB000FFF77EFA0C480D490D4A002302E0D45811
:108FC000C4500433C4188C42F9D30A4A0A4C002313
:108FD00001E013600432A242FBD317F07DFEFEF7DE
:108FE000B9FA70470000022000000020600600204F
:108FF000B872020860060020DCD60120EFF305807D
:1090000000BEFEE780B1CB6873B18A6862B130B44C
:109010000C6964B1D1E90051C0E90423C0E90251EF
:109020008461002030BC70474FF0FF3070474FF034
:10903000FF30F7E770B5446882B0002301931CB19C
:109040000026304602B070BD8368054603B19847DC
:1090500020232B60002607E0019B03F01F03A3429F
:1090600015D00134202C0BD06B6901AA12212046A7
:1090700098470028F0DA0134202C6FF00406F3D171
:109080002B681F2B07D81EB1304602B070BD2C6074
:1090900001236B60D4E76FF00206D2E730B583B0EE
:1090A000002543690195044601AA006801219847FB
:1090B000A8423DDB6369206801AA01219847002886
:1090C00036DB019B5B072AD56369206801AA294624
:1090D000984700282CDB019BDD0414D563692068C8
:1090E00001AA1F219847002822DB019BDA041DD525
:1090F00003F01C03182B17D0082B13D0142B0BD103
:10910000042003B030BD03F40452B2F5045F0BD069
:10911000980407D4D905F3D4052003B030BD01204D
:1091200003B030BD0320F8E70220F6E70620F4E79D
:109130006FF00400F1E700BF08B50B4B1A6842F46A
:1091400000721A601A6842F480621A601A6842F467
:1091500080721A60032000F061FA0F20FFF78AF88E
:10916000FFF768F8002008BD003C0240034A044BAA
:1091700011681B780B441360704700BF3CFA002055
:1091800078030020014B1868704700BF3CFA0020AC
:1091900038B50446FFF7F6FF631C054602D0044BC2
:1091A0001B781C44FFF7EEFF401BA042FAD338BDEA
:1091B00078030020002800F09E8038B5056C044636
:1091C0003DB1236CDB060CD5002384F83C30012034
:1091D00038BDF8F785F96564236C84F83C50DB06EC
:1091E000F2D4236C474A23F4885323F0020343F05C
:1091F000020323645168236821F4403151605168AF
:109200006068014351605A682069A16822F4807245
:109210005A605A6842EA00225A605A68E06822F0AE
:1092200040725A605A680A435A609A68A16A22F4E6
:1092300000629A609A6802439A60334A91429A683F
:1092400051D022F07062E06A9A609A681143996086
:109250009A6822F040529A609A6802439A609A682B
:1092600022F002029A609A68217E42EA41029A60E4
:1092700094F82020002A40D05A68616A42F40062C3
:109280005A605A6822F460425A605A68013942EAC8
:1092900041325A60DA6AE16922F47002DA62DA6A0B
:1092A000013942EA0152DA629A68616922F4007275
:1092B0009A609A6894F8300042EA40229A609A686C
:1092C00022F480629A609A68002042EA81229A60C1
:1092D0006064236C23F0030343F001032364002341
:1092E00084F83C3038BD22F070629A609A6822F0AF
:1092F00040529A60B3E7012070475A6822F4006236
:109300005A60C7E7002301400100000F10B490F835
:109310003C3083B00022012B019268D00123026807
:1093200080F83C309368DB0714D4354B354C1B6810
:109330009168A4FB03439B0C03EB430341F0010141
:1093400091600193019B2BB1019B013B0193019B18
:10935000002BF9D1936813F0010F036C37D023F47D
:10936000E06323F0010343F48073036453685C05F6
:1093700005D5036C23F4405343F480530364036C1A
:1093800013F480531CBF436C23F0060343646FF057
:1093900022011D4B002480F83C4011605968C8062A
:1093A00021D11A498A4209D001F580718A4223D01D
:1093B00017498A4212D15B68DB060FD4936813F019
:1093C000405F0BD1936843F08043936006E043F025
:1093D00010030364436C43F001034364002003B0B3
:1093E0005DF8044B7047094B9A42F7D1E6E702203B
:1093F00003B05DF8044B70475B68D906DED0EDE73B
:109400006C03002083DE1B43002301400020014049
:109410000022014003689A6870B50D465105044664
:1094200002D59B68DA0544D4FFF7ACFE22680646F5
:109430001368990704D46B1C23D113689807FCD5D3
:109440006FF012031360236C43F40073236493687A
:1094500013F0405F13D1237E8BB9D36A13F4700FDE
:1094600002D093685A050AD4236C23F480732364D2
:10947000236CDB0403D4236C43F00103236400203A
:1094800070BD5DB9136813F00203D1D1226C84F86A
:109490003C3042F004022264032070BDFFF772FEEC
:1094A000801BA8422268C3D9136813F00203BFD1FE
:1094B000ECE7036C002243F0200380F83C200364B7
:1094C000012070BD0368D86C704700BF70B590F87C
:1094D0003C3082B00246012B4FF00000019000F0BA
:1094E0009380012382F83C300D6813688C68092D45
:1094F000A8B228D81E6905EB450E4FF0070C0CFAF0
:109500000EFC26EA0C061E611E6904FA0EF43443B2
:109510001C614C68062C04EB84012AD85C6B05396D
:109520004FF01F0C88400CFA01F124EA0101596345
:10953000596B0843586336498B422BD0002082F880
:109540003C0002B070BD00EB400CDE68ACF11E0CBC
:109550004FF0070E04FA0CF40EFA0CFC26EA0C0687
:10956000DE60DE683443DC604C68062C04EB84016A
:10957000D4D90C2C34D81C6B23391F26884006FA0A
:1095800001F124EA01011963196B084320491863AA
:109590008B42D3D1122D30D0A5F11003012BCDD8A1
:1095A0001C494B68102D43F400034B60C6D11A4B85
:1095B00001F146711B6801F52E3101F28331A1FBE7
:1095C00003139B0C03EB83035B000193019B002BB4
:1095D000B4D0019B013B0193019B002BF9D1ADE776
:1095E000DC6A41391F26884006FA01F124EA0101AC
:1095F000D962D96A0843D8629DE7D1F8043343F4AD
:109600008003C1F8043399E7022002B070BD00BFA7
:1096100000200140002301406C0300200749CA6874
:1096200003024FF6FF0003F4E0630240134343F0EC
:10963000BF6343F40033CB60704700BF00ED00E030
:109640001B4BDB68C3F3022300B5C3F1070EBEF169
:10965000040F03F1040C28BF4FF0040EBCF1060FF9
:109660001CD9A3F1030C4FF0FF3303FA0CF322EAE9
:1096700003024FF0FF3303FA0EF321EA030303FA68
:109680000CF313431B010028DBB20ADB00F160403E
:1096900000F5614080F800335DF804FB0022944639
:1096A000E7E7044A00F00F00024413765DF804FB7C
:1096B00000ED00E0FCEC00E0002807DB044A410973
:1096C000012300F01F00834042F82130704700BFA3
:1096D00000E100E000280CDB4309064900F01F0010
:1096E00020330122824041F82320BFF34F8FBFF384
:1096F0006F8F704700E100E0BFF34F8F0549064BC5
:10970000CA6802F4E0621343CB60BFF34F8F00BF1F
:10971000FDE700BF00ED00E00400FA05002808DBCB
:109720004309044900F01F0001226033824041F8E0
:109730002320704700E100E038B50446FFF722FD22
:10974000002C6BD023680022022184F8351084F8A5
:1097500034201A6822F0010205461A6005E0FFF77E
:1097600011FD431B052B37D823681A68D107F6D49F
:10977000D4E90120E16802430A43D4E90451A06915
:109780002A430A43E1691D6802430A4331492940DB
:10979000256A2A430A43616A042924D01A605A6957
:1097A00022F007021143D8B22B4A59611038A2FBAC
:1097B0000052120929496FF30903895CE1655F28AA
:1097C00088BF04333F228A40A36500209A600123AA
:1097D000606584F8353038BD03232022626584F843
:1097E0003530184638BDD4E90B512943114319606F
:1097F0005969A26A21F00701114341F00401002DCB
:10980000D1D068B9012A21D032F00202CBD1EA01CD
:10981000C9D540220123626584F83530012038BD66
:10982000B0F5005F04D0022AF3D9032AEFD0BAE7DB
:10983000032AB8D801A050F822F000BF13980008FE
:109840000F980008139800084D980008B5F1C07FE4
:10985000A9D1DEE73F8010F0ABAAAAAA9C68020853
:10986000002835D090F83520022A0346D0B22ED0F9
:109870001A681849D0B2103830B4A1FB0041090968
:109880001468154D24F001046D5C14600021116012
:1098900051609160D1601161212151615F286FF3A6
:1098A000090288BF04323F240021AC40DD65C3E9D2
:1098B0000F11C3E91111C3E913119A659460596539
:1098C00083F8341083F83510084630BC7047704771
:1098D00001207047ABAAAAAA9C68020870B490F84D
:1098E0003440856D012C0AD090F835404FF0010CC2
:1098F000644580F834C005D0002380F8343002205D
:1099000070BC7047022680F8356004680026466502
:10991000266826F48026266063608368402B0EBF8D
:10992000A260A160E260C26D08BFE1603F23934086
:10993000AB602368026C43F0160323601AB12368FE
:1099400043F008032360236843F0010300202360F1
:1099500070BC704770B50446866DFFF713FC94F831
:109960003530022B06D080236365002384F8343021
:10997000012070BD23681A6822F016021A605A6925
:1099800022F080025A61226C054642B31A6822F026
:1099900008021A601A6822F001021A6005E0FFF757
:1099A000F1FB431B052B10D823681B6813F0010340
:1099B000F5D1E16D3F228A40184601210023B260B3
:1099C00084F8351084F8343070BD0323202262659A
:1099D000184684F83530002384F8343070BDA26C0A
:1099E000002AD3D1D6E700BF90F83530022B03D040
:1099F00080234365012070470268052380F83530D5
:109A0000136823F00103002013607047F0B583B0A2
:109A1000674A876D166800230193C36D3D6808226D
:109A20009A402A42044603D001680868400778D467
:109A300001229A402A4203D02168496908066AD463
:109A400004229A402A4203D02168096889075CD41D
:109A500010229A402A4203D021680868000741D4A6
:109A600020229A402A4214D021680868C00610D5E6
:109A7000BA6094F83520052A63D00B6813F4802F60
:109A80000B687ED0190340F18980E36B0BB120464F
:109A90009847636D23B3636DDA071AD52268454989
:109AA000052384F835301368A1FB061623F0010363
:109AB000B60A136002E01368DB0704D5019B01338B
:109AC000B3420193F7D90122002384F8352084F8AA
:109AD0003430E36C23B1204603B0BDE8F0401847B2
:109AE00003B0F0BDBA600A6812F4802F0A6822D170
:109AF000D20503D40A6822F008020A60226C002A08
:109B0000AED020469047E36DAAE7BA60626D42F09E
:109B1000040262659CE7BA60626D42F0020262650F
:109B20008EE7086820F004000860BA60626D42F0B9
:109B3000010262657CE71103E0D5A26C002AE0D146
:109B40008EE70A6822F016020A604A6922F0800253
:109B50004A61226C3AB30A6822F008020A603F2286
:109B600002FA03F3216DBB600122002384F8352043
:109B700084F834300029B3D0204603B0BDE8F0406B
:109B8000084713F4807380D10A6822F010020A603B
:109B9000012284F8352084F8343076E7636C002B9A
:109BA0007FF475AF75E7A26C002AD4D1D7E700BF68
:109BB0006C030020B5814E1B406D70472DE9F043CA
:109BC000876A8E6800EB870CDCF818301C68002C64
:109BD0007CDBDCF82C40002C78D134689C605C681D
:109BE00075686FF30C042C430D685C609146EA07BE
:109BF00006D51C6824F4400E4C694EEA04041C602F
:109C0000AC0605D50C69196821F040612143196043
:109C10006A0703D5196841F0800119601968B468B2
:109C200041F080511960002C7DD0DFF804E13D4601
:109C300001262AE041F0804119606B1C032B94BF80
:109C40001D46033D00EB85018B69D3F80080B8F118
:109C5000000F26DBC96A21BB1968D4F8008062684E
:109C600021F080511960C3F80880596801EA0E019B
:109C700011435960BFF35F8F1968A46841F0004138
:109C800006F10108196024B34646196821F0005115
:109C900019601968B9F1000FCCD121F08041196029
:109CA000CBE7DCF818208EB10021BFF35F8F13687B
:109CB0007C1C032C23F000438CBF033F274613601A
:109CC000013100EB8703B1429A69EED10220BDE871
:109CD000F083DCF818101A68B9F1000F1FD042F0B9
:109CE00080421A601A6842F000521A60BFF35F8F18
:109CF0000B68C26B43F000430B6000EB8503DA6234
:109D00008562EFF31082012383F31088036C013323
:109D10003344036482F310880020BDE8F08322F00E
:109D200080421A60DEE73D4626461946D3E700BF6B
:109D300000E0FFFF70B58B680C46D1E905120B43BC
:109D4000616A1343A27B05460B43E07F217F43EA10
:109D5000426343EA004343EA013321792A6843EA34
:109D60008123E17B106843EAC11394F8281043EA89
:109D700001132B4901400B43217CB1FA81F14909C0
:109D800043EAC153617CB1FA81F1490943EA815345
:109D9000A17FB1FA81F1490943EA413394F82010D7
:109DA000B1FA81F1490943EA4123136001201668A1
:109DB000FFF7EEF92968A26C236D0E60886943EA0B
:109DC000024394F84C204FF6417C00EA0C00B2FAB2
:109DD00082F25209034343EAC21394F8552094F8DF
:109DE0005600A2F10102B2FA82F2520943EAC2031A
:109DF00094F85420A0F10100B0FA80F0A2F1010221
:109E00004009B2FA82F243EA8003520943EA42036C
:109E10008B6101208C69FFF7BBF92B689C6170BDD9
:109E20000F8120FD70B54B6902680C46096A0B432F
:109E3000617B43EA4163A17B43EA4153217F43EACB
:109E4000C113A17F02F5805243EA811394F82410D4
:109E5000054643EA810390691A4901400B43217B7F
:109E6000B1FA81F1490943EA8163617FB1FA81F175
:109E7000490943EA0153936101209669FFF788F984
:109E80002A68A368A169A06A02F580520B43966113
:109E900094F8251043EAC11321690B4321680B4351
:109EA000217943EA800343EA416343F400031360EA
:109EB00001201468FFF76CF92B6803F580531C60D0
:109EC00070BD00BF233FDEF82DE9F041D0E91A78DC
:109ED00082B007F11203002250F82340204E019275
:109EE0000546B8F1000F18D0236A83B3AA6D6B69D9
:109EF0004ABB3343636023687A1C032A43F0004360
:109F00008CBF033F1746236007F1120308F1FF38A7
:109F100055F82340B8F1000FE6D1EB6E43450FD062
:109F2000BFF35F8F2A682969FB1C03F0030303EB6F
:109F3000830302F5805201EBC3019160C5E91A78F1
:109F400002B0BDE8F08143F480436360D3E701A829
:109F500006F020F9019B002BDFD02362A360C5E748
:109F600000400080002800F016812DE9F041D0F873
:109F70008430A6B00546002B00F00781874AA86808
:109F800000230193516C864B41F480415164526C23
:109F900002F480420192019A5A6822F400025A6047
:109FA00059682A68014302F5805259605B6813685A
:109FB00043F001031360FFF7E5F8064606E0FFF7FC
:109FC000E1F8801BB0F5FA7F00F2D5802B6803F52D
:109FD00080531C6814F00104F1D14FF48043012632
:109FE000704A12930DA94FF400632846ADF85260F1
:109FF0008DF83860CDF8422013930F948DF85040BF
:10A000008DF8544016948DF85C401F948DF8804074
:10A0100021948DF88A40ADF88840FFF78BFE4FF40D
:10A020008072ADF824204FF480014FF4803240F26A
:10A030000113049208914FF4005202A92846ADF88A
:10A0400014308DF816608DF80C600692ADF82C3047
:10A0500007948DF826400A940C940294FFF7E2FED0
:10A06000EA68146054609460D46011682E46134608
:10A0700041F4801146F8182F02F1A00743F8281B7D
:10A080001146CB60086840F4400008601C605C60CA
:10A090009C60DC6046F8043F186840F48010194664
:10A0A00043F8280B9F42ECD1C2F88420D5E904176D
:10A0B0002E68936F06F5805E43F4400347F48047B3
:10A0C0004FF0004C9367AC62CEF810200C604C60EF
:10A0D0008C60CC60C1F800C04F604B68C1E9084497
:10A0E0002C4623F000434B6044F8481F01F128033D
:10A0F00005F1540808460022C3601A605A609A604D
:10A10000DA60C3F800C05F60586820F00040586013
:10A11000C3E9082244F8043FA045184603F1280388
:10A12000EAD1C1F88410C5E91722C5E91A22AA6547
:10A13000CEF80C1069681C4B88881864096859644B
:10A14000F36B43F40273F363D6F80C3143F400333A
:10A1500043F06003C6F80C31D6F81031102143F4F7
:10A1600003130020C6F81031C5F88820C5F8841004
:10A1700026B0BDE8F0810422E0230120C5F8882044
:10A18000C5F8843026B0BDE8F0812023C0F88430C3
:10A1900005F026FFF2E60120704700BF00380240BC
:10A1A000003801400100010100800240D0F88430F5
:10A1B000102B01D00120704770B5202204460126E3
:10A1C000042382B0C0F884208665C366FFF77CFE56
:10A1D000236830461D68FEF7DBFF226802F58053D6
:10A1E00015609A6942F400529A619A69002542F01A
:10A1F00002029A6101959A6942F480129A619B6900
:10A2000001933046FEF7C4FF2368019903F580529D
:10A21000304691611A6842F008021A601E68FEF723
:10A22000B7FF23681E601A6803F5805142F00402EC
:10A230001A60CB6943F4D0332846402243F0C1036F
:10A24000CB61C4F8842002B070BD00BFD0F8843068
:10A25000402B01D00120704730B50168202201F564
:10A26000805383B0C0F88420DA6922F4D03222F01F
:10A27000C102DA619A6922F400529A619A6922F065
:10A2800002029A610B68044623F004030B6001206C
:10A290000D68FEF77DFF236800221D6003F58053E3
:10A2A00001929A6942F480129A619B69019301209C
:10A2B000FEF76EFF2368019903F58052012091613A
:10A2C0001A6822F008021A601D68FEF761FF224634
:10A2D00004F1540052F8443B1D6052F8041F4B68CF
:10A2E000824243F000434B60F7D100201023A06569
:10A2F000C4F8843003B030BD10B5044631B3D0F893
:10A300008420402A01D0012010BD4B6BC363012281
:10A31000FFF754FC98B9BFF34F8FA36A5A1C032A66
:10A3200088BFDA1E2368A26203F580535A69520778
:10A3300003D50421002259615A60002010BDD4F8D1
:10A34000883043F00203C4F88830DCE7D0F8883066
:10A3500043F00103C0F88830D5E700BF2DE9F04F86
:10A36000054685B0002975D0D0F88430402B5BD1EC
:10A37000C76DC36E07F11202C3F1040A50F8224000
:10A380002268002A74DBBAF1000F73D000F1800359
:10A390004FF00008019300F17C030293C146039142
:10A3A00003E0C24539D0002E48D12368D90503D532
:10A3B000E369AB67A3696B6723689A0501D4EE6F05
:10A3C000EEB123689B0548BFC5E918992368266844
:10A3D00016F48076C3F30D4B02D022682A6701265B
:10A3E000A2682262DDE901105B4605F0F7FE2A6EE5
:10A3F00001322A666A6E5A446A66C4F820907B1C51
:10A40000032B8CBF033F1F4607F1120308F101081D
:10A4100055F823402368002BC3DAEB6E03994344BD
:10A42000EB662BB9EF657EB9012005B0BDE8F08F72
:10A4300028460191FFF748FD0199F3E7EB6E039978
:10A440004344EB666BB9EF65EA6F0A600023184678
:10A45000EB67EAE7D0F8883043F00103C0F88830B2
:10A46000E2E728460191FFF72FFD0199EF65EBE741
:10A47000002BD9D02846FFF727FDEF65D4E700BFB2
:10A480002DE9F041D0E9105475B106464FF00008AF
:10A4900006EB8407A300F86A2344013D38B1F26853
:10A4A00052F83330002B0BDA0020BDE8F081631C3A
:10A4B000032B13D9033C002DEAD10020BDE8F08125
:10A4C00005F0A8FE631C032B8CBF033C1C46C7F899
:10A4D0002C80C6E91054002DDAD1EEE71C46002D81
:10A4E000D6D1EAE7704700BF704700BF026802F5A7
:10A4F00080532DE9F041D2F838805D69304ADE6939
:10A5000057696906044601D5720647D4E90701D5A3
:10A51000F20739D42B0401D5300406D418F0080F03
:10A520001BD13B0327D4BDE8F081D4F8883043F039
:10A530000803C4F88830236803F58053A9045A69D6
:10A5400031D448F280610A40C4F88C205961204619
:10A5500005F036FC18F0080FE3D02368DB6A03F03F
:10A560006003C4F894302046FFF7BCFF0023C4F812
:10A5700094303B03D7D5124B4FF400225A6120464A
:10A58000FFF7B2FFBDE8F081236803F580534FF079
:10A5900001125A61204605F00DFCBBE7094A5A61D9
:10A5A00005F002FCB2E708490A40C4F88C20DA69D9
:10A5B00022F4C032DA61E023C4F88430C7E700BF78
:10A5C000003C01404000010000207E0070B50446C0
:10A5D00000681D460369920103F01C0302F4F8624F
:10A5E000C9021A4389B2114341F001010161FEF72A
:10A5F000C9FD064604E021680A6912F0010207D08D
:10A60000FEF7C0FD801BB0F5803FF4D3012070BD84
:10A610004B699BB210462B6070BD00BF38B5044635
:10A6200000689DB203694561920103F01C0302F4C6
:10A63000F862C9021A4389B2114341F00301016172
:10A64000FEF7A0FD054604E023681B6913F0010333
:10A6500007D0FEF797FD401BB0F5803FF4D30120F3
:10A6600038BD184638BD00BF002964D003681A6899
:10A67000C2F3001210B481F828201C681A6882F412
:10A680000072C2F3402281F820201A68C2F300420F
:10A69000CA771A6882F40052C2F340328A771A6885
:10A6A000C2F300320A7704F060044C621C681A6836
:10A6B00004F4006402F48042C1E905241A6882F4BB
:10A6C0008002C2F380524A741A6882F40002C2F314
:10A6D000C0520A741A68C2F3C012CA731C681A689E
:10A6E000C2F380220A711A68C2F340628A739A69BF
:10A6F00004F46024C2F340028C6081F854209A690B
:10A7000082F08002C2F3C01281F84C209C699A69E1
:10A71000120C8A649A69C2F3800281F856209B6900
:10A7200004F03004C3F3C00300200C6581F85530F9
:10A730005DF8044B70470120704700BF31B108B588
:10A74000D0F88430102B03D0012008BD01207047C1
:10A75000FFF7F0FA002008BD38B5036805461C690C
:10A7600001F0A6FF0F4B984224F01C0404D844F0DB
:10A7700008042B681C6138BD0B4B984204D22B682F
:10A7800044F00C041C6138BD084B9842F1D9084BC9
:10A7900098422B6894BF44F0040444F010041C61F8
:10A7A00038BD00BFBF0E160200879303FFE0F5051A
:10A7B0007FD1F008D0F88800704700BFD0F88C0037
:10A7C000704700BF2DE9F04F00230C68DFF814A29A
:10A7D00085B04FF0010B894603E00133102B00F0E8
:10A7E00092800BFA03F202EA0408A243F5D1D9F8E9
:10A7F000041001F0030C5A0003250CF1FF369540BC
:10A80000012E6FEA050540F28180BCF1030F40F094
:10A81000D98006680CFA02F235402A4311F4403F11
:10A820000260DAD000220392DAF8442042F4804237
:10A83000CAF84420DAF8442002F480420392039AD2
:10A8400023F0030202F1804203F003060F2702F512
:10A850009C32B60007FA06FC5F4F9568B84225EABD
:10A860000C0527D007F58067B84200F087805B4F62
:10A87000B84200F08980DFF870C1604500F08A803E
:10A88000DFF868C1604500F08B80DFF864C1604587
:10A8900000F08C80DFF85CC1604500F08D80DFF84F
:10A8A00058C160450CBF4FF0070C4FF0080C0CFA74
:10A8B00006F6354395604A4A9268CE026FEA08056B
:10A8C000474E54BF2A4048EA0202B260F268444E42
:10A8D0008F0254BF2A4048EA0202F26072688E0377
:10A8E0003F4E54BF2A4048EA020272603268C903F0
:10A8F00003F101033A4954BF2A4048EA0202102BEF
:10A900000A607FF46EAF05B0BDE8F08F866806EA96
:10A91000050ED9F80C60964046EA0E068660466839
:10A9200026EA080EC1F300169E4046EA0E0646606F
:10A93000C66806EA050ED9F80860964046EA0E0693
:10A94000BCF1020FC6607FF464AFDE0800EB860640
:10A950000196376AD9F81060009703F0070E4FEAA6
:10A960008E0E0F2706FA0EF607FA0EFE009F27EA54
:10A970000E0E019F46EA0E063E624AE74FF0010CBA
:10A980000CFA06F6354395E74FF0020C0CFA06F682
:10A9900035438FE74FF0030C0CFA06F6354389E791
:10A9A0004FF0040C0CFA06F6354383E74FF0050C24
:10A9B0000CFA06F635437DE74FF0060C0CFA06F666
:10A9C000354377E7C66806EA050ED9F80860964071
:10A9D00046EA0E06C6601CE700000240000802407E
:10A9E000003C014000380240000C024000100240D0
:10A9F0000014024000180240001C02402DE9F04FF4
:10AA00000023534F83B001264FF00F094FF0030A84
:10AA100002E00133102B76D006FA03F232EA010489
:10AA200002EA010CF5D123F0030505F1804503F09E
:10AA30000304A40005F59C3509FA04F80194454C7B
:10AA4000D5F808E0A04208EA0E0E20D004F5806494
:10AA5000A0425BD0404CA0425CD0404CA0425FD0B2
:10AA60003F4CA04262D0DFF8FCB0584564D0DFF81C
:10AA7000F8B0584566D0DFF8F4B0019C58450CBFDB
:10AA80004FF0070B4FF0080B0BFA04F400E0002422
:10AA9000A64513D13C6824EA0C043C607C6824EA97
:10AAA0000C047C60FC6824EA0C04FC60BC6824EAAA
:10AAB0000C04BC60AC6824EA0804AC6004685D0067
:10AAC0000AFA05F54FEAD30C24EA050400EB8C0CD6
:10AAD000046003F00704DCF820E0A40009FA04F4A1
:10AAE0002EEA0404CCF82040C46824EA0504C460BB
:10AAF000446824EA020242608268013322EA0502C5
:10AB0000102B826088D103B0BDE8F08F019C06FA5B
:10AB100004F4BDE7019C4FF0020B0BFA04F4B7E715
:10AB2000019C4FF0030B0BFA04F4B1E7019C4FF0CA
:10AB3000040B0BFA04F4ABE7019C4FF0050B0BFA86
:10AB400004F4A5E7019C4FF0060B0BFA04F49FE711
:10AB5000003C01400000024000080240000C02409E
:10AB6000001002400014024000180240001C024085
:10AB70000369194214BF01200020704702B909047B
:10AB800081617047436901EA030221EA030141EA56
:10AB900002418161704700BF044A5169014200D1FE
:10ABA000704708B55061FCF74DF808BD003C014006
:10ABB0002DE9F8430D46804616461F464FEA1149D7
:10ABC000B9F1010FD8F8003002D111E07A1C19D187
:10ABD0009C6925EA040C1FFA8CFCBCFA8CFC4FEA39
:10ABE0005C1C6645F2D00020BDE8F883791C09D1D1
:10ABF0005C6925EA0404A4B2B4FA84F46409A642A8
:10AC0000F4D0F0E7FEF7BEFA089BC01AB84220D98C
:10AC1000D8F80030B9F1010F0CBF5B699B6925EAD8
:10AC200003039BB2B3FA83F35B09B342C8D100229A
:10AC30002023C8F8302088F83D3088F83E20D8F826
:10AC4000403088F83C2043F02003C8F84030012011
:10AC5000CAE7002FB4D1DBE72DE9F843046880464A
:10AC60000E461746994604E065696A0509D47B1CBF
:10AC700021D1606926EA000080B20028F4D1BDE845
:10AC8000F883236843F400732360002220236FF4C9
:10AC900080616161C8F8302088F83D3088F83E2036
:10ACA000D8F8403043F00403C8F84030002388F857
:10ACB0003C300120E3E7FEF765FAA0EB0900B8425B
:10ACC000D8F8004001D8002FD3D1636926EA0303E6
:10ACD0009BB2002BCDD000232022C8F8303088F85A
:10ACE0003D2088F83E30D8F840301343C8F8403053
:10ACF000DCE700BFF8B5036806465869400624D46F
:10AD00000D4617460DE0FEF73DFAC01BA84233681A
:10AD100000D81DB95C6914F0400418D05A69520675
:10AD200013D45A69D106EED500226FF0100020210D
:10AD30005861326386F83D1086F83E20336C3364E8
:10AD4000002386F83C300120F8BD0020F8BD202308
:10AD5000346386F83D3086F83E40336C43F0200380
:10AD60003364EDE7F8B5046805460E46174601E082
:10AD7000731C1AD1636913F0800314D16069420512
:10AD8000F6D56FF48061202261612B6385F83D2048
:10AD900085F83E302B6C43F004032B64002385F8C8
:10ADA0003C300120F8BD0020F8BDFEF7EBF9C01BD8
:10ADB000B0422C6801D8002EDCD1636913F0800307
:10ADC000D8D120222B6385F83D2085F83E302B6CAE
:10ADD00013432B64E2E700BFF8B5046805460E464E
:10ADE000174601E0731C1AD1636913F0040314D1F0
:10ADF00060694205F6D56FF48061202261612B63A2
:10AE000085F83D2085F83E302B6C43F004032B641D
:10AE1000002385F83C300120F8BD0020F8BDFEF786
:10AE2000B1F9C01BB0422C6801D8002EDCD1636997
:10AE300013F00403D8D120222B6385F83D2085F838
:10AE40003E302B6C13432B64E2E700BF2DE9F04F3B
:10AE5000056883B09B462B68DDF83080DDF834A0B0
:10AE600043F4807306460F4691462B606B69DB07FF
:10AE700005D4B8F1FF3F0ED16C69E007FCD507F0AF
:10AE8000FE0732492F61534642463046FFF7E4FE43
:10AE900000B301241AE0FEF775F9A0EB0A00804523
:10AEA000356830D26B69D907E0D4002220233263A1
:10AEB00086F83D3086F83E20336C86F83C2043F01F
:10AEC000200333642B68DA0524D40324204603B01E
:10AED000BDE8F08F33680190596901919B69019336
:10AEE000524641463046019BFFF73CFF044618BBE3
:10AEF000BBF1010F336811D15FFA89F220461A6164
:10AF000003B0BDE8F08FB8F1000FAFD16B69D9077E
:10AF1000ACD4CAE74FF400733364D6E74FEA192084
:10AF20001861524641463046FFF71CFF20B932688F
:10AF30005FFA89F31361C9E7336C042BA9D1326836
:10AF4000136843F400731360A3E700BF020001001D
:10AF50002DE9F04F05689B462B6843F4806385B06C
:10AF60002B602B68DDF83880DDF83CA043F480735B
:10AF700006460F4691462B606B69DA0705D4B8F197
:10AF8000FF3F4AD16C69E407FCD507F0FE032B6153
:10AF90004349534642463046FFB2FFF75DFE002864
:10AFA00069D133680390596903919B6903935246B1
:10AFB00041463046039BFFF7D5FE002853D1BBF135
:10AFC000010F336859D15FFA89F21A61524641463E
:10AFD0003046FFF7C7FE002845D1024630680168B9
:10AFE00041F4807101604346CDF800A04FF001119B
:10AFF0003046FFF7DDFD336800284DD147F00107EB
:10B000001F612749534642463046FFF725FE003868
:10B0100018BF012005B0BDE8F08FFEF7B3F8A0EB34
:10B020000A008045356817D26B69D807A4D400227E
:10B030002023326386F83D3086F83E20336C86F854
:10B040003C2043F0200333642B68D90502D54FF42C
:10B05000007333640320DDE7B8F1000F8CD16B6916
:10B06000D80789D4E3E7336C042B04D13268136822
:10B0700043F4007313600120CCE74FEA19221A61F0
:10B08000414652463046FFF76DFE0028EBD132684C
:10B090005FFA89F3136199E71B68DB05DAD5D6E718
:10B0A00002000100002800F0B88070B590F83D3033
:10B0B000044603F0FF02002B00F09880236824224E
:10B0C00084F83D201A6822F001021A601A6842F4DE
:10B0D00000421A601A6822F400421A6001F0EEFA87
:10B0E0004F4B65689D424FD84E4B98427CD94E4B92
:10B0F0006A00A3FB0035431EB3FBF2F322685168DC
:10B1000021F03F0141EA95415160116A4FEA954CA7
:10B110000CF1010C21F03F0141EA0C011162D169EF
:10B1200040F6FC70013321F44F41034221F0FF014E
:10B1300061D104230B43D361D4E907301168034381
:10B1400021F0C0010B4313609168D4E9030321F49B
:10B150000341034321F0FF010B439360D4E9053021
:10B16000D168034321F0FF010B43D3601168002332
:10B1700041F0010120201160236484F83D00236325
:10B1800084F83E30184670BD284B98422CD922686E
:10B19000254B274EA3FB003C431E506820F03F0088
:10B1A00040EA9C4050604FEA9C414FF4967000FB8F
:10B1B00001F1A6FB0161106A890920F03F0001310D
:10B1C00001431162D169A06821F44F4121F0FF01D0
:10B1D000A0B905EB4505B3FBF5F30133C3F30B034E
:10B1E000CBB143F40043A5E7012070BD80F83C20BB
:10B1F000FBF77EFD62E7C3F30B039BE705EB8505D9
:10B2000005EB8505B3FBF5F30133C3F30B0313B172
:10B2100043F440438EE701238CE70120704700BFD1
:10B22000A08601007F841E0083DE1B43FF083D00D3
:10B23000D34D62102DE9F047044682B09946BDF81F
:10B240002CA00C9E0F469046FDF79CFF94F83D30D5
:10B25000202B03D0022002B0BDE8F0870546009005
:10B260004049192301222046FFF7A2FC0028F1D112
:10B2700094F83C30012BEDD00123206884F83C3059
:10B280000368DA075ED53946076827F40067076068
:10B290000A9860622120CDE9006584F83D004020D5
:10B2A00084F83E0000202064A4F82AA0608D208548
:10B2B0002D48E0624B4642462046FFF7C7FD002876
:10B2C0004DD1238D002B2AD02A4631462046FFF748
:10B2D00049FD00283BD1676A2068B4F828C03A4687
:10B2E0000CF1FF3112F8013B0361638D013B9BB20E
:10B2F00063854369626289B25B0721850DD571B1AF
:10B300007A780261628DACF1020C013A1FFA8CF17D
:10B31000023792B26762218562850029D4D12A461C
:10B3200031462046FFF758FD88B92268136820216E
:10B3300043F40073136084F83D1084F83C0084F8F3
:10B340003E0088E7036843F0010303609BE7236C3A
:10B35000042B04D12268136843F4007313600120A6
:10B3600079E700BF020010000000FFFF2DE9F04761
:10B37000044686B09946BDF83CA0109E0F46904604
:10B38000FDF700FF94F83D30202B05D04FF0020868
:10B39000404606B0BDE8F087054600909349192362
:10B3A00001222046FFF704FC0028EFD194F83C303E
:10B3B000012BEBD00123206884F83C300368D907C7
:10B3C00039D53946076827F4006707600E98606230
:10B3D0002220CDE9006584F83D00402084F83E003D
:10B3E00000202064A4F82AA0608D20858048E062B7
:10B3F00042464B462046FFF7ABFD8046A8B9238D59
:10B400002268EBB902905369029393690293029BFD
:10B41000136843F4007313600023202284F83D2056
:10B4200084F83C3084F83E30B2E74FF001084046E3
:10B4300006B0BDE8F087036843F001030360C0E78E
:10B44000012B00F0C480022B00F08A800590516926
:10B45000059192690592059A664F032B4ED8012BF0
:10B4600000F0A880022B009533464FF000023946C9
:10B47000204600F08480FFF79BFB02460028D4D1D1
:10B480002368196821F4806119601969636A197069
:10B49000616A638D01316162013B218D9BB26385DD
:10B4A0004B1E23853946009533462046FFF780FB27
:10B4B0000028BAD12368616A1A6842F400721A60DF
:10B4C0001B690B70638D626A2168013B9BB26385C7
:10B4D000531C09696362238D013B23855170238DC1
:10B4E000628D616A013B013A01319BB292B26162A5
:10B4F00023856285002B8FD0032BB0D92A46314695
:10B500002046FFF7F7FB00288FD12268636A126993
:10B510001A70628D2168238D606A013A92B2628549
:10B520004A69013B9BB200F1010C52072385C4F824
:10B5300024C0DFD5032B03D10B6823F480630B6099
:10B540000B694370628D238D013A92B26285626A03
:10B55000013B9BB2013223856262002BCCD15BE7B9
:10B56000116821F480611160116841F4006111607B
:10B5700004905169049192690492049A6CE7FFF770
:10B5800017FB00287FF451AF2368616A1A6842F400
:10B5900000721A601B690B70638D626A013B9BB27B
:10B5A0006385238D013B23852368511C1B696162E0
:10B5B0005370C7E72A4631462046FFF79BFB002819
:10B5C0007FF433AF23681A69636A1A70BAE71168A7
:10B5D00021F4806111600390516903919169039195
:10B5E0000399116841F40071116035E70200100001
:10B5F0000000FFFF0400010070B582B000B390F8B6
:10B6000095340568044603F0FF02002B5AD0284603
:10B610000323B5F1A04F84F8953404BF0023A37130
:10B6200003F044FC237C8DF80030251D95E80E00C6
:10B63000206803F071FB014630B1022384F8953491
:10B640000125284602B070BD206803F037FC014692
:10B650000028F2D1267906B3234622464FF0010C8A
:10B660001175D1850131B142C2E9070082F815C0D8
:10B67000107642F8240FF3D100210A4683F85412C1
:10B680000131B142C3E9972283F8552283F8582249
:10B69000C3F8642203F12403F0D1207C95E80E0066
:10B6A0008DF80000206803F08FFC05460028C4D107
:10B6B00001236074206884F8953404F021F828464A
:10B6C00002B070BD80F8942414F010F820689FE751
:10B6D00010B590F89434012B0446006817D001236C
:10B6E00084F89434C3685B0602D5637B012B09D0D0
:10B6F00003F0D4FB206803F0F3FF002384F89434B4
:10B70000184610BD836B43F480338363F0E7022057
:10B7100010BD00BF2DE9F04F066889B004463046E1
:10B7200004F02CF810B109B0BDE8F08F0546206890
:10B7300003F0F6FF0028F6D0D6F808382068C3F3E7
:10B740000D23C4F8D43406F50063039303F0E8FF37
:10B7500010F0020F20681EBF436903F0020343612B
:10B7600003F0DEFF10F0100F206814D0836923F07F
:10B7700010038361376A07F4F013B3F5802F07F0E5
:10B780000F0800F0BB82B3F5402F00F0628283699E
:10B7900043F01003836103F0C3FF10F4002F20680F
:10B7A00040F0F68103F0BCFF470300F151812068AF
:10B7B00003F0B6FF0028C0F2C280206803F0B0FF9B
:10B7C00002057ED4206803F0ABFFC70400F1E180DE
:10B7D000206803F0A5FF10F4005F206840F0C280ED
:10B7E00003F09EFF000700F12A81206803F098FF14
:10B7F00001061DD5B36923F08003B3612379012BC2
:10B8000016D92746012504E00135AB4207F124078C
:10B810000ED997F87B22012AF6D105EBC50104EB7E
:10B820008101206801F5157103F06CFE2379EBE7C7
:10B83000206803F075FFC20241D52379012B20D97E
:10B8400006F512682746012506E00135AB4208F1EE
:10B85000200807F1240714D997F83C20D8F80010E5
:10B86000012AF2D10029F0DA242305F00F0103FBAD
:10B870000141206887F83B20143103F043FE23790F
:10B88000E3E72068436903F48013436103F048FF52
:10B89000830221D4206803F043FF400000F1C680FA
:10B8A000206803F03DFF41077FF53DAF23685D68E9
:10B8B0006A0700F144825A682A435A6033E72068D5
:10B8C000E4E7039B9B68DB0700F13582206843694E
:10B8D00003F40063436176E794F804C0BCF1010F00
:10B8E00027D906F532622346012103E0614503F1C1
:10B8F00024031ED093F87C021568012801F1010190
:10B9000002F12002F2D1002DF0DAD4F8D47487EAE3
:10B910001547FF07EAD483F87B02B06940F0800046
:10B92000B06170690506E1D4039A536843F400736B
:10B9300053602068436903F400134361ABE7039A43
:10B94000536823F00103536094F8CC34012B00F0CA
:10B950007981204613F056FF2068436903F00043C5
:10B9600043612BE703F00EFF206803F007FCE07152
:10B97000256800F09DFEE2790146284603F014FA9E
:10B98000204613F011FF2068436903F4005343611C
:10B9900026E7039A2068536823F0010353601021BF
:10B9A00003F0C4FA2079D8B106F510634FF67F3161
:10B9B00099601A6822F400121A60C3F80812D3F8CA
:10B9C000002222F40012C3F80022D3F8002201352D
:10B9D00042F000628542C3F8002203F12003E7D160
:10B9E000039AD36943F00113D361E37B002B40F04A
:10B9F0001D81039A536943F4005343F02B035361B1
:10BA0000136943F00B031361D6F80038206823F460
:10BA1000FE63C6F80038A17904F29C4203F0C2FE2E
:10BA20002068436903F480534361D2E6204613F053
:10BA3000F5FE2068436903F08043436131E7204607
:10BA400013F0AEFE2068436903F008034361CDE6BE
:10BA5000206803F071FE81462068B9F1000F3FF4C1
:10BA6000A7AECDE9046506F51067A0464FF0000AC1
:10BA7000064609E05FEA59090AF1010A08F12408BB
:10BA800007F1200700F0F88019F0010FF2D05FFAFB
:10BA90008AFB5946304603F061FEC107054612D5C0
:10BAA00003980121436B0AF00F0201FA02F223EA24
:10BAB00002034363B960A179012900F04581594629
:10BAC000204613F063FE2A0744BF0823BB60EB0641
:10BAD00044BF1023BB606E0644BF4023BB60A80771
:10BAE00000F1018129062668C4D5D8E90953AB4283
:10BAF000C0D806F51061D8F81C00079601EB4A1172
:10BB0000A5EB030C84458A6928BF84461FFA82FE90
:10BB10000CF1030CBEEB9C0FC0F04D81CDF818A0CA
:10BB20008A4621E0D8F81C30D8F820109D4228BF62
:10BB30001D46A37900935A46ABB2304603F02CFD64
:10BB4000D8F82030DAF818202B44C8F82030D8F87C
:10BB5000283092B22B440335B2EB950FC8F8283049
:10BB6000C0F02481D8F824509D42A5EB0305D9D814
:10BB7000DDF818A02668079B0AF00F0503F50061A1
:10BB80000122D3F83438AA4023EA02034B6371E759
:10BB900003F0CAFD07462068002F3FF403AE04956A
:10BBA00006F53068A3464FF0000A254607E07F08F7
:10BBB0000AF1010A08F120080BF1240B60D0FC0700
:10BBC000F5D55FFA8AF4214603F0BEFD10F0010FAF
:10BBD000814669D119F0080F55D119F0100F1CBF1B
:10BBE0001022C8F8082019F0020F0FD07269100651
:10BBF00004D5039B5A6842F480625A609BF857222E
:10BC0000012A00F0DC800223C8F8083019F0200F68
:10BC10001CBF2023C8F8083019F4005F18BF4FF488
:10BC20000053286818BFC8F80830C0E7039AD2F854
:10BC3000843043F00B03C2F88430536C43F00B03A1
:10BC40005364E1E6002184F8CC14204600F07AFA2F
:10BC500082E6082204F29C41304608EBC80803F053
:10BC6000B1FC04EB8802C7F30A13D2F8681220680B
:10BC70000B44C2F868328AE53046059D049E97E57C
:10BC80002C46049D8EE529680822C8F80820086C17
:10BC900001F530626B4902EB4A128842936866D81C
:10BCA000284613F063FD98E728680122C8F80820A9
:10BCB000A979D0F840E000F5306202EB4A12012980
:10BCC000936866D060498E4500F08180BAF1000F1C
:10BCD00004D1D5F86422002A00F0A7802146284626
:10BCE00013F04AFD76E70498514603F01FF998F8DF
:10BCF0001730012B72D00223BB60F3E647F6F073D6
:10BD00001F423FF444AD08EBC80804EB8808C7F3B2
:10BD10000A12D8F860123046174603F053FCD8F8E0
:10BD2000603220683B44C8F86032D8F868323B443F
:10BD3000C8F868322BE5204613F04CFDC6E52046D6
:10BD400013F070FD2368B6E5D8E907231344C8F85B
:10BD50002030BAF1000F7FF4B2AE636A002B7FF49B
:10BD6000AEAE206804F29C4203F01CFDA7E61B0463
:10BD700044BF4FF400419160284613F0F7FCA979C5
:10BD800001297FF42AAF286805F29C4203F00AFDDE
:10BD900023E719072AD52B498E457FF61BAF1804D8
:10BDA0007FF518AF4FF40041916013E7DDF818A05C
:10BDB000D8F824502668AB42FFF45CAEDBE60022E4
:10BDC00021468BF85722284613F020FD1BE7180464
:10BDD000E8D4990682D5202191607FE7002388F876
:10BDE00017305946204613F015FD84E7990602D511
:10BDF00020219160EEE613498E4501D91B04D1D470
:10BE00001169DBF87422C1F31201521ACBF86822CF
:10BE1000BAF1000F7FF462AFD5F8641259B1D5F8CA
:10BE200060121144C5F8601258E705F29C42514671
:10BE300003F0B8FC52E705F29C42012103F0B2FC8A
:10BE40004CE700BF0A30544F0A31544F90F8942405
:10BE5000012A0DD010B504460122006884F894240C
:10BE6000617403F02DFC002384F89434184610BD4F
:10BE70000220704710B501F00F0E0EEBCE0C090634
:10BE800004464FEA8C0C27D40CF5157101440EEBD7
:10BE9000CE0004EB80004FF0000C80F855C2C2F3D6
:10BEA0000A028A604A7881F800E00B710AB1A1F8B1
:10BEB0001AE0022B04BF00234B7194F89434012B39
:10BEC00016D0012384F89434206803F063F900232A
:10BED00084F89434184610BD0CF1140101440EEBA3
:10BEE000CE0004EB80004FF0010C80F815C0D6E7BF
:10BEF000022010BD01F00F0301F00F0210B503EB9B
:10BF0000C3030446090602EBC2004FEA830304EBB5
:10BF1000800016D403F51573E1184FF0000C80F87B
:10BF200055C20A7094F89434012B15D0012384F87B
:10BF30009434206803F076F9002384F8943418468A
:10BF400010BD1433E1184FF0010C80F815C00A70D1
:10BF500094F89434012BE9D1022010BD10B501F002
:10BF60000F0E0EEBCE0C00EB8C0C1446CCF86432AA
:10BF700000238CF854E2CCF86022CCF868328CF8BC
:10BF800055328279242101FB0E01012A01F5157138
:10BF900008BFCCF87042006803F0A6F9002010BD7D
:10BFA00001F00F0101EBC10100EB8100D0F8680244
:10BFB000704700BF10B501F00F0E0EEBCE0C00EB7A
:10BFC0008C0C1446CCF824300023CCF82830012304
:10BFD0008CF814E0CCF820208CF8153082792421DC
:10BFE00001FB0E019A4201F1140108BFCCF8304068
:10BFF000006803F079F9002010BD00BF38B503795F
:10C0000001F00F05AB4232D30B0604461CD401EB02
:10C01000C103242202FB010100EB830301F515712A
:10C02000002283F8552201238B700D7094F894241C
:10C030009A421AD0206884F8943403F0E7FAC5B124
:10C04000002084F8940438BD05EBC503242101FBCE
:10C05000050100EB8303012214315A7501238B7013
:10C060000D7094F894249A42E4D1022038BD012046
:10C0700038BDA179206804F29C4203F093FBDFE70E
:10C0800038B5037901F00F0293422ED3044602EB38
:10C09000C20302EBC20009064FEA830304EB8000EF
:10C0A00016D403F51573E118002580F855520025C4
:10C0B0008D700A7094F89434012B14D001232068F9
:10C0C00084F8943403F0D0FA84F89454284638BDA8
:10C0D0001433E1180125457500258D700A7094F818
:10C0E0009434012BEAD1022038BD012038BD00BFB5
:10C0F00010B404681204636A29B91A43A2620020CA
:10C100005DF8044B7047A06A013903EB104C0AD06C
:10C11000002303F1400004EB8000013340689942A2
:10C120000CEB104CF5D1403104EB810442EA0C02D7
:10C13000626000205DF8044B704700BF0368002078
:10C1400059627047704700BF002800F0D8812DE980
:10C15000F0410368DD0782B004462FD59D498A6807
:10C1600002F00C02042A00F0EC808A6802F00C0253
:10C17000082A00F0E2806368B3F5803F00F0EB80AE
:10C18000B3F5A02F00F07381924D2A6822F480321B
:10C190002A602A6822F480222A60002B40F0E08086
:10C1A000FCF7F0FF064605E0FCF7ECFF801B642877
:10C1B00000F200812B689F03F6D423689D0728D5E1
:10C1C000844A916811F00C0F00F09B80916801F097
:10C1D0000C01082900F09180E368002B00F00C812D
:10C1E0007D4B7C4E01221A60FCF7CCFF054605E032
:10C1F000FCF7C8FF401B022800F2DC8033689F0771
:10C20000F6D53368226923F0F80343EAC2033360AA
:10C2100023681A075CD45D073AD56E4A136C13F095
:10C22000805340F088800193136C43F08053136473
:10C23000136C03F080530193019B0125674E336813
:10C24000D80540F1A780A368012B00F0B780052B2B
:10C2500000F01D815F4E326F22F001023267326FB3
:10C2600022F004023267002B40F0AD80FCF78AFF19
:10C2700041F28838074605E0FCF784FFC01B4045C3
:10C2800000F29880336F9B07F6D4002D40F0F980C0
:10C29000A369CBB14F4DAA6802F00C02082A00F046
:10C2A000BC80022B4C4B4FF000021A6600F0F98064
:10C2B000FCF768FF044604E0FCF764FF001B02285B
:10C2C00078D82B689B01F7D4002002B0BDE8F0813C
:10C2D0006369FBB1404B3F4E0122C3F8802EFCF74F
:10C2E00051FF054604E0FCF74DFF401B022861D8D2
:10C2F000736F9B07F7D523688DE7526851023FF5AE
:10C300006BAF344A1268920738D5E268012A35D0FB
:10C310000120DAE7304A2F4EC2F8803EFCF732FFA8
:10C32000054604E0FCF72EFF401B022842D8736F3D
:10C330009F07F7D4DFE7002580E74A6851027FF5C1
:10C340001AAF244A126892037FF538AF6268002A58
:10C350007FF434AFDCE71F4A136843F48033136083
:10C36000FCF710FF1B4E054604E0FCF70BFF401BDB
:10C3700064281FD833689B03F7D51EE71549206949
:10C380000A6822F0F80242EAC0020A601A077FF542
:10C3900042AF9DE7336843F480733360FCF7F2FEED
:10C3A00007463368D9053FF54EAFFCF7EBFEC01BDF
:10C3B0000228F6D9032002B0BDE8F081054A136FC8
:10C3C00043F001031367FCF7DDFE024F064641F21E
:10C3D00088380AE000380240000047420070004000
:10C3E000FCF7D0FE801B4045E4D83B6F9A07F7D599
:10C3F000002D3FF44DAF44E0424A434E1360FCF73A
:10C40000C1FE054604E0FCF7BDFE401B0228D1D862
:10C4100033689907F7D42368FBE6012B3FF478AF24
:10C420006B68E26903F4800191427FF471AF226A84
:10C4300003F03F0191427FF46BAF616A47F6C0722F
:10C440001A40B2EB811F7FF463AFA26A520803F473
:10C450004031013AB1EB024F7FF45AAFE26A03F088
:10C460007063B3EB026F14BF012000202DE7264B51
:10C470001A6842F480221A601A6842F480321A6004
:10C480006EE7214A136C23F08053136400E71E4BC0
:10C490001A6F42F004021A671A6F42F001021A671B
:10C4A00091E7FCF76FFE064605E0FCF76BFE801B8C
:10C4B00002283FF67FAF2B689901F6D4D4E9073103
:10C4C000626A0B4343EA8213D4E90A2052080D49F9
:10C4D00043EA0063013A43EA024301226B600A66C1
:10C4E000FCF750FE084D044605E0FCF74BFE001B30
:10C4F00002283FF65FAF2B689A01F6D5E4E60120EB
:10C50000704700BF0000474200380240164908B596
:10C510008B6803F00C03042B1BD0082B01D01348AD
:10C5200008BD4A684B68496813F4800302F03F0273
:10C5300011D10E48C1F38811A1FB0001F4F784FC6E
:10C54000094B5B68C3F3014301335B00B0FBF3F0BD
:10C5500008BD074808BD0648C1F388110023A1FBA8
:10C560000001F4F771FCEBE7003802400024F4000E
:10C5700000127A00002800F08780484A136803F010
:10C5800007038B422DE9F0410D46044609D2CBB298
:10C590001370136803F007038B4202D00120BDE83B
:10C5A000F0812368980714D5590704D53C498A6857
:10C5B00042F4E0528A601A0704D539498A6842F485
:10C5C00060428A603649A0688A6822F0F00202431D
:10C5D0008A60DF0721D56268012A57D0931E012B9C
:10C5E0002F4B1B684DD99907D8D52D4EB36823F032
:10C5F00003031343B360FCF7C5FD41F288380746D7
:10C6000004E0FCF7BFFDC01B404544D8B368626836
:10C6100003F00C03B3EB820FF3D1204A136803F04D
:10C620000703AB4206D9EBB21370136803F007039C
:10C63000AB42B3D123685A0706D51949E0688A6826
:10C6400022F4E05202438A601B0707D5144A21698D
:10C65000936823F4604343EAC1039360FFF756FFF6
:10C660000F4A104C92681049C2F303120346A25CB1
:10C670000E48D34000680B60FBF7FCFD0020BDE8CE
:10C68000F0819801B1D489E701207047044B1B6801
:10C690009E03AAD482E7032081E700BF003C02404A
:10C6A00000380240846802086C0300207C030020EC
:10C6B000014B1868704700BF6C030020044B05490C
:10C6C0009B68054A0868C3F38223D35CD84070474F
:10C6D000003802406C0300207C680208044B0549C6
:10C6E0009B68054A0868C3F34233D35CD84070475F
:10C6F000003802406C0300207C6802080E4B0F22B9
:10C7000010B402609A680D4C02F0030242609A680D
:10C7100002F0F00282609A6802F4E052C2609B6804
:10C72000DB0803F4E053036123685DF8044B03F076
:10C7300007030B60704700BF00380240003C024016
:10C74000F0B5036813F0050F83B0044604D19807D1
:10C750003BD4002003B0F0BD454B464E00229A6604
:10C76000FCF710FD054604E0FCF70CFD431B022B13
:10C7700028D833681B01F7D4D4E901131B0743EA17
:10C7800081133B4AC6F8843001239366FCF7FAFC18
:10C79000384E054604E0FCF7F5FC431B022B11D88C
:10C7A00033681F01F7D52368D1E7FCF7EBFC41F2B2
:10C7B000883706462B6F9B073CD4FCF7E3FC801BB5
:10C7C000B842F7D9032003B0F0BD2A4B2A4D00220E
:10C7D00001921A6C42F080521A641B6C03F0805371
:10C7E0000193019B2B6843F480732B60FCF7CAFC18
:10C7F000064604E0FCF7C6FC831B022BE2D82B683C
:10C80000D905F7D51B4DE3682A6F12F4407203F483
:10C81000407112D08A4210D02B6F154A0121C2F804
:10C82000401E23F440730021C2F8401E2B672B6F7B
:10C83000DA07BAD4E36803F44071B1F5407F0BD056
:10C840000C498A6822F4F8128A600A4A116FC3F30D
:10C850000B030B4313677CE70648826823F07041A3
:10C8600021F4407122F4F8120A438260EDE700BF20
:10C87000000047420038024000700040036830B5B5
:10C880009C6A18691B68C0F30E00C1E90140C3F33C
:10C8900005440020C3F3062E64F3070003F07F0C69
:10C8A0006EF30F20C3F306456CF31740C3F38053B8
:10C8B00063F31F600860DAB94FEA1E1303EB8303CA
:10C8C0000EF00F0E0EEB430E24094FEA1C1304EB7F
:10C8D000840405F00F0503EB83030CF00F0C05EB4C
:10C8E00044050CEB430C0D7081F801E081F802C0A7
:10C8F000002030BD03685B6810B50020C3F3423EE2
:10C900006EF30700C3F3042EC3F3074CC3F30724ED
:10C910006EF30F2003F03F0363F317406CF31F60C7
:10C920000860D2B91A0902EB820203F00F0303EB8D
:10C9300042034FEA1E1E8B704FEA1C130EEB8E0E45
:10C9400004F00F0403EB83030CF00F0C04EB4E0414
:10C950000CEB430C4C7081F803C0002010BD00BFED
:10C9600038B50368DA68520601D5002038BDDA68A8
:10C9700042F08002DA600446FCF704FC05462368B6
:10C98000DB685B06F1D4FCF7FDFB431BB3F57A7F54
:10C99000F5D9236804226277DB68012038BD00BF27
:10C9A00038B50368DA6822F08002DA609A68920685
:10C9B00001D5002038BD0A4ADA600446FCF7E2FBE4
:10C9C00005462368DB689B06F3D4FCF7DBFB431BBF
:10C9D000B3F57A7FF5D904236377012038BD00BF12
:10C9E0005F7F0100002845D038B5437F044603F03F
:10C9F000FF024BB1022223686277DA68D20607D5BC
:10CA000001236377002038BD0277FBF77FFAF1E757
:10CA1000CA215322596220465A62FFF7A1FF2368B8
:10CA200010B1FF225A6238BD99686268256921F405
:10CA3000E00121F040019960616998682A430A4346
:10CA40000243E1689A6019611A69A16842EA0142E9
:10CA50001A612046FFF7A4FF23680028E1D11A6C71
:10CA6000A06922F480221A641A6CFF2102431A641E
:10CA70005962C5E701207047037F012B78D070B55C
:10CA80000E46012102230177016843778B68054632
:10CA9000002A37D113F0400C18BF96F803C0337842
:10CAA0000CBF86F803C04FEA8C5C092B09D9002023
:10CAB0000A3BDBB2092B00F10100F9D843EA00136D
:10CAC000DBB21C047378092B09D900200A3BDBB2C6
:10CAD000092B00F10100F9D843EA0013DBB2B0786A
:10CAE00009284FEA032308D90A38C0B2092802F1FD
:10CAF0000102F9D840EA0210C0B244EA0C041C4317
:10CB000004430FE07478327813F040034FEA0424B2
:10CB100014BFF378F37044EA0244B27818BF9B055F
:10CB200014431C43CA234B6253234B622846FFF72E
:10CB300017FF28B12A68FF21002351622B7770BDAF
:10CB40002B683069F26804F07F3424F0FE441C60E6
:10CB5000996821F480219960996802430A43284624
:10CB60009A60FFF71DFF0028E4D101236B77E1E70E
:10CB70000220704738B5037F012B6FD00546022392
:10CB8000012028776B7791F800E0CB78487891F80E
:10CB900002C04FEA4E3EAAB14EEA034444EA0C04F6
:10CBA00044EA00242B68CA215322596228465A625B
:10CBB000FFF7D6FE002840D02A68FF2100235162EB
:10CBC0002B7738BDC40646D520F010000A30C0B21D
:10CBD000092B487098BF1C040DD900210A3BDBB219
:10CBE000092B01F10101F9D843EA0113DBB209284D
:10CBF0004FEA034409D900230A38C0B2092803F1D7
:10CC00000103F9D840EA0313D8B2BCF1090F4FEA87
:10CC100000200CD9ACF10A0C5FFA8CFCBCF1090FB6
:10CC200002F10102F6D84CEA02125FFA82FC44EAF1
:10CC30000E04044344EA0C04B4E72B6824F07F4458
:10CC400024F0C0045C602846FFF7AAFE0028B3D198
:10CC500001236B77B0E7092BBFD8C8E7022038BDA6
:10CC6000F8B5037F012B50D01646012202770368E6
:10CC700002224277CA225A6253225A629A680446B2
:10CC800050050D460DD5FCF77DFA074605E0FCF78B
:10CC900079FAC01BB0F57A7F2ED82368DA6851077D
:10CCA000F5D49A6822F480629A60DA68D2B262F4AB
:10CCB0009062DA60FCF766FA074605E0FCF762FA74
:10CCC000C31BB3F57A7F17D82368DA685207F5D506
:10CCD0009A6822F007029A609A6832439A605D610E
:10CCE0009A6842F480629A600021FF200122586213
:10CCF000627721770846F8BD2268FF21032351623D
:10CD00006377002323770320F8BD0220F8BD00BF1E
:10CD10000B4A03684FF4800110B55161DA6852057F
:10CD2000044602D40123637710BDDA68D2B262F4FC
:10CD30009062DA60FBF758FB0123637710BD00BFF8
:10CD4000003C01400368503343F82120704700BF86
:10CD50000368503353F82100704700BF836B1A6893
:10CD6000D36B43F48073D363704700BFF0B589B0D1
:10CD700005460F46FCF706FA002200230646082166
:10CD80002868CDE9002301F02DFE044610B12046AD
:10CD900009B0F0BD296D2868090401F083FE04463E
:10CDA0000028F4D14FF0FF320823CDE902233022CE
:10CDB0000223CDE9042302A9002201232868CDE93A
:10CDC000062301F009FD286801F088FE044640B101
:10CDD000DDE7436B9B0415D5FCF7D4F9831B0133C6
:10CDE00027D02868436B13F02A0F0BD1436B9A02AC
:10CDF000EFD501F0D7FC08AB03EB8403013443F813
:10CE0000200CE9E7436B190719D4436B9A0516D434
:10CE1000436B9B0710D4446B14F0200412D1DDE95E
:10CE2000003240F23A5112BA1BBA8163C7E90023BB
:10CE3000ADE74FF00044AAE702248463A7E7082483
:10CE40008463A4E720248463A1E700BF80B110B508
:10CE500004460323006884F8343001F0B1FC204616
:10CE6000FBF73EF90023A36384F83430184610BD65
:10CE7000012070472DE9F043044687B000297FD098
:10CE800090F8340001285FFA80F866D11E46E36D01
:10CE90001746324400259A42A56308D9A36B43F094
:10CEA0000073A3630125284607B0BDE8F0830A4656
:10CEB0002168206CDFF8ECC0032384F83430CD62A5
:10CEC000CB6B43F44A7343F00203CB630565856083
:10CED0000568314BC3632B68C0F84CC023F0C00316
:10CEE0004FEA46292B6080314FEA9903FCF7F6FCA4
:10CEF0000546002836D1294B2068C3F88C85636C21
:10CF0000CDF80490012B4FF090024FF00203CDE9D1
:10CF100002234FF000014FF00103CDE904134FF05D
:10CF2000FF33694618BF7F02009301F055FC012EC4
:10CF30002BD9822320682363394601F06DFD002838
:10CF4000B1D02368164A9A63A36B012103430022E0
:10CF5000A36384F834102263A4E70225284607B0AF
:10CF6000BDE8F08323680E49DA6B22F49572DA6328
:10CF70009963A36B43F08043A36384F8348091E703
:10CF8000836B43F0006383638CE781232068236312
:10CF9000394601F033FDD2E7D9D0000800802542A0
:10CFA000FF054000ADD600082DE9F041044686B0EB
:10CFB00000296DD01D4690F83430012B30D1C36D5F
:10CFC0000E4600218163501998422ED820683D4FAB
:10CFD000032384F83430C162C36B43F4067343F017
:10CFE0000203C363E36B1965616CDF63012918BF3A
:10CFF0005202354FDF64012D11464ED9A023236321
:10D0000001F024FD07462268C7B1304B9363A36B40
:10D0100001213B430022A36384F83410226308E01B
:10D020000226304606B0BDE8F081A36B43F00073E2
:10D03000A3630126304606B0BDE8F081E06B244BC7
:10D0400031464FF001080668C3F88C85336823F039
:10D05000C00343F040034FF0400C6D02C0F808C01D
:10D0600080323360AB08FCF739FC0646D8B1226841
:10D07000D36B23F4067323F00203D363134B936340
:10D08000A36B43F08043A36384F834802763D0E725
:10D09000836B43F000638363CBE79023236301F04A
:10D0A000C9FC0746AFE790230293206801954FF033
:10D0B000FF336946CDE90377CDF81480009301F082
:10D0C0008BFBAEE75DCD0008ADD60008FF05400044
:10D0D00000802542704700BF10B5846B236B206829
:10D0E000822B0FD0C36A23F00803C36240F23A5187
:10D0F00001220023816384F834202046236302F058
:10D10000BFFB10BD01F0B0FC034608B92068E9E799
:10D11000A26B13432046A363FFF7DCFFF6E700BFD3
:10D12000426E10B40346940FC2F383600C704870D3
:10D13000C2F30164C2F307408C70C870C2F30720C9
:10D14000D2B208714A719A6E140DCC80C2F30344B6
:10D150000C72C2F3C0344C72C2F380348C72C2F3CE
:10D160004034CC720020C2F300340C734873586C06
:10D1700000286FD1D86E40F6FC7404EA820242EABD
:10D180009072C0F3C2640A610C75C0F34252C0F3DE
:10D1900002644C758A75C0F38244C0F3C232CC7508
:10D1A0000A760C690A7E02F00702023201349440CA
:10D1B0005C6591F808C001220CF00F0C02FA0CF229
:10D1C0009A65520A04FB02F2DA65C0F380324FF42A
:10D1D00000741C664A76C0F3C61200F07F008A769F
:10D1E000C8761B6FDC0FC3F341720C774A77C3F329
:10D1F0008264C3F383528C770020CA77C3F3405410
:10D20000C3F3004281F8204081F82100C3F3C03409
:10D2100081F82220C3F3803281F8234081F8242052
:10D22000C3F34034C3F3003281F8254081F826204F
:10D23000C3F38124C3F3012281F82740C3F34603DB
:10D2400081F82820012281F8293081F82A205DF810
:10D25000044B704701280FD1D86E120402F47C12DF
:10D2600042EA10420A610A69013292024FF40074E4
:10D27000C3E916425A65A8E71A68064991639A6B92
:10D28000012142F080529A6383F8341008465DF819
:10D29000044B7047FF054000F0B5002299B076239B
:10D2A000CDE90A230024099409AB054693E8070059
:10D2B0008DE80700CDE906440894824E286806AB45
:10D2C0000ECB01F053FA01272868C6F8A04001F000
:10D2D00073FA0220C6F8A070FBF75AFF286805947D
:10D2E00001F090FA044648B1012385F83430AB6B65
:10D2F0002343AB630124204619B0F0BD286801F038
:10D30000CFFC002840F0C880AF642868002101F0FD
:10D31000C9FB08BB059B4FF6FE76B3421FD86A4F88
:10D320000DE02146286801F053FA059B013305936F
:10D33000059BB34204464FEAD07210D87AB9002157
:10D34000286801F0AFFB394604460028CCD1286894
:10D3500001F07CFA0028E4D04FF08054C4E7059A2D
:10D360004FF6FE739A4200F2A980C4F38074012341
:10D3700028686C64ADF8123001F026FA002800F03D
:10D3800095806B6C2868032B1CD1042101F020FAD6
:10D39000000DE8640DA92846FFF7C2FE04460028E8
:10D3A00040F087802A6D28681204234601F06CFB48
:10D3B0000146002853D0012385F83430AB6B0B4372
:10D3C000AB6397E701F0D2FB01460028F3D1286850
:10D3D00001F0FEF9034604216B67286801F0F8F9B3
:10D3E00003460821AB67286801F0F2F90346EB67B2
:10D3F00028680C2101F0ECF96B6CC5F88000032B58
:10D400002868C2D00DF1120101F00EFC014600287F
:10D41000D1D16B6C2868032BB7D0BDF812102965E9
:10D42000090401F0AFFB01460028C4D1286801F0CF
:10D43000CFF9034604216B66286801F0C9F9034659
:10D440000821AB66286801F0C3F90346EB6628683B
:10D450000C2101F0BDF903462B67286895E72A46A1
:10D460002B1D52F8106B07CA8DE8070030460ECB13
:10D4700001F07CF928684FF4007101F0B3FA00283C
:10D480003FF439AF2B68114A9A63AB6B0122034317
:10D49000AB6385F834202DE72868AC6401F0B2F95D
:10D4A00050B9AB6C012B7FF435AF2EE74FF08061A4
:10D4B00081E74FF080517EE7044615E74FF0807416
:10D4C00012E700BF00802542000010C1FF054000A8
:10D4D000C8B110B590F83430044603F0FF0273B1C0
:10D4E000032384F834302046FFF7D6FE28B9012301
:10D4F000A063206384F8343010BD012010BD027792
:10D50000FAF738FDECE70120704700BFF0B4D0E92E
:10D5100011C7D0E91365D0E91542D0E91730C1E948
:10D5200000C7C1E90265C1E90442C861F0BC00203E
:10D530008B6170470000000070B5426C0323032A22
:10D540008AB0044680F834300E46036825D0B1F521
:10D55000805F22D0B1F5006F61D000293DD0826B91
:10D5600042F000628263A56BF5B9D4E90512CDE9FA
:10D570000812D4E90112CDE90412E2680796069276
:10D580000AAA12E907008DE8070004AE184696E8DB
:10D590000E0001F0EBF823680CE0A26B42F0805221
:10D5A000A263A56B002DE0D0012235499963154691
:10D5B00084F834204FF40071184601F013FA30B1AA
:10D5C00023682F4A9A63A36B03430125A3630123B6
:10D5D000284684F834300AB070BD00221846002373
:10D5E000CDE9042301F0F4F8820139D404A92046DE
:10D5F000FFF7BCFB014668B9059BDB0335D5216D00
:10D600002068090401F04EFA014618B9206801F0BB
:10D6100057FA0146A26B23680A43A263C1E79FED54
:10D62000167B184600218DED047B01F0D1F88001B6
:10D6300019D404A92046FFF799FB60B9059B59034B
:10D6400016D5216D2068090401F02CFA18B920685C
:10D65000022101F035FAA26B23680243A263A0E71E
:10D660004FF40061D6E73046F5E74FF08061D1E72F
:10D670004FF08060EFE700BF0000000000000000F6
:10D68000FF054000016D10B509040446006801F073
:10D6900035FA014620B1A36B0B430020A36310BDF4
:10D6A000206801F095F8C0F3432010BD10B5846BDD
:10D6B000FCF782FA02280AD0D4E90F235B6D526D81
:10D6C000012B05D0012A03D02046FFF703FD10BD32
:10D6D0002368104A9A63DA6B22F49D72DA63A36BB3
:10D6E00043F080432046A363FFF7CCFF05380128B1
:10D6F00008D90122002384F8342020462363FFF751
:10D70000E9FCE4E7206801F0AFF9A36B0343A363EE
:10D71000EFE700BFFF05400010B5846B236840F2BF
:10D720003A529A632046FFF7ADFF012205380023E5
:10D73000904284F83420236308D9A36B204613B9A0
:10D7400002F096F810BDFFF7C5FC10BD206801F08F
:10D750008BF9A36B0343A363EFE700BF2DE9F0410F
:10D7600004460068256B436B1A0482B01DD52B0755
:10D7700000F1C080436BDB056BD54FF4807383638E
:10D78000C36B23F4434323F03A03C363C36A23F018
:10D790000103C362290605D5AA0600F1EC80AB0798
:10D7A00000F0BB8002B0BDE8F081436BDF0523D5FC
:10D7B0004FF480738363C36B23F4434323F03A0332
:10D7C000C363C36A2E0723F00103C362E2D515F0D9
:10D7D000220F40F0B08040F23A53836301220023CD
:10D7E00084F8342020462363AC0700F09F8002F0C9
:10D7F00047F802B0BDE8F081436B5F042AD52E07DD
:10D8000028D5666A002ECDD0276A07F1040807F1F3
:10D81000240500E0206818F8043C019318F8032C54
:10D8200043EA0223019318F8022C43EA02430193CE
:10D8300018F8012C01A943EA026308F104080193D6
:10D8400000F0B4FF4545E5D12037203EC4E9087615
:10D85000A8E7436B426B40F23A231A42A2D0436BD3
:10D86000990703D5A36B43F00203A363436B1A0725
:10D8700003D5A36B43F00803A363436B9B0603D557
:10D88000A36B43F02003A363436BDF0603D5A36BB5
:10D8900043F01003A363436B9E0503D5A36B43F0D2
:10D8A0000803A36340F23A738363C36B23F44E739C
:10D8B00023F00203C36301F0D7F8A36B290743EAFF
:10D8C0000003A3633DD42A067FF56CAF15F0300F3B
:10D8D00047D115F003055BD0206C324B0365FCF794
:10D8E00083F800283FF45EAF206C02B0BDE8F04141
:10D8F000FFF712BFD4E90A57002F3FF453AF05F1E9
:10D90000200600E0206800F04DFF45F8040BB5420A
:10D91000F8D1203FC4E90A5744E72268D36A0121BD
:10D9200023F00803D362204684F8341001F0A4FFEA
:10D9300002B0BDE8F08101F097F8034650B92068C5
:10D9400049E70122002384F8342020462363FFF7AF
:10D95000C1FB27E7A26B13432046A363FFF7BAFB83
:10D96000EDE7E06B104B0365FCF73EF800283FF451
:10D9700019AFE06BB9E701F077F8034600283FF4F0
:10D980000EAFA26B13432046A363FFF7A3FB06E78A
:10D990000123A563204684F83430256301F068FF35
:10D9A00000E700BFADD9000819D70008FFF7B4BEE3
:10D9B00000285CD070B50446406A002847D0002398
:10D9C000C4E9043394F851300022A26203F0FF014D
:10D9D000002B42D094462168A568A269266A0223DA
:10D9E00084F851300B6823F040030B60636805F442
:10D9F000044503F482732B43E56805F400652B436B
:10DA0000256905F002052B43656905F001052B43E7
:10DA1000E56906F0800E02F4007605F03805334320
:10DA20002B43120C00F0100043EA0E0302F0040234
:10DA300043EA0C0302430B604A60CB69002023F4E5
:10DA400000630122CB61606584F8512070BD63687A
:10DA5000B3F5827FB6D0E061B4E7204684F8501079
:10DA6000FAF78EFBD4E9090303F4005CB3E7012065
:10DA7000704700BF704700BF30B5026851689368B7
:10DA800013F0400F85B00446C3F3801516D113F090
:10DA9000010F53D198076AD508067CD4980613D491
:10DAA000DB0568D58D0666D5636D002043F008035D
:10DAB0006365039093680393039B18E0980742D52E
:10DAC000080668D4980640D5880654D5002D56D14E
:10DAD000606D40F001006065002002909068029047
:10DAE000106820F0400010600298DB05DCD4636D04
:10DAF000002B40D05368012023F0E0038D075360D2
:10DB000084F8510059D05368E06C23F0030353604C
:10DB100040B12C4B0365FBF767FF18B1636D43F011
:10DB200040036365A06C30B3264B0365FBF75CFFD5
:10DB300008B3636D43F0400363651CE011F0400FD0
:10DB4000A8D0036C29E09D0617D4880613D594F855
:10DB50005100032817D0606D40F00400606500207C
:10DB60000090D0680090906800900098BDE79806FB
:10DB700096D58806ACD405B030BD8D06FBD594F89B
:10DB8000510003280DD100230193D36801939368BA
:10DB90000193019BEFE7636C204605B0BDE8304080
:10DBA0001847606D40F00400606500200090D06868
:10DBB00000909068009000988AE72046FFF75AFF8F
:10DBC000D9E700BFC9DB000808B5806B0023C38715
:10DBD000C386FFF74FFF08BD90F83D30012B2FD1D2
:10DBE00003681849022280F83D20DA688B4242F02F
:10DBF0000102DA6019D0B3F1804F16D0124A934275
:10DC000013D002F5806293420FD002F580629342F6
:10DC10000BD002F57842934207D002F5705293423E
:10DC200003D0A2F59432934204D19A6802F007021D
:10DC3000062A03D01A6842F001021A6000207047D9
:10DC40000120704700000140000400400368DA68CA
:10DC500022F00102DA601A6A41F211110A4208D177
:10DC6000196A40F24442114203D11A6822F00102BB
:10DC70001A60012380F83D300020704790F83C2066
:10DC8000012A6ED00346026830B40120022483F8D2
:10DC90003C0083F83D40946824F47F4424F07704EA
:10DCA00094600C68602C76D011D8402C5BD02ED8B4
:10DCB000202C04D000F2888034F010011FD191682C
:10DCC00021F07001214341F00701916016E0B4F5A5
:10DCD000805F13D0B4F5005F33D0702C0FD1D1E941
:10DCE000015094682843CD6824F47F4140EA052020
:10DCF00008439060916841F0770191600020012114
:10DD0000002283F83D1083F83C2030BC7047502C33
:10DD1000F5D14868CC68116A21F00A010843116AFC
:10DD200021F001011162916921F0F00141EA041131
:10DD300091611062916821F0700141F0570191608A
:10DD4000DCE7D1E9015094682843CD6824F47F4191
:10DD500040EA052008439060916841F48041916059
:10DD6000CCE7022070474868CC68116A21F00A01AC
:10DD70000843116A21F001011162916921F0F0015B
:10DD800041EA041191611062916821F0700141F043
:10DD900047019160B2E74868CC68116A21F0A001A0
:10DDA00041EA0011106A20F010001062906920F41E
:10DDB000704040EA043090611162916821F0700176
:10DDC00041F06701916099E7302C3FF478AF96E716
:10DDD000704700BF704700BF704700BF704700BF6B
:10DDE000036870B5DE681D69A907044601D5B2074E
:10DDF00051D4690701D572073AD42B0701D53007F2
:10DE000024D4EA0601D5F30610D4E80701D5F107BA
:10DE100057D42A0601D533065BD4680601D57106AE
:10DE20005FD4AA0601D5B30642D470BD23686FF053
:10DE300010021A6108222277DB6913F4407F204622
:10DE400063D0FFF7C7FF00232377DEE723686FF077
:10DE500008021A6104222277DB699907204651D112
:10DE6000FFF7B6FF2046FFF7B7FF00232377C8E789
:10DE700023686FF004021A61022222779B6913F46F
:10DE8000407F20463BD1FFF7A3FF2046FFF7A4FFCA
:10DE900000232377B1E76FF002021A6101220277B3
:10DEA0009B699B0725D0FFF795FF00232377A0E709
:10DEB00023686FF0200220461A61BDE8704000F030
:10DEC00009B923686FF001021A612046F9F782FC54
:10DED0009FE723686FF080021A61204600F0FCF88B
:10DEE0009BE723686FF040021A612046FFF776FF38
:10DEF00097E7FFF76DFF2046FFF76EFFD5E7FFF7C7
:10DF000069FFC5E7FFF766FFAFE7FFF761FF204650
:10DF1000FFF762FF97E700BF70B4344E4A690368A9
:10DF20008D680C68B04245D0B0F1804F34D0A6F572
:10DF30007C46B04230D006F58066B0422CD006F563
:10DF40008066B04228D006F57846B04232D0284EDE
:10DF5000B04225D006F58066B04221D006F5806635
:10DF6000B0421DD0A6F59836B04233D006F5806693
:10DF7000B04215D006F58066B04211D023F0800380
:10DF8000C5621A4384620368012143F004030360FD
:10DF900070BC4161026070474E6823F070033343E8
:10DFA000C968C56223F440730B4323F080031A430E
:10DFB0008462E8E74E6823F070033343CE68C5629D
:10DFC00023F44073334323F0800384621A430B69C4
:10DFD0000363D8E7C96823F440730B4323F080033D
:10DFE0001A43044BDD629C62CDE700BF0000014094
:10DFF000004001400018004050B310B590F83D308B
:10E00000044603F0FF02F3B12146022384F83D30B9
:10E0100051F8040BFFF780FF012384F8463084F8A1
:10E020003E3084F83F3084F8403084F8413084F842
:10E03000423084F8433084F8443084F8453084F822
:10E040003D30002010BD80F83C20FAF7C9FBDBE72B
:10E050000120704790F83C20012A37D0034602681F
:10E06000022030B483F83D0050680D68946820F0B9
:10E07000700028435060164882421AD0B2F1804F97
:10E0800017D0A0F57C40824213D000F58060824218
:10E090000FD000F5806082420BD000F578408242BC
:10E0A00007D000F57050824203D0A0F59430824230
:10E0B00004D1496824F080040C43946000200122BC
:10E0C00083F83D2083F83C0030BC70470220704745
:10E0D00000000140704700BF704700BF026802F1B6
:10E0E0000C0353E8003F23F4907302F10C0C4CE84E
:10E0F00000310029F3D102F1140353E8003F23F06B
:10E10000010302F1140C4CE800310029F3D1036B38
:10E11000012B05D02022002380F8422003637047A2
:10E1200002F10C0353E8003F23F0100302F10C0C42
:10E130004CE800310029F3D1ECE700BF0268116917
:10E1400038B50446C068A36821F4405101432069F2
:10E15000116103436069D1680343E06921F416410A
:10E1600021F00C0103430B43D3605369A069234999
:10E1700023F4407303438A42536105D0204B9A42F3
:10E1800002D0FEF79BFA01E0FEF7A8FAE269192136
:10E19000B2F5004FD4E90053A0FB010113D09A005F
:10E1A0009B0FF2F751FE174AA2FB00135B09642193
:10E1B00001FB130000013230A2FB00201B0103EB26
:10E1C0005013AB6038BDDA184FF000035B41F2F733
:10E1D0003BFE0C4AA2FB00314909642303FB1103F7
:10E1E000DB003233A2FB0323C3F342121B0902EB11
:10E1F000011203F4F8731344AB6038BD0010014002
:10E20000001401401F85EB5170B310B590F84130F8
:10E21000044603F0FF0213B32268242384F841303C
:10E22000D36823F400532046D360FFF787FF2368A9
:10E23000196921F490411961596921F02A01596144
:10E24000D96800224FF0200C41F40051D96062647B
:10E2500084F841C084F842C01046626310BD80F863
:10E260004020FAF76DFDD7E701207047002832D033
:10E2700010B590F84130044603F0FF0233B3226832
:10E28000242384F84130D36823F400532046D3601C
:10E29000FFF754FF2368196921F490411961596906
:10E2A00021F022015961596941F008015961D96889
:10E2B00000224FF0200C41F40051D960626484F8D0
:10E2C00041C084F842C01046626310BD80F840200F
:10E2D000FAF736FDD3E70120704700BF90F84130D0
:10E2E000202B15D101B10AB90120704710B40023C9
:10E2F000046801622121C284436480F84110E1680E
:10E30000828441F08001E16018465DF8044B70475B
:10E310000220704790F84230202B03D101B11AB986
:10E32000012070470220704710B404698162002305
:10E33000222103638285C2854364036880F842100A
:10E340001CB1DA6842F48072DA605A695DF8044BF5
:10E3500042F001025A61DA6842F020020020DA60DD
:10E36000704700BF704700BF704700BF08B5806BA3
:10E370000023C385FFF7F8FF08BD00BF704700BF4B
:10E3800090F84230222B57D183680168826AB3F536
:10E39000805F44D0002B4BD10369002B48D14B68E0
:10E3A000DBB21370826A0132C38D8262013B9BB281
:10E3B000C385002B40D100B50268D16821F020014F
:10E3C00083B0D160D16821F48071D16051694FF080
:10E3D000200C21F00101516180F842C04363016BC0
:10E3E00001292AD1036302F10C0353E8003F23F013
:10E3F000100302F10C0C4CE800310029F3D1136832
:10E40000DB0606D50023019313680193536801933B
:10E41000019B818DFFF7B2FF03B05DF804FB036938
:10E42000002BBCD14B68C3F3080322F8023BBBE7C7
:10E430004B6803F07F03B4E77047FAF73FFD03B082
:10E440005DF804FB70B505682B68EE68696913F028
:10E450000F0F82B004462A4672D19D0602D5B1063E
:10E4600000F1C680216B01290BD0180602D53106B8
:10E4700000F194805B0602D5750600F1AE8002B013
:10E4800070BDD806F1D5F106EFD5002301931368CE
:10E49000019353680193019B5169A38D4D0640F18F
:10E4A0000C81E06B0168496889B2002900F048815D
:10E4B000994280F04581E185C169B1F5807F36D010
:10E4C00002F10C0353E8003F23F4807302F10C05C2
:10E4D00045E800310029F3D102F1140353E8003F6D
:10E4E00023F0010302F1140545E800310029F3D1BE
:10E4F00002F1140353E8003F23F0400302F1140536
:10E5000045E800310029F3D1202384F8423021630B
:10E5100002F10C0353E8003F23F0100302F10C0555
:10E5200045E800310029F3D1FBF714FAA38D02224C
:10E530006263E18D591A204689B2FFF71FFF9EE7FB
:10E5400011F0010176D116F4907F8BD0DA070AD54D
:10E55000F00540F1EC80626C580742F00102626401
:10E560004FD500296AD198075AD5190700F1A28022
:10E57000626C002A83D09A0602D5B30600F1DB80D4
:10E580006B69626C03F0400302F0080253EA020672
:10E5900020465CD1FFF7E8FE666470E794F84130EE
:10E5A000212B7FF46CAFA168236AB1F5805F00F086
:10E5B000D080591C21621B785360E38C013B9BB2D5
:10E5C000E384002B7FF45BAFD36823F08003D36038
:10E5D000D36843F04003D36051E7D368202123F090
:10E5E0004003D360204684F84110FFF7BBFE46E7A6
:10E5F00002B0BDE87040FFF7C3BEF005ABD45A07C8
:10E600001CD498070CD50029AFD0626C42F00402EC
:10E6100062641A07ACD5626C42F008026264A7E734
:10E620001807A5D506F020020A43F4D1636C002B2D
:10E63000A6D124E7DA07E0D4580738D5626C9907E9
:10E6400042F002026264E0D41A07E4D490E7FFF7D4
:10E6500045FD6B695E0626D505F1140353E8003FBE
:10E6600023F0400305F1140141E8003262B1226851
:10E6700002F1140353E8003F23F0400302F11400B9
:10E6800040E800310029F3D1E06B60B1364B0365FF
:10E69000FBF7AAF900283FF4F2AEE06B036D02B07D
:10E6A000BDE8704018472046FFF75EFEE7E6990791
:10E6B000ABD4C9E7B206AED4B8E7E08DE18D89B23C
:10E6C00080B200293FF4DBAE1B1A99B200293FF457
:10E6D000D6AE02F10C0353E8003F23F4907302F12D
:10E6E0000C0545E800300028F3D102F1140353E88B
:10E6F000003F23F0010302F1140545E80030002833
:10E70000F3D1202384F84230206302F10C0353E854
:10E71000003F23F0100302F10C0545E8003000280B
:10E72000F3D1022363632046FFF728FEA7E65A07CA
:10E730003FF519AF65E72046FFF722FE25681FE782
:10E7400099427FF49CAEC369B3F5807F7FF497AEA6
:10E75000E7E7216900297FF42CAF33F8021BC1F3EE
:10E7600008015160236228E76DE3000884B010B40B
:10E770000DF1080C8CE80E000B46049913430B4373
:10E78000DDE90541426823430B4307995DF8044BDB
:10E7900022F4FD420B4322F07F021343436004B096
:10E7A00000207047D0F88000704700BF0B68C0F8A9
:10E7B00080300020704700BF0323036000207047B3
:10E7C0000346002018607047006800F0030070479F
:10E7D00014304058704700BF10B4D1E900428B6834
:10E7E0004462CC6882622343D1E90441C26A234374
:10E7F00022F0F7020B431343C3625DF8044B002081
:10E80000704700BF00220F4B8260C2680E491B6830
:10E810006FF30B02A1FB031342F480625B0A41F227
:10E820008831C26001FB03F343B1426B120603F16E
:10E83000FF33F9D5C5238363002070474FF00040B4
:10E84000704700BF6C030020D34D621041F00041BF
:10E8500041F48011164B8160C26816491B686FF342
:10E860000B02A1FB031342F48D625B0A41F2883173
:10E8700042F0010201FB03F38446C26043B1DCF8BD
:10E88000342012F0450F01D0120504D5013BF6D11A
:10E890004FF000407047DCF8340010F0040015BF62
:10E8A0000420C523CCF83800CCF83830704700BFBE
:10E8B0006C030020D34D6210474B10B41B68474CCB
:10E8C000A4FB03435B0A03FB02F2531E4AB1426BF3
:10E8D00012F0450F03F1FF3301D0120506D55C1C81
:10E8E000F5D14FF000405DF8044B7047436B5B0778
:10E8F0003CD4436BDC0707D4C52383630369DBB2D5
:10E90000994204D00120EEE701238363FAE74369CB
:10E91000334818400028E6D0002B2BDB5A002CD4BB
:10E920009C002CD4D9002CD41A012DD45C012ED4F7
:10E93000D9012FD41A0230D45C0231D499023BD4CD
:10E94000DA0236D45C0331D499032CD4DA033FD4F1
:10E950001C043AD4590435D49A0430D413F0080F67
:10E960000CBF4FF480304FF40000BCE704238363F6
:10E970001846B8E74FF00070B5E74020B3E78020B5
:10E98000B1E74FF48070AEE74FF40070ABE74FF49F
:10E990008060A8E74FF40060A5E74FF48050A2E73D
:10E9A0004FF400509FE74FF480209CE74FF4003075
:10E9B00099E74FF4004096E74FF4804093E74FF417
:10E9C000800090E74FF400108DE74FF480108AE745
:10E9D0004FF4002087E700BF6C030020D34D621086
:10E9E00008E0FFFD8160C1686FF30B0141F48A61AB
:10E9F000C16041F288321021FFF75EBF8160C368B9
:10EA00006FF30B0343F48A6343F0010341F288324E
:10EA1000C3601121FFF750BF8160C3686FF30B0320
:10EA200043F48A6343F0020341F28832C360122147
:10EA3000FFF742BF8160C1686FF30B0141F48B6146
:10EA4000C16041F288321821FFF736BF8160C36888
:10EA50006FF30B0343F48B6343F0010341F28832FD
:10EA6000C3601921FFF728BF00238360C368054AEC
:10EA70006FF30B0343F4896343F00403C3600C2179
:10EA8000FFF71ABF00E1F5058260C3686FF30B035F
:10EA900043F4886343F0070341F28832C3600721DF
:10EAA000FFF70ABF8160C3686FF30B0343F48E6303
:10EAB00043F0070341F28832C3603721FFF7FCBE01
:10EAC0008160C3686FF30B0343F4886343F006036C
:10EAD00041F28832C3600621FFF7EEBE0023836057
:10EAE000C3686FF30B0343F48E6343F0030341F2F7
:10EAF0008832C3603321FFF7DFBE00BF8160C36887
:10EB00006FF30B0343F4896343F0050341F288324A
:10EB1000C3600D21FFF7D0BE124B134A1B68A2FB46
:10EB2000032341F288315B0A01FB03F301463BB149
:10EB30004A6B12F0450F01D0120504D5013BF7D105
:10EB40004FF0004070474B6B5B0707D4486B10F0E9
:10EB5000010014BF0123C5238B6370470420886321
:10EB6000704700BF6C030020D34D62100023836008
:10EB7000C3686FF30B0343F4986343F00203C3606D
:10EB8000FFF7CABF8160C3686FF30B0343F4996357
:10EB900043F00103C360FFF7BFBF00BF204B10B4B9
:10EBA0001B68204CA4FB03435B0A41F2883404FB3E
:10EBB00003F33BB1446B14F0450F01D0240506D597
:10EBC000013BF7D14FF000405DF8044B7047436BB9
:10EBD0005B071BD4436BDC0705D40369DBB29942A6
:10EBE00004D00120F0E701238363FAE7C5238363A0
:10EBF000436913F4604010D05A040BD413F4004F4F
:10EC00000CBF4FF480304FF48050DDE70423836362
:10EC10001846D9E74FF40050D6E71B0C1380D3E712
:10EC20006C030020D34D621000238360C3686FF330
:10EC30000B0343F4886343F003030A46C3600321D4
:10EC4000FFF7ACBF144B154A1B68A2FB032341F22C
:10EC500088315B0A01FB03F301463BB14A6B12F0BA
:10EC6000450F01D0100504D5013BF7D14FF000400E
:10EC700070474B6B5A070CD4486B10F0010005D15C
:10EC80004B6B5B06F4D540238B63704701238B638A
:10EC900070470420886370476C030020D34D6210D6
:10ECA0004FF4D5728260C2686FF30B0242F489623E
:10ECB000C260FFF7C7BF00BF82B00023019302E02C
:10ECC0000369002B09DB019B01330193019BB3F125
:10ECD000706FF5D9032002B070470A230193019B9E
:10ECE0002BB1019B013B0193019B002BF9D10369DF
:10ECF00043F00103036103E0036913F0010307D04C
:10ED0000019B01330193019BB3F1706FF4D9E1E7EB
:10ED1000184602B0704700BF84B010B50DF10C0C5E
:10ED20008CE80E009DF81130012B044624D1836B32
:10ED30009DF8182023F480338363C36823F484038D
:10ED400023F04003C360C368012A23F44013C36067
:10ED500025D02046FFF7B0FF9DF80E30012B07D1DC
:10ED6000A36843F00603A360A36843F02003A360F5
:10ED7000BDE8104004B07047C36843F04003C3606F
:10ED8000FFF79AFF9DF8153023B9A36B43F4803346
:10ED9000A363E1E7A36B23F48033A363DCE7C368D9
:10EDA00043F48013C360D4E7022A03460AD04FF429
:10EDB0001051DA6822F47052DA60DA680A430020EF
:10EDC000DA607047264A27480A44824232D9264AE6
:10EDD00026480A44824230D92548A1F57402A2F59A
:10EDE000105282422CD92348A1F18372A2F5E74246
:10EDF000824228D3204A21480A44824226D9204A06
:10EE000020480A44824224D31F4A20480A448242AE
:10EE1000CDD31F48A1F1B772A2F5585282421BD33D
:10EE20001C4A1D480A4482422CBF4FF4C0514FF483
:10EE3000E051BEE74FF47051BBE74FF46051B8E7C3
:10EE40004FF45051B5E74FF44051B2E74FF4305111
:10EE5000AFE74FF42051ACE74FF40051A9E700BFF2
:10EE6000405327FFFF340C00401E1BFF3F420F00A2
:10EE70007F4F120020D6130060B6E5FE5FE3160058
:10EE800000D3CEFE40771B00C05BB3FEC0912100D3
:10EE900020753800E05459FEE09C410003460020F4
:10EEA0009A6842F001029A60704700BF0346002052
:10EEB0009A6822F001029A60704700BF38B5C368B3
:10EEC000012923F0C0430546C36018D0A9B9C3681F
:10EED00043F080430C46C36001E0C82C0DD00A20EB
:10EEE000FAF756F96B69DB0704F10A04F5D4A4F1CB
:10EEF000C800B0FA80F0400938BD012038BDC368B1
:10EF000043F000530024C36001E0C82CF5D00A2070
:10EF1000FAF73EF96B69DA0704F10A04F5D5A4F1B2
:10EF2000C800B0FA80F04009E6E700BF82B00023D5
:10EF3000019302E00369002B09DB019B013301937C
:10EF4000019BB3F1706FF5D9032002B070478901BE
:10EF5000002341F020010193016103E0036913F0F4
:10EF6000200307D0019B01330193019BB3F1706F24
:10EF7000F4D9E9E7184602B0704700BF82B0002319
:10EF8000019302E00369002B09DB019B013301932C
:10EF9000019BB3F1706FF5D9032002B070470022D6
:10EFA00010230192036103E0036913F0100307D0FB
:10EFB000019B01330193019BB3F1706FF4D9EBE72F
:10EFC000184602B0704700BF84B0F8B507AC84E8BB
:10EFD0000E0000239DF81C509DF82660044619463B
:10EFE00003F1400204EB820201330F2B5160F7D191
:10EFF00004F50067002E40F09F807B6843F0020319
:10F000007B60A36B43F40013A363A36B23F400237F
:10F01000A363A36B23F48023A3630023C4F8003EFF
:10F020009DF82130012B00F09780D4F8003843F090
:10F030000303C4F8003810212046FFF777FF01468C
:10F040002046FFF79BFF41EA000E5FFA8EFE00228A
:10F05000BEF1000E3A6118BF4FF0010E7A61FA61FD
:10F0600005B3D4F80019002904F5106315DB00215D
:10F07000196000204FF67F310132AA421861996071
:10F0800003F1200336D0D3F800C0BCF1000FEEDA54
:10F090004FF0904CC3F800C0EEE74FF00061C4F8A9
:10F0A0000019E6E73B6923F480733B6100229DF879
:10F0B0001E30A2616FF0804262611BB9A36943F008
:10F0C0001003A361A2692C4B13439DF82220A36176
:10F0D0001AB1A36943F00803A361012E05D1A36906
:10F0E00043F0804343F00403A3617046BDE8F84059
:10F0F00004B07047D4F8002B002A04F5306315DB08
:10F100000022002119604FF0000C4FF67F300132D1
:10F11000AA42C3F810C0986003F12003C2D0196856
:10F120000029EEDA4FF090411960F0E74FF00062ED
:10F13000C4F8002B0022E6E7A36B23F40013A363BB
:10F14000A36B43F40023A3630023C4F8003E9DF89F
:10F150002130012B7FF469AF9DF81F3023B9D4F81B
:10F160000038C4F8003866E7D4F8003843F00103EB
:10F17000C4F800385FE700BF00383C80D0F808389A
:10F1800013F0060004D013F0020F14BF02200F206A
:10F19000704700BF10B50A78012302F00F0E03FA82
:10F1A0000EF391F801E0BEF1010F00F5006C00EBE9
:10F1B00042101AD0DCF81C2042EA0343CCF81C3081
:10F1C000D0F8003B1B040ED48B68D0F8004B0A79B2
:10F1D000C3F30A03234343EA824343F0805343F4D7
:10F1E0000043C0F8003B002010BDDCF81C40234366
:10F1F000CCF81C30D0F800391C04F4D48B68D0F85B
:10F2000000490979C3F30A03234343EA814343EAEC
:10F21000825343F0805343F40043C0F80039002088
:10F2200010BD00BF10B40A784978012900EB4213E1
:10F230002CD0D3F8001B00291BDBD0F83C484FF43E
:10F24000803102F00F0201FA02F224EA0204C0F84F
:10F250003C48D0F81C48224924EA0202C0F81C2885
:10F26000D3F8002B5DF8044B11400020C3F8001BBD
:10F270007047D3F8001B41F00061C3F8001BD3F8BE
:10F28000001B41F08041C3F8001BD6E7D3F80019FA
:10F2900000290BDAD3F8001941F00061C3F8001916
:10F2A000D3F8001941F08041C3F80019D0F83C1898
:10F2B00002F00F040122A24021EA0201C0F83C182A
:10F2C000D0F81C48074924EA0202C0F81C28D3F8E9
:10F2D00000295DF8044B11400020C3F80019704765
:10F2E0000078F3EF007833EC2DE9F0434C780E789A
:10F2F0000D6991F804E0012C00EB46135BD0D3F8C4
:10F30000104B6FF31204C3F8104BD3F8104B6FF38C
:10F31000DC44C3F8104B03F5306C8C6856BB05B168
:10F320000C610C62DCF81050C4F312042C43CCF8CE
:10F330001040DCF81040012A44F40024CCF81040BE
:10F3400033D0BEF1010F0CD1D0F8082812F4807F21
:10F35000D3F8002B0CBF42F0005242F08052C3F8A9
:10F36000002BD3F8002B42F00442C3F8002B0020FE
:10F37000BDE8F083002DD5D0614E2544013DB5FB9D
:10F38000F4F5ADB205FB04F406EAC545DCF81060FF
:10F390000C623543CCF81050DCF81050C4F3120462
:10F3A0002C43012ACCF81040CBD1CA68002AC8D01F
:10F3B000CCF81420C5E703F510648DB32769D1F8A4
:10F3C00008906FF31207276127696FF3DC47276105
:10F3D000002E4FD12769A94547F400273CBFC1F84B
:10F3E00010904D4627612769C5F312053D43012A58
:10F3F000256123D0D3F80049BEF1010F44F0044445
:10F40000C3F800490C6958D0002CB0D0D0F834288B
:10F4100006F00F060123B3401343C0F83438A6E7C3
:10F4200025696FF3DC452561256945F400252561D3
:10F430002569012A6FF312052561DBD1CA6902B182
:10F440006261BEF1010F0CD1D0F8082812F4807F60
:10F45000D3F800290CBF42F0005242F08052C3F8AA
:10F460000029D3F8002942F00442C3F80029002003
:10F47000BDE8F083224FD4F8108009EB050C0CF1A5
:10F48000FF3CBCFBF9FC07EACC4747EA0807BEF1A2
:10F49000010F27611FFA8CFCA5D14FEA4C7C0CF0C0
:10F4A000C047D4F810C02CF0C04CC4F810C0D4F839
:10F4B00010C047EA0C07276195E7D0F8085815F403
:10F4C000807FD3F800590CBF45F0005545F08055BA
:10F4D000C3F80059002A7FF44AAFA3B203339B0854
:10F4E0003FF445AFCA6800EB063606F5805602EBDE
:10F4F000830352F8041B31609342FAD137E700BF0F
:10F500000000F81F10B44A780B7883B00021012A5C
:10F5100001914FEA431323D000F53060C218C1585F
:10F52000002904DB002003B05DF8044B7047C45889
:10F5300044F00064C450C45844F08044C45042F2C3
:10F54000107102E01368002BECDA019B0133019388
:10F55000019B8B42F6D9012003B05DF8044B704744
:10F5600000F51060C218C1580029DBDAC45844F015
:10F570000064C450C45844F08044C45042F2107136
:10F5800002E01368002BCDDA019B01330193019B4C
:10F590008B42F6D9DFE700BF10B49DF8044064B990
:10F5A00003339B0809D0013200EB023001EB8303E7
:10F5B00051F8042B02608B42FAD100205DF8044B15
:10F5C000704700BF70B55FEA920E054602F0030671
:10F5D0001AD000F580548C460023013322684CF881
:10F5E000042B9E45F9D101EB8E0066B105F58055DF
:10F5F00006442968002321FA03F200F8012BB042E7
:10F6000003F10803F7D170BD0846EEE74A780B789E
:10F61000012A00EB43100CD0D0F8002B002A00DBAD
:10F62000D3B9D0F8003B43F40013C0F8003B0020EE
:10F630007047D0F80029002A06DB2BB1D0F800393A
:10F6400023F08043C0F80039D0F8003943F40013A8
:10F65000C0F8003900207047D0F8003B23F0804309
:10F66000C0F8003BDDE700BF0B794A7891F800C095
:10F67000023B012A00EB4C10DBB211D0D0F8002B7A
:10F68000012B22F40012C0F8002B01D90020704792
:10F69000D0F8003B43F08053C0F8003B0020704797
:10F6A000D0F80029012B22F40012C0F80029EDD86F
:10F6B000D0F8003943F08053C0F80039002070477B
:10F6C000D0F8003823F4FE63C0F80038D0F80038D2
:10F6D000090101F4FE611943C0F8001800207047C9
:10F6E000D0F8002E034622F00302C3F8002ED3F810
:10F6F000043800F5006123F0020300204B607047DE
:10F70000D0F8002E034622F00302C3F8002ED3F8EF
:10F71000043800F5006143F0020300204B6070479D
:10F720004269806910407047D0F8183800F50060D1
:10F73000C0691840000C7047D0F8183800F5006018
:10F74000C069184080B2704700EB411100F50060BD
:10F75000D1F8082B40691040704700BFD0F810283E
:10F76000D0F8343800EB411001F00F01CB40DB0141
:10F77000D0F80809DBB2134318407047406900F025
:10F7800001007047D0F8002903466FF30A02C3F85E
:10F790000029D3F8043800F5006143F48073002099
:10F7A0004B60704730B4056C114CA54200F53063D6
:10F7B00003D9D0F8004B002C16DB00241C611C6917
:10F7C00044F400241C611C6944F018041C611C6989
:10F7D000012944F0C0441C6106D15A61D0F8003BB5
:10F7E00043F08023C0F8003B002030BC704700BFCE
:10F7F0000A30544F08B50349034803F0BBFE034BDE
:10F80000187008BD40FA0020A468020844FA0020DD
:10F8100000207047844608B5044813460A466146EE
:10F82000FDF728FB003818BF012008BD40F7002075
:10F83000844608B5044813460A466146FDF7B4FB02
:10F84000003818BF012008BD40F7002008B5034864
:10F85000FDF718FF043818BF012008BD40F700204D
:10F8600001460148FDF752BE40F70020704700BF37
:10F8700008B5FFF7FBFF08BD08B500F02DF908BD7E
:10F8800008B500F031F908BD00B583B001238DF84B
:10F89000073000F021F808B98DF807009DF807003F
:10F8A00003B05DF804FB00BF08B5FFF7EDFF0128CA
:10F8B00001D0012008BD0748FDF70AFE0028F9D154
:10F8C0004FF400610348FDF737FE003818BF0120F0
:10F8D00008BD00BF40F7002008B508210348FBF72A
:10F8E00047F9B0FA80F0400908BD00BF000C0240A3
:10F8F00030B5164B187810F0010489B006D11546C2
:10F90000032920D8DFE801F0030F1706032420465F
:10F9100009B030BD6846FFF7A3FF079B20465B0A8E
:10F920002B6009B030BD6846FFF79AFF069B2B603D
:10F93000204609B030BD6846FFF792FF079B2B8039
:10F94000204609B030BD0424E1E700BF8003002059
:10F950002DE9F04184B00D4616461F4603F0CAFE5D
:10F9600047F22F58044602E0FFF770FF40B103F062
:10F97000C1FE001B4045F7D9012004B0BDE8F0816D
:10F980003A4631462846FFF753FF0028F4D10E4B84
:10F9900047F23052196801A804F00CF8019B102BB3
:10F9A000EAD1029B022BE7D103F0A4FE47F22F55C8
:10F9B000044603E0FFF74AFF0028DED003F09AFE7A
:10F9C000031BAB42F6D9D7E748FA002070B5184CB4
:10F9D00084B00125257003F085FE10B9207804B0AD
:10F9E00070BDFFF761FFB8B12378012BF6D0114D40
:10F9F0002E68002EF2D1104B0FCBEC468CE80F0096
:10FA00003146604603F09AFF28600028E6D123784B
:10FA100043F001032370E1E72570FFF717FF18B9E2
:10FA2000237803F0FE0323702378DBB22370DBE737
:10FA30008003002048FA00203435020810B5064C37
:10FA400001232370FFF702FF18B9237803F0FE03A8
:10FA50002370207810BD00BF800300202DE9F04105
:10FA600084B00D4616461F4603F044FE47F22F5859
:10FA7000044602E0FFF7EAFE40B103F03BFE001B44
:10FA80004045F7D9012004B0BDE8F0813A4631463F
:10FA90002846FFF7BFFE0028F4D10E4B47F2305244
:10FAA000196801A803F086FF019B102BEAD1029B85
:10FAB000012BE7D103F01EFE47F22F55044603E069
:10FAC000FFF7C4FE0028DED003F014FE031BAB4298
:10FAD000F6D9D7E748FA0020024B00221868022125
:10FAE00003F03EBF48FA0020024B002218680121B3
:10FAF00003F036BF48FA0020704700BF2DE9F047F9
:10FB0000DFF8E0802C4F2D4E2D4D8CB000244FF4AB
:10FB10007A7A4FF00409CDF808A0009701233C60E1
:10FB200034602C603022CDF80490A0214046FBF7D1
:10FB30001DFCCDE9019A009601233422A021404604
:10FB4000FBF714FC009501233822CDE9019A4046C9
:10FB5000A021FBF70BFC2146204607F0F3FE0094A2
:10FB6000184A33681360184B2868184918603C68B5
:10FB7000174D18480C60029017480190284608F06D
:10FB800041FB284608F0DCFB144C284608F0DEFB5D
:10FB90002846134908F04EFC0FCC0DF1140CACE8CC
:10FBA0000F0094E807008CE80700294605A803F039
:10FBB000A9FD0CB0BDE8F08754FA002050FA0020EF
:10FBC0004CFA00205CFA002058FA002060FA00206D
:10FBD00064FA0020A9780108DDFD00084435020818
:10FBE000F9FA0008A0F5002000207047F8B590F859
:10FBF0002D305A0728D52E4D2E4E28680C464FF42E
:10FC0000FA6103F03DFE2C48FAF73AFC302200215D
:10FC1000304610F05EFF14B3D4E9002333606389EB
:10FC20007360A2B106F10C034FF0010C50685189CA
:10FC3000126843F8043CC3E900010C3342B10CF1F3
:10FC4000010CBCF1040FF1D16FF00B00F8BD94462C
:10FC50000CEB4C0C06EB8C0C0023CCF80830174F47
:10FC60002389BE60144E7B6020467C6308F068FEEA
:10FC700039463046FAF740FB0028E7D03046FAF71D
:10FC800099FD83074FF4FA610CD5286803F0F8FD5D
:10FC90003046FAF7F5FB39463046FAF72DFB0028D7
:10FCA000D4D0EBE7204608F0CDFC6FF00B00CDE799
:10FCB000D8FB002098FA002028FB0020F0FA002052
:10FCC000F9F760BA844608B5054813460A46614606
:10FCD000FAF77CFC003818BF0120404208BD00BF85
:10FCE00028FB002008B50248FAF736FD002008BDC1
:10FCF00028FB0020844608B5054813460A4661469D
:10FD0000FAF78CFC003818BF0120404208BD00BF44
:10FD100028FB002008B50146074808F0A7F9074B63
:10FD20001A78012A00D008BD054900221A70BDE8E2
:10FD30000840086803F0D0BDF068020820FD0020EC
:10FD4000DCFB00202DE9F043144CDFF85480DFF891
:10FD5000549083B00646002720684FF0FF3103F02F
:10FD60008FFD0028F8D198F800300197002BF3D1CF
:10FD700001A94846FAF7F2FA019D31462846002DBE
:10FD8000EAD0336998470028EDD0284608F05AFC9D
:10FD900098F800300197002BDED1E9E7DCFB00206A
:10FDA00020FD002028FB0020014B186803F094BDC3
:10FDB000DCFB0020014B186803F08EBDD8FB00204F
:10FDC00008B5FAF7FBFC030600D408BD024B18681F
:10FDD000BDE8084003F080BDDCFB00202DE9F041C8
:10FDE0000446AAB0002800F0C980684B684A694EF2
:10FDF00047F27341C4E90523E1856422002111A87B
:10FE000010F067FE04AB0093634A73604FF4000385
:10FE10003260B3604FF47A72604B02924FF0060882
:10FE2000F3605F4BCDF804805E4933614FF4C063EB
:10FE3000002573614022012304915B48ADF8145002
:10FE4000A021FBF793FA3046FAF78CF8574B294676
:10FE500034220746184610F03CFE212240F8042CBC
:10FE60004FF440020261524808F088F8736884F841
:10FE70002C80197884F82610597884F827109978FE
:10FE800084F82810D97884F82910197994F82D204D
:10FE900084F82A105B7984F82B3042F00A0240F291
:10FEA000DC5384F82D20A384012106A8069507952C
:10FEB00003F0BAFC3F4E0121306008A8CDE9085597
:10FEC00003F0B2FC034630683B4E2946336003F032
:10FED000D7FC2946394D306803F0D2FC0FCD0DF127
:10FEE000280CACE80F0095E807008CE807002146D5
:10FEF0000AA803F007FC32493248F9F783F8314881
:10FF0000F9F798F858BB27BB2E48F9F7C7F801282E
:10FF100025DD033802282CD82B4A2C4B52F82060C0
:10FF200053F820501B4811A9FAF79EFB11A9194854
:10FF3000CDE91656FAF702FC1648FAF737F92046CB
:10FF400008F004FA204608F037FA00202AB0BDE88D
:10FF5000F081F7F785FC00202AB0BDE8F08120464B
:10FF600008F04EFA204608F00BFA00202AB0BDE84F
:10FF7000F0814FF480454FF40066D3E7144B1549E8
:10FF8000154840F20D2210F09FFC2EE7EDFB000813
:10FF90008DE0010828FB002000800240E0FB0020EB
:10FFA00080FC00200080E100A0F50020F4FA002091
:10FFB000F0680208DCFB0020D8FB00206035020856
:10FFC00084030020D0FA0020E4680208D868020800
:10FFD000EC3D0208083E0208183E0208F9F7D2B8C4
:10FFE000F0B53B4B02688DB000249A42CDE906443F
:10FFF000CDE908440A9401D00DB0F0BDA3F59043BB
:020000040801F1
:1000000000941A6B334842F000721A631A6B02F0C4
:1000100000720092009A01941A6B42F080621A6397
:100020001A6B02F080620192019A02941A6B42F0FC
:1000300000621A631A6B02F000620292029A039441
:100040001A6B42F004021A631A6B02F00402039264
:10005000039A04941A6B42F001021A631A6B02F0BD
:1000600001020492049A05941A6B42F040021A634A
:100070001B6B03F040033222059303260B2506A9D0
:100080000223CDE906230227059BCDE90965FAF78E
:1000900099FB862306A910480A95CDE90637CDE9D4
:1000A0000846FAF78FFB4FF4D04306A90B48069396
:1000B000CDE9084607970A95FAF784FB2246062100
:1000C0003D20F9F7BDFA3D20F9F7F6FA0DB0F0BD85
:1000D0000080024000080240000002400018024078
:1000E0002DE9F04F9BB000270446642200216846AA
:1000F00010F0EFFCDFF894B0DFF894A0214D224E11
:10010000B946B84604E001280DDC642003F02AFB60
:100110002846F8F7C3FF94F82D305A07F3D5012885
:1001200022DD5B07F1D40238032819D85BF8207070
:100130005AF8209069463046FAF796FA69463046F2
:10014000CDE90579FAF7FAFA3046FAF72FF82046A2
:1001500008F032F9204608F0F9F84FF00108D4E72A
:10016000B8F1000FD1D0E5E73046FAF76FF8204636
:1001700008F006F9204608F043F9E369204698475D
:10018000C3E700BFD0FA002028FB0020C86802089F
:10019000B868020810B5044682B00D4807F036FF73
:1001A000034678B100F120020A4922604FF4C06092
:1001B00019610021CDE900204122084608F090F99C
:1001C00002B010BD044A20600121117002B010BDC0
:1001D000F068020815FD000820FD002030B400255D
:1001E00042F8205CA2F1200422F8163C22F8185CA8
:1001F000026862B10A6814600C6002682AB1118951
:10020000194411811268002AF9D130BC704704608A
:10021000F2E700BF08F016BAD0F8D43200EB830042
:1002200010B5D0F8C04284B1D0F8C4325BB194F8B4
:100230000002FF2807D09B6894F8012221469847C6
:10024000FF2384F80032002010BD032010BD00BF42
:100250000A230380004870471404002070B58221EF
:1002600006460F4800F0BAFB012105460C4800F095
:10027000B5FB812104460A4800F0B0FB0DB1102205
:10028000AA711CB1002240212171627118B10022B3
:1002900040210171427143230148338070BD00BF8A
:1002A00098030020FFF7DABF70B5822106460F4899
:1002B00000F094FB012105460C4800F08FFB8121E2
:1002C00004460A4800F08AFB0DB11022AA711CB145
:1002D000002102222171627118B1002102220171F4
:1002E000427143230148338070BD00BF9803002052
:1002F00038B5D0F8D432B03350F8235095B1044615
:100300000FF03CFBD4F8D432C5F80C0204EB8304A4
:10031000D5F80402D4F8C43205F50371DB689847B8
:10032000002038BD032038BD70B5D0F8D442D0F8D5
:10033000C86200EB840EDEF8C05245B301F00F0432
:1003400004EB840C00EB8C0C0A46DCF814306BB91F
:10035000DEF8C4321B690021C5F8141223B1D5F8A8
:10036000080205F504719847002070BD04EBC40431
:1003700006EB8406F469B3FBF4F604FB1633002B9A
:10038000E6D1CCF814301A460FF0E0FAECE703207F
:1003900070BD00BF70B5D0F8D43200EB830382B0DB
:1003A000D3F8C06200228DF80520ADF8062066B1B2
:1003B00091F800C01CF0600204460D461ED0202AB1
:1003C00006D02946204600F0C9FD032002B070BDCA
:1003D000CA8891F801E07AB31CF0800F4CD0D3F8B2
:1003E000C43231469B6870469847EA88072A3146EE
:1003F00028BF0722204600F0E9FD22E04B780B2BB6
:10040000DFD801A252F823F0510401084304010887
:10041000C3030108C3030108C3030108C3030108A0
:10042000C3030108C3030108C3030108C303010890
:100430006504010847040108D3F8C43270469B687C
:1004400098470020C2E790F89C32032BF9D0B8E718
:1004500090F89C32032BB4D102220DF1060100F07A
:10046000B5FDEEE790F89C32032BAAD101220DF1E5
:10047000050100F0ABFDE4E7402A28BF402286F8E2
:1004800000E286F80122314600F0B6FDD9E700BF50
:1004900038B50446002581210FF014FA012184F8B3
:1004A000375020460FF00EFA822184F8775120460B
:1004B0000FF008FAD4F8D43284F84B5004EB8303DD
:1004C0006564D3F8C0228AB1D3F8C4325B68984718
:1004D000D4F8D432B03354F823000FF057FAD4F8DC
:1004E000D432B03344F82350C4F8BC52002038BD95
:1004F000F8B504464FF407700FF044FA054600289B
:100500005BD04FF40772002110F0E3FAD4F8D43234
:10051000B03344F82350237CC4F8BC52B3B3402317
:100520000222812120460FF0BFF90121402384F8E7
:100530003710022220460FF0B7F9012710230322BB
:1005400063648221082384F8777120460FF0ACF9A8
:10055000D4F8D43284F84B7004EB83030026D3F82C
:10056000C432C5F804621B689847D5F80422C5F860
:100570001462C5F818622AB3237CC3B94FF4007320
:10058000394620460FF0EEF90020F8BD4FF4007315
:100590000222812120460FF087F901214FF40073D8
:1005A00084F83710022220460FF07EF9C5E7402379
:1005B000394620460FF0D6F9E6E7D4F8D432B03306
:1005C00044F823000220F8BD034639B1D0F8D42204
:1005D00003EB82030020C3F8C41270470320704766
:1005E000D0F8D432B03350F823302BB1C3F808120E
:1005F000C3F810220020704703207047D0F8D4328F
:10060000B03350F823301BB1C3F8041200207047F8
:1006100003207047D0F8D432B03350F8232092B181
:1006200010B5D2F814420CB1012010BD0123C2F85C
:100630001432D2F81032D2F80822836281210FF0EE
:1006400085F9204610BD0320704700BFD0F8D422A2
:10065000B03250F822208AB108B5037CD2F80422C7
:100660002BB1402301210FF07DF9002008BD4FF48C
:10067000007301210FF076F9002008BD03207047B8
:1006800078B10023C0F8B832C0F8C432C0F8D03214
:1006900009B1C0F8B412012380F89C3202700FF047
:1006A000C5B80320704700BF10B582B00023ADF875
:1006B000063089B1CB6AC0F8B812044623B10DF1F7
:1006C00006009847C4F8D002D4F8D832002001338D
:1006D000C4F8D83202B010BD032002B010BD00BF74
:1006E0000FF0D6B8D0F8B8320BB11B6818471846CF
:1006F000704700BF08B5D0F8B8325B68984700284B
:1007000018BF032008BD00BF38B5044600F2AA2573
:10071000284600F017FC94F8AA12B4F8B022C4F8E6
:1007200098220123C4F8943201F01F03012B0ED04C
:10073000022B06D08BB929462046BDE8384000F090
:1007400063B929462046BDE8384000F049BB294638
:100750002046BDE8384000F003BB204601F0800190
:10076000BDE838400FF0BAB810B5044629B9D0F842
:100770009422032A10D0002010BD90F89C32032B45
:10078000F9D1D0F8B8329B69002BF4D00022BDE833
:100790001040C0F8D4221847B0F860210B46D0F8BA
:1007A0005811914208D890F89C22032A12D0204672
:1007B00000F03AFC002010BD8B1AD0F86411C0F88C
:1007C000583111449A42C0F8641138BF1A4600F0FB
:1007D00023FCD0E7D0F8B8221269002AE7D0C0F88D
:1007E000D4329047E3E700BF70B5044659B9D0F85A
:1007F0009432022B16D094F8A03213B1002384F85F
:10080000A032002070BD90F89C32032BF9D1D0F8B3
:10081000B8325B69002BF4D00022BDE87040C0F80C
:10082000D42218478269038C9A420D4610D81DD0F5
:1008300094F89C32032B26D0802120460FF04EF8EE
:10084000204600F0FDFB94F8A032002BD9D0D5E76C
:10085000416AD21A19448261416200F0C5FB2B46FD
:100860002A46294620460FF07DF8C4E743699A429C
:10087000DED8D0F898229342DAD20A4600F0B4FBD0
:10088000C4F89852EBE7D4F8B832DB68002BD3D029
:100890000022C4F8D42220469847CDE7F8B5D0F816
:1008A000B8320021012280F89C2204464160C0F841
:1008B0009412C0F8A41280F8A0121BB15B680BB1AF
:1008C0009847B8B900270022402511460126402349
:1008D00020460EF0E9FF84F86361A4F860512B46CE
:1008E0000022802120460EF0DFFF84F8236025845B
:1008F0003846F8BD0327E6E701740020704700BFC3
:1009000090F89C32042B04D090F89C32DBB280F833
:100910009D32042380F89C320020704790F89C326E
:10092000042B04D190F89D32DBB280F89C32002079
:10093000704700BF90F89C22032A01D00020704726
:1009400008B5D0F8B83213B1DB6903B1984700207D
:1009500008BD00BFD0F8D422AE3250F8222062B1D8
:1009600008B590F89C32032B01D0002008BD136A13
:10097000002BFAD09847002008BD0320704700BF25
:10098000D0F8D422AE3250F8222062B108B590F8E7
:100990009C32032B01D0002008BD536A002BFAD0F3
:1009A0009847002008BD0320704700BF0020704713
:1009B000D0F8B822012180F89C1242B108B55268E3
:1009C0000179904708B9002008BD032008BD002028
:1009D000704700BF00207047002070470278B0F8D1
:1009E00002C09445134603D80CE09C450AD902780E
:1009F000104413444278052A9BB2F6D182788A4289
:100A0000F3D170470020704770B50B7803F0600396
:100A1000202B82B00D46044628D0402B26D05BB157
:100A2000802120460EF05AFF002120460EF056FF8E
:100A30000025284602B070BD4B78092BF0D801A2E2
:100A400052F823F0BD0A0108E50A0108210A01084D
:100A5000030B0108210A01081B0B01085D0B0108AB
:100A6000210A0108910B0108850A0108D4F8D43243
:100A7000AE33294654F823309B68204602B0BDE8C7
:100A8000704018478978B54D0129297000F24181DD
:100A900090F89C32022BDEB200F02081032E00F091
:100AA000FB8080210EF01AFF002120460EF016FF79
:100AB00029782046FFF71EFE0325BAE790F89C32FE
:100AC000013B022BACD8CA88022AA9D1D0F8A432A3
:100AD0000146002B0CBF0123032341F80C3F00F01B
:100AE00075FAA5E790F89C32013B022B98D84B8809
:100AF000012B9DD10023C4F8A432204600F094FAC3
:100B000096E74B88012BF6D0022B89D18B881B0AE4
:100B100080F8A03200F088FA8AE78B88002B7FF4F7
:100B20007FAFCB88002B7FF47BAF4B887F2B3FF6CA
:100B300077AF90F89C22032A3FF472AFDDB280F8C1
:100B40009E5229460EF0F6FE204600F06DFA002D6A
:100B500000F0FF80022384F89C3269E74A88130A78
:100B60000021013BADF80610062B3FF659AF01A15D
:100B700051F823F0370C01081D0C01080B0C01087B
:100B8000210A0108210A0108F50B0108B90B010827
:100B9000CA88012A7FF444AF90F89C32022BD9B264
:100BA00000F2B08000293FF43BAF0146002341F83A
:100BB000083F00F00BFA3BE7037C002B7FF430AFDB
:100BC000D0F8B8320DF106001B6B9847072343702D
:100BD000EB88002B91D0BDF80620002A3FF420AF0F
:100BE0009A4228BF1A4601462046ADF8062000F07A
:100BF000EDF91DE7037C002B7FF412AFD0F8B8327B
:100C00000DF106005B6B9847E2E7D2B2052A3FF68A
:100C100007AFDFE802F03B352F292318027CD0F81C
:100C2000B832002A40F087809B6A0DF10600984791
:100C300002234370CCE7D0F8B432007C1B680DF17E
:100C400006019847C4E7D0F8B4329B69002B3FF403
:100C5000E7AE207C0DF106019847B9E7D0F8B43231
:100C60005B69002BF5D1DBE6D0F8B4321B69002BB1
:100C7000EFD1D5E6D0F8B432DB68002BE9D1CFE66E
:100C8000D0F8B4329B68002BE3D1C9E6D0F8B43277
:100C90005B68002BDDD1C3E6002942D04168012901
:100CA0003FF42BAFC9B2FFF725FD297861602046DC
:100CB000FFF718FD054600283FF41FAF80212046AE
:100CC0000EF00CFE002120460EF008FE2179204691
:100CD000FFF710FD022384F89C32AAE600293FF4B6
:100CE0000CAF01214160FFF7FDFC054650B38021A8
:100CF00020460EF0F3FD002120460EF0EFFD84F8B3
:100D00009C6296E603297FF48BAE011D00F05EF92C
:100D10008EE680210EF0E2FD002120460EF0DEFD81
:100D2000CAE6022380F89C324160FFF7E3FC2046CC
:100D300000F07AF97CE6DB6A0DF1060098470223A1
:100D4000437045E7204600F06FF9032384F89C3296
:100D50006EE6012384F89C326AE600BFAB460120B0
:100D600070B50B785A060D4604460DD503F06002A7
:100D7000402A09D080210EF0B1FD002120460EF05E
:100D8000ADFD0026304670BD94F89C32013B022B2D
:100D900002D82979012908D9802120460EF09EFD2C
:100DA000002120460EF09AFDEBE72046FFF712FEE9
:100DB00090B9D4F8B8329B6873B1C4F8D40229460C
:100DC00020469847EB880646002BDBD10028D9D176
:100DD000204600F029F9D5E70326304670BD00BF54
:100DE00030B50C468A88237803F06003202B83B04B
:100DF0000546D1B24DD0402B4BD053B1802128466F
:100E00000EF06CFD002128460EF068FD002003B0B6
:100E100030BD6378012B2BD0032B4CD0002BEDD1B0
:100E200090F89C32022BD8B25FD00328E6D101F0B3
:100E30000F0303EB8303120605EB830365D493F8DA
:100E40006331002BDAD0142404FB015404F5AA7496
:100E5000002968D028460EF059FD00286BD00123E8
:100E6000A373022204F10E01284600F0AFF8CDE78B
:100E700090F89C32022BDAB22ED0032ABED16388BE
:100E8000002BC3D14B0651D12846019100F0CCF87C
:100E900001992846FFF7A0FD0028B7D1D5F8B83250
:100EA000C5F8D4029B68002BB0D02146284603B079
:100EB000BDE83040184790F89C32022BDAB20BD0D4
:100EC000032A9BD163881BB9480601D0E388A3B3EA
:100ED000284600F0A9F899E74A068FD00EF0FEFCEC
:100EE000802128460EF0FAFC90E7480686D11106CC
:100EF0004CBF05F1140105F5AA71002301F80E3F5E
:100F00000222284600F062F880E793F82330002B95
:100F10003FF474AF01F07F04013404EB84048029B2
:100F200005EB840496D10023A3739AE701910EF098
:100F3000E1FC0199A8E7A07393E728460EF0CEFCE8
:100F4000C6E700BF0B7803704B7843704B88438033
:100F50008B888380CB88C380704700BF10B5802109
:100F600004460EF0BBFC20460021BDE810400EF008
:100F7000B5BC00BF30B370B503780E4614460546C5
:100F80000BB3034613F8011F0029FBD1681CEFF7D0
:100F900029F9431CDBB201335B00DAB2238003235F
:100FA000327073702C7864B12846022300215A1CD9
:100FB000D2B2F454B15410F8014F0233DBB2002C1A
:100FC000F5D170BD704702221346E7E708B5134616
:100FD0000A460221C0E90533C0F89412426200219A
:100FE0000EF0B4FC002008BD08B513460A460021E7
:100FF0000EF0ACFC002008BD08B513460A460321DC
:10100000C0E95533C0F89412C0F8642100210EF0F5
:10101000A9FC002008BD00BF08B513460A46002100
:101020000EF0A0FC002008BD08B504210023C0F884
:1010300094121A4619460EF089FC002008BD00BF24
:1010400008B505210023C0F894121A4619460EF07F
:1010500089FC002008BD00BF034B03EB8002034462
:101060005268187A53681847D446012038B5084D9D
:101070002B5C5BB905EB80022B1852680446187A8A
:101080001368984708B901232B5538BD002038BD97
:10109000D446012030B4054C04EB800504446D684F
:1010A000207AAC68A44630BC604700BFD44601201B
:1010B00030B4054C04EB800504446D68207AEC687C
:1010C000A44630BC604700BFD4460120044B03EB6C
:1010D000000C03EB80039CF808005B681B69184751
:1010E000D4460120264A136870B4ABB10468A34209
:1010F00009D01369ABB1A3423AD002290CBF00203A
:10110000122070BC704784685568A5420CD01569E0
:101110003DB1AB42F1D110E0146914B10568A542AC
:101120000DD0002070BC704745699668AE4225D04E
:101130001569002DF5D09D42DFD1002501E08468BE
:1011400001255369A34202D0002DD6D0E9E7946966
:1011500043699C42F8D1012369B902EB031270BCC8
:101160009089A0F58070B0FA80F0400900017047C6
:1011700084680025E5E7102070BC70470023EBE78A
:10118000AC4601200246294BF0B418681568854228
:1011900024D01C69AC4206D000282FD0002C41D0AE
:1011A0000020F0BC70475E699768BE42F4D19E692A
:1011B0005769BE4208BF4FF0010CEDD103EB0C1292
:1011C0004FEA0C149289A1B1002AE9D10CF1010077
:1011D0004FF480722344F0BC9A81704794685E6833
:1011E000A642D6D154699E68A642D2D14FF0000CD7
:1011F000E4E7013292B20CF10100EBE784460120F2
:101200004FEA0C1400291D519568526903EB0C112B
:10121000C1E901524FF000028A8114BF4FF480727D
:101220000122D7E702204FF0010CE9E7AC4601208C
:10123000016899B191F800C0BCF11F0F13D90A469B
:10124000634603E012F8013F1F2B0CD93A2BF9D16A
:10125000BCF1300F02D101318A4202D04FF0FF3091
:101260007047013202600020704700BFF8B5C378B4
:101270000BB90020F8BD456B00F138070446012387
:1012800040782A463946FFF713FFA8B9A26A236AB5
:10129000E070AA1A9A42ECD2A678012E01D8E8E7AB
:1012A000236A60781D442A4601233946013EFFF730
:1012B000FFFE012EF4D1DCE70120F8BD2DE9F0415D
:1012C0000026D0F800808E75C369002B5AD0036BBE
:1012D000013307460D461CD0D8F80C30188898B159
:1012E00001F1150601240AE0412C0DD006F8010F8A
:1012F000D8F80C3033F81400621C30B114460021C9
:1013000002F05CF90028EFD100242C440023A375DF
:10131000AE7D3F6A00237C1E18464FF0E50C14F8A2
:10132000011F202900F101001DD0052903F1010250
:101330002AD0092834D02B4459726EBBA1F1410E3A
:10134000BEF1190F27D8082897F80CE057D81EF0DF
:10135000080F18BF2031997514F8011F2029134672
:1013600000F10100E1D10B28D9D12B44B6B3002202
:101370005A72FB7A2B72FB692B60D7F81630EB8020
:101380001B0CAB80BDE8F08109282DD02B4483F8DD
:1013900009C00EB9E52199750B281346BFD1E4E7C2
:1013A0002A4405EB030E4FF02E0896B98EF81680EE
:1013B0008EF80980A1F1410EBEF1190F517205D8C6
:1013C00097F80CE01EF0100F18BF20319175023312
:1013D000A5E78EF8098002335172A0E79E753A7B2B
:1013E000002A08BF2B46C2E72A447EB1E9184FF015
:1013F0002E0E81F809E0E521023351728FE71EF0CD
:10140000100FC8D02031C9B29975C5E705EB030E9E
:1014100071464FF02E088EF816804EF22E5EA1F81F
:1014200009E0E5210233917579E700BF38B5436BD8
:101430008B4201D1002038BD05460C46FFF716FF50
:101440000028F8D122466878012305F13801FFF71A
:1014500021FE00281CBF4FF0FF3401206C6338BD13
:10146000F8B50546FFF702FF50B92B78032B08D0DB
:10147000002268781146FFF729FE003818BF0120C6
:10148000F8BD2E79012EF3D105F138070146044647
:101490004FF4007238460FF01CFB4AF65523A5F8AE
:1014A00036320C4BAB6303F1FF536A6AA869C5F887
:1014B000200203F500532033C5F81C3201326B695A
:1014C000C5F8243268786A6333463946FFF7F0FD81
:1014D0002C71CDE75252614138B50D4640B10368D9
:1014E00004462BB11A781AB18188DA88914203D068
:1014F000092000232B6038BD186902F0DDF803468F
:1015000068B123685878FFF7A7FD10F00100236841
:10151000F0D0002BECD0186902F0D8F8E8E70F20E3
:10152000E8E700BF70B54FF0FF360023B142044634
:10153000C370466322D1B4F836224AF655239A4244
:101540001AD194F83830E92B07D0A36B134A03F073
:10155000FF13934201D0022070BDD4F86E30104AC0
:1015600023F07F43934217D0D4F88A000D4BC01A62
:1015700018BF0120400070BD032070BD0D460A4613
:101580004078012304F13801FFF784FD10B1666350
:10159000042070BD6563CEE7002070BDEB009000B5
:1015A0004641540046415433F0B5002385B00B60EA
:1015B0000E461746FFF73CFE041EC0F2C580944B52
:1015C00053F82450002D00F0BC80286902F074F814
:1015D00010B90F2005B0F0BD35602B7807F0FE077D
:1015E000002B40F08680E0B200232B706870FFF77C
:1015F0003DFDC60700F1B28017B1440700F19F809E
:1016000000212846FFF78EFF02287DD0042800F035
:10161000A980012898BF002600F28E80B5F84330DB
:10162000B3F5007F40F08880B5F84E10002900F037
:10163000978095F848202962531E012BAA707BD809
:1016400095F845306B81002B76D0581E184273D127
:10165000B5F849702F8138076ED1B5F84B0000B945
:10166000A86DB5F846C0BCF1000F65D001FB02F2D1
:101670000CEB17141444A0425ED3001B9842B0FB3D
:10168000F3FE59D30CEB06034FF6F57CE6453444E4
:101690000EF1020068D9AB62B5F862302C633B43AF
:1016A000E8616E6248D1830003F2FF136A6EEA625A
:1016B000B1EB532F40D3B5F868204FF0FF338021B2
:1016C000012AC5E9053329717FD003205149524AC7
:1016D00028700B88106801339BB285420B80EB8029
:1016E00004BF0023136013699D420BD100231361D3
:1016F00008E06878FFF7B0FCC3073FF574AF0FB19F
:1017000047071CD4002065E76C4605F5FB7305F21E
:10171000362021461A7902B19A6841F8042B103319
:101720008342F7D104F1100754F8046B032076B913
:10173000BC42F9D1042815D00D2005B0F0BD0A2017
:1017400048E70C2005B0F0BD0B2005B0F0BD3146D8
:101750002846FFF7E7FE0128EAD85FE7032039E7CC
:10176000E96D66E7012035E740F6F57CE6456E62F7
:101770002C63E861AB6216D8002FDDD01A4400F06C
:10178000010303F2FF1300EB400003EB5003B1EB46
:10179000532FEA62D0D34FF0FF338022C5E90533DF
:1017A0002A71012092E7002FC6D04000134400F2B6
:1017B000FF12B1EB522FEB62BED34FF0FF3380220A
:1017C000C5E905332A71022080E7711C2846FFF71E
:1017D0002DFE00287FF479AFB5F8361228714AF64D
:1017E000552291427FF471AFAA6B0C4B9A427FF461
:1017F0006CAF03F1FF53D5F81C2203F500532033DF
:101800009A427FF462AFD5E98832C5E905235CE7E7
:10181000D0460120CC460120AC4601205252614105
:101820002DE9F8430778022F04460D46164642D0AC
:10183000032F2ED0012F53D1836A01EB510803EB04
:101840005829436B99454ED100F1380708F1010939
:1018500015F00105C8F30808F1B24FEA592274D017
:1018600017F8083003F00F0343EA011307F80830B4
:101870000123E370A36A02EB0308636B98456ED102
:10188000C9F308094F44C6F3071301223B70E27005
:1018900023E0826A436B02EBD118984545D100F1F1
:1018A0003807AD0005F4FE7501227B5966F31B0372
:1018B0007B51E27011E0826A436B02EB112898457C
:1018C00022D100F138076D0005F4FF757A197E55B5
:1018D0000123C6F307265670E3700020BDE8F883A5
:1018E0000220BDE8F883FFF7C1FC0028F9D13B4690
:1018F00004F1380760784A463946FFF7CBFB0028E9
:101900004BD1C4F83490A1E7FFF7B0FC0028E8D130
:1019100004F138076078012342463946FFF7BAFBE5
:1019200000283AD1C4F83480CDE7FFF79FFC0028A7
:10193000D7D104F138076078012342463946FFF7D2
:10194000A9FB50BBC4F83480ABE707F808100123AB
:10195000E370A36A02EB0308636B434513D0204690
:10196000FFF784FC0028BCD1607801234246394649
:10197000FFF790FB88B9C9F30809C4F834804F44D5
:10198000002D80D102E0C9F308094F443B78C6F32B
:10199000032623F00F03334377E74FF0FF336363EE
:1019A00001209EE701292BD9C36999422DE9F04115
:1019B0000C46054602D30120BDE8F0810678022ED0
:1019C0002ED0032E1ED0012EF5D1836A01EB5107D4
:1019D000416B03EB572888452ED1C7F3080207F166
:1019E00001082A4403EB58278F4292F838605AD0F6
:1019F0002846FFF73BFC00284CD04FF0FF30DBE7D8
:101A000001207047866A436B06EBD1169E4233D1A4
:101A1000A40004F4FE742544A86B20F07040CBE7CA
:101A2000866A436B06EB11269E4217D1630003F4CE
:101A3000FF732B44188FBFE7FFF718FC0028DCD199
:101A400068783346424605F13801FFF723FB00284A
:101A500036D1AB6AC5F834804146BEE7FFF706FCD5
:101A60000028CAD168780123324605F13801FFF712
:101A700011FB28BB6E63D9E7FFF7F8FB0028BCD148
:101A800068780123324605F13801FFF703FBB8B946
:101A90006E63BDE7687801233A4605F13801FFF728
:101AA000F9FA68B96F63C8F308072F4497F838301C
:101AB00046EA0320E3074CBF0009C0F30B007BE7B5
:101AC0004FF0FF336B6398E70129F8B505680E46C0
:101AD00028D9EB698B4225D90746114622BB2846F7
:101AE00011E0FFF79DFEF0B9D5E90632911E8B4259
:101AF00005D22979013341F001012971AB61A2427C
:101B00001FD9386826463146FFF74CFF04460022AD
:101B100031462846ACB1012C04D0631C13D0EB69CC
:101B20009E42DED30220F8BD012AFBD09342F9D9B0
:101B30004FF0FF322846FFF773FE0028F3D13868D4
:101B4000E1E70020F8BD0120F8BD00BF2DE9F0411C
:101B500007680646884600294BD17D69FB699DB31D
:101B60009D4228BF01252C4606E001283DD00130CA
:101B700050D0AC424AD0FB6901349C4202D3012DC3
:101B800044D0022430682146FFF70CFF0028ECD136
:101B9000012C2AD9FB699C4227D24FF0FF32214603
:101BA0003846FFF73DFEF0B9B8F1000F0ED1D7E986
:101BB0000623023B9A427C6101D8013ABA613B7923
:101BC00043F001033B7111E00125CCE7B8F1010FAF
:101BD0000BD0FB69984508D2224641463846FFF7AC
:101BE0001FFE0028E3D0012814D001242046BDE8C0
:101BF000F0813846FFF7D6FE01280446F5D9431C8C
:101C000008D0FB698342F1D84546ACE70024204662
